:100000000C94380A0C94570A0C94570A0C94130C4D
:100010000C944D0C0C94570A0C94570A0C94570AE4
:100020000C94570A0C94570A0C94570A0C94570ACC
:100030000C94570A0C94570A0C94570A0C94670FA7
:100040000C94570A0C94570A0C94570A0C94570AAC
:100050000C9471770C941F6F0C94570A0C94570AE8
:100060000C94570A0C94F26F0C94570A0C94E66F98
:100070000C94570A0C94570A0C94570A0C94570A7C
:100080000C94CB870C94570A0C94570A0C94570A7B
:100090000C9430700C94570A0C9424700C94570AEA
:1000A0000C94570A0C94570A0C94570A0C94570A4C
:1000B0000C94570A0C94570A0C94570A0C94570A3C
:1000C0000C94570A0C94570A0C94570A0C94570A2C
:1000D0000C94570A0C94570A0C94570A0C94570A1C
:1000E0000C94570A0C942A770C9434770C9420774C
:1000F0000C94E0760C9465770C9456770C944A77C0
:100100000C943E770C94570A0C94570A0C94570A97
:100110000C94570A0C94570A0C94570A0C94570ADB
:1001200000911F9199918B92AB92CB92D392809236
:10013000084AD73B3BCE016E84BCBFFDC12F3D6C4E
:1001400074319ABD56833DDA3D00C77F11BED9E4B4
:10015000BB4C3E916BAAAABE000000803F076342E1
:1001600036B79BD8A71A39685618AEBAAB558C1D4E
:100170003CB7CC5763BD6DEDFD753EF6177231BFD0
:10018000000000803F08000000BE922449123EABF0
:10019000AAAA2ABECDCCCC4C3E00000080BEABAAA1
:1001A000AAAA3E00000000BF000000803F0000003F
:1001B0000000084178D3BB4387D1133D190E3CC3DF
:1001C000BD4282AD2B3E68EC8276BED98FE1A93E5E
:1001D0004C80EFFFBE01C4FF7F3F00000000000025
:1001E000256300256300496E76616C69642069327D
:1001F0006320737065656420696E20454550524FD9
:100200004D2E2053657474696E67203130206B6207
:1002100069742F730025730A005854414C5F54527F
:10022000494D3D25640025730A0025730A00546575
:10023000737420362025730A0054657374203520AA
:1002400025730A005465737420342025730A005402
:1002500065737420332025730A005465737420324B
:100260002025730A005465737420312025730A0019
:100270006368616E3D25640A0074787077723D256D
:10028000640A003530306B0A003235306B0A0031B9
:1002900031356B0A0035366B0A0033386B0A00259E
:1002A000730A00765F6C6F773D252D332E32660A18
:1002B0000025730A0073656E743D252D75206475E5
:1002C000703D252D752069676E6F7265643D252D23
:1002D000752074746C5F7A65726F3D252D750A0008
:1002E00025372E33662025372E33660025352E32EE
:1002F0006620004572726F72203020566F6C740059
:100300004E6F7420737570706F727465640A004567
:1003100072726F72203020566F6C74004572726F6B
:1003200072203020566F6C740062756C6B5F646570
:100330006C61793D252D750062756C6B3D252D75C1
:100340000056616C7565206E6F7420616C6C6F7700
:1003500065640062756C6B3A206D61783D2575208F
:1003600073746172743D25752C20656E643D25752E
:100370002C20696E5F7573653D25750A00706232C9
:100380003D25730A007062313D25730A00256C75A6
:1003900000416C6C6F776564207370656564203113
:1003A0002F31302F3130302F343030206B62697470
:1003B0002F730025630074746C3D252D6420007438
:1003C000746C3D252D6420004E65772074746C3D5F
:1003D000252D6420002563004D53353631312050E2
:1003E0003D252D372E326620252D372E32666D0A9B
:1003F00000424D5030383520256C642043200042A7
:100400004D5030383520256C642050612020252D3A
:10041000372E32666D00256300545F484541545FB6
:100420004944583D252D352E32662000545F444501
:10043000573D252D352E3266200041483D252D356E
:100440002E32662000545F53485432583D252D35D6
:100450002E3266200052485F53485432583D252DB5
:10046000352E32662000545F52483D252D342E3102
:1004700066200052483D252D342E3166200025632C
:100480000025630025630025630025630072657005
:100490006F72745F616C6C3D007265706F72743D59
:1004A00000256300256300256300256300204F536A
:1004B0004343414C3D2564200020467573653A2036
:1004C00065653D253032782068663D2530327820DC
:1004D0006C663D25303278206C623D2530327800E4
:1004E0004D43553D2530366C780025630074785FA8
:1004F0006C656E3D252D6C752C765F6C6F773D2598
:100500002D6C752C73687432783D252D6C752C62BA
:10051000756C6B3D252D6C75002563004F4B0A00F3
:1005200025630025630025630025630025630025FE
:10053000630025630025630064656275675F616C15
:100540006C3D0064656275673D0064656275673D7A
:100550000025730A00646565700A006E6F6E650A97
:1005600000707772733D007062323D25730A00702F
:1005700062313D25730A00696E74725F7365635F53
:1005800070313D252D372E33660A00696E74725F17
:1005900070313D252D6C640A00696E74725F73655D
:1005A000635F70303D252D372E33660A00696E7407
:1005B000725F70303D252D6C640A00765F6D637547
:1005C0003D252D352E32660A00745F6D63753D251D
:1005D0002D352E32660A00707077723D25730A0041
:1005E00064656275673D0072636D643D25730A0042
:1005F00025730A006175746F0A006C6F675F6D6F19
:1006000064653D007573625F7077723D25730A0003
:1006100072656C61793D25730A0074746C3D252DFB
:10062000640A0052494D455F616464723D252D6442
:100630002E252D640A006E65696768626F725F74AB
:1006400061626C655F73697A653D25640A00765F57
:100650006C6F773D252D332E32660A0074787077E3
:100660003D25640A006368616E3D25640A00696483
:100670003D006932635F6275733D006932635F7389
:10068000706565643D252D6C750A007478743D2590
:10069000730A0053797374656D2053756D6D6172C3
:1006A000790A002530366C780041744D65676132F7
:1006B0003536524652320041744D656761313238E9
:1006C000524652320041744D65676136345246528B
:1006D000320041744D656761313238524641310014
:1006E0004D43553D006D61736B3D002C00696E7488
:1006F000657276616C3D252D750023252D642C00D7
:10070000705F626D653238300072685F626D6532AD
:10071000383000745F626D653238300070623200CC
:1007200070623100745F686561745F696478007439
:100730005F64657700616800705F6D7335363131D5
:100740000072685F736874327800745F7368743223
:10075000780070610070006164340061643300618E
:100760006432006164310061330061320061310044
:10077000765F696E007268006572720075707469E8
:100780006D650070315F6C73740070315F74007060
:10079000310070305F6C73740070305F74007030C3
:1007A00000765F6D637500745F6D63750074310072
:1007B000740069640065363400747874002D002B71
:1007C000006175746F006E6F6E650062756C6B0012
:1007D000706F7765725F736176655F6C656472795F
:1007E0000072656C61795F6C65647900636F6D7030
:1007F00061737300616363656C0070726573007090
:100800005F707772006165730070315F6C65647949
:100810000070305F6C656472006576656E74006CA4
:100820006564006F7700706B740074785F6C65644A
:10083000790072785F6C656472006F706572006E2B
:100840006F6E65002530327800765F6164343D2537
:100850002D382E3666002000765F6164333D252DED
:10086000382E3666002000765F6164323D252D38D3
:100870002E3666002000765F6164313D252D382ECE
:100880003666002000765F6C696768743D252D38F8
:100890002E3666002000765F61323D252D372E33DF
:1008A00066002000765F61313D252D372E336600CE
:1008B0002000765F696E3D252D352E326600204E74
:1008C000657665722D7573656420737461636B2042
:1008D0003E2025642062797465730A00757074691E
:1008E0006D653D252D642D646179732D253032644D
:1008F0003A253032643A253032642D686F75727350
:100900000A0074657374205B6F66667C317C327C90
:10091000337C347C355D20202020202020202D2099
:1009200074657374206D6F6465730A0D00747820AC
:100930005B706B74207061796C6F61645D20202046
:100940002020202020202020202D2073656E642070
:10095000726164696F20706B74206B6579626F617E
:1009600072640A0D00776474205B6F6E7C6F66663C
:100970007C746573745D202020202020202020209E
:10098000202D207761746368646F670A0D00765FBD
:100990006C6F77205B765F6C6F775D202020202066
:1009A000202020202020202020202D206C6F776503
:1009B0007374207265706F727420766F6C746167E7
:1009C000650A0D00757067722020202020202020ED
:1009D0002020202020202020202020202020202017
:1009E0002D207265626F6F742076696120626F6F6F
:1009F000746C6F616465720A0D0075617274205BBE
:100A000033386B7C35366B7C3131356B7C3235302D
:100A10006B7C3530306B5D202D20736574207465E0
:100A2000726D2F756172742073706565640A0D00B4
:100A3000626F6F7420202020202020202020202082
:100A40002020202020202020202020202D20726502
:100A5000626F6F740A0D0070777273205B64656556
:100A6000707C6E6F6E655D2020202020202020206D
:100A70002020202D206D637520736C656570206DBE
:100A80006F64650A0D007265737420656570726F1E
:100A90006D20202020202020202020202020202009
:100AA00020202D20726573746F72652065657072E9
:100AB0006F6D0A0D0070707772205B6F6E7C6F66D1
:100AC000665D2020202020202020202020202020A3
:100AD000202D2070726F6772616D6D61626C652090
:100AE0007077720A0D0070623220205B6F6E7C6F2F
:100AF00066665D202020202020202020202020202D
:100B000020202D2070726F6772616D6D61626C655F
:100B10002070696E2062320A0D0070623120205B05
:100B20006F6E7C6F66665D202020202020202020B4
:100B30002020202020202D2062756C6B20475049FA
:100B40004F2070696E0A0D00747874205B737472A4
:100B5000696E675D2020202020202020202020207A
:100B6000202020202D20536574207265706F7274D0
:100B7000207465787420737472696E670A0D00744E
:100B8000787077205B31352D305D202020202020AB
:100B900020202020202020202020202D20545820DC
:100BA0005077722E2048696768657374203020285A
:100BB0003364426D290A0D0074746C205B302D3152
:100BC000355D2020202020202020202020202020D3
:100BD000202020202D2074696D652D746F2D6C6987
:100BE000766520666F72207061636B6574730A0DA1
:100BF000007373202020202020202020202020206F
:100C0000202020202020202020202020202D207384
:100C1000797374656D2073756D6D6172790A0D005D
:100C2000727320202020202020202020202020201F
:100C30002020202020202020202020202D20726114
:100C400064696F2073746174730A0D007269205BAC
:100C5000236E5D205B696E745D20202020202020A3
:100C600020202020202020202D207265706F72749B
:100C700020696E74657276616C0A0D0072636D6432
:100C8000205B6F6E7C6F66665D2020202020202018
:100C900020202020202020202D20616C6C6F7720C8
:100CA000636D642066726F6D206E65746F726B0A7F
:100CB0000D007265205B236E5D205B2B7C2D5D201B
:100CC0005B6D61736B7C6175746F2C6D61736B5DB3
:100CD000202D206D6F7465207265706F72742073A3
:100CE00065742F6D6F646966790A0D006F77202037
:100CF00020202020202020202020202020202020F4
:100D000020202020202020202D206F6E652D776947
:100D100072652073656E736F72730A0D006C6F6776
:100D2000205B6175746F7C6F6E7C6F66665D2020E2
:100D30002020202020202020202D206D6F7465731E
:100D40002064617461206F6E205553420A0D006E5D
:100D500065205B666C7573685D2020202020202054
:100D600020202020202020202020202D206E65699A
:100D70006768626F72207461626C650A0D0065724B
:100D80007220202020202020202020202020202011
:100D9000202020202020202020202D206572726F0E
:100DA000722073746174730A0D006D6375202020C6
:100DB0002020202020202020202020202020202033
:100DC0002020202020202D206D637520696E666F05
:100DD0000A0D00693263205B70726F62657C73700C
:100DE00065656420236E5D20202020202020202D9A
:100DF000206932632070726F6265206275737C7344
:100E00006574206275732073706565640A0D0069EE
:100E100064205B72657365745D2020202020202093
:100E200020202020202020202020202D2069642028
:100E300068616E646C696E670A0D0068756D2020CC
:100E400020202020202020202020202020202020A2
:100E5000202020202020202D2068756D6964697471
:100E6000792073656E736F720A0D0072656C61791B
:100E7000205B6F6E7C6F66667C73746174735D203B
:100E8000202020202020202D2072656C6179206E8A
:100E90006574776F726B207265706F7274730A0D70
:100EA000006465205B6D61736B5D20202020202035
:100EB000202020202020202020202020202D2064E1
:100EC000656275670A0D006368616E205B31312DC4
:100ED00032365D20202020202020202020202020AD
:100EE0002020202D206368616E2031312D32362084
:100EF00028322E3430352D32343830204D687A295E
:100F00000A0D0063616C69205B5B765F696E7C61D2
:100F1000317C61325D20766F6C747C7265736574B0
:100F20007C6E6F6E655D202D2063616C69627261FD
:100F300074650A0D0062756C6B205B5B73686F777C
:100F40007C666C7573685D205B7365742074687271
:100F500073682064656C61795D5D20202D20627569
:100F60006C6B696E67207061636B657473200A0D2A
:100F700000616463202020202020202020202020C9
:100F8000202020202020202020202020202D207301
:100F9000686F7720765F696E2C2061312C2061327A
:100FA00020766F6C74616765730A0D0075202020D0
:100FB0002020202020202020202020202020202031
:100FC00020202020202020202D20757074696D6540
:100FD0000A0D007620202020202020202020202004
:100FE0002020202020202020202020202020202DF4
:100FF0002076657273696F6E0A0D006820202020CC
:1010000020202020202020202020202020202020E0
:10101000202020202020202D2068656C700A0D00E3
:10102000256300756E6B6E6F776E20636D640A00CA
:10103000484D43353838330025730025730020258B
:1010400073002025362E3266200025303278007459
:10105000656D705F65787465726E3D252D362E3234
:101060006600202573002025362E3266204F6E2D17
:10107000426F61726400253032780074656D705F74
:10108000626F6172643D252D362E3266000A004281
:10109000756C6B2072656D3A2073746172743D25B6
:1010A000752C20656E643D25752C20696E5F757307
:1010B000653D25750A0042756C6B206164643A20B9
:1010C00073746172743D25752C20656E643D2575C1
:1010D0002C20696E5F7573653D25750A0042756C3D
:1010E0006B207468726573683A2074696D65723D2F
:1010F00025750A00503A20256C6420506120202577
:101100002D372E3266206D0A004932433A200045C1
:101110002025642E256420636C6F636B20256C751D
:101120002063707520256C75206C706D20256C75A2
:101130002069727120256C7520676C656420256CB0
:101140007520796C656420256C7520726C6564204F
:10115000256C7520747820256C75206C6973746516
:101160006E20256C752073656E736F727320256C0D
:10117000752073657269616C20256C750A005320B7
:1011800025642E256420636C6F636B20256C7520AD
:10119000747820256C7520727820256C7520727407
:1011A0007820256C752072727820256C7520726508
:1011B000786D697420256C752061636B74782025C7
:1011C0006C75206E6F61636B747820256C7520617F
:1011D000636B727820256C752074696D65646F751A
:1011E0007420256C752062616461636B72782025C0
:1011F0006C7520746F6F6C6F6E6720256C75207432
:101200006F6F73686F727420256C752062616473F0
:10121000796E636820256C75206261646372632057
:10122000256C7520636F6E74656E74696F6E647281
:101230006F7020256C752073656E64696E676472CB
:101240006F7020256C75206C6C747820256C75206F
:101250006C6C727820256C750A00257325730A0062
:101260004F6E6C696E650A000A002C206368656326
:101270006B207261746520257520487A00257320E3
:1012800025732C206368616E6E656C202575207057
:101290006F776572202575000A0025783A004D4168
:1012A000432061646472657373200052616E646FE1
:1012B0006D2045554936342061646472657373202E
:1012C00067656E6572617465640A000A2A2A2A2AB3
:1012D0002A2A2A426F6F74696E672025732A2A2A88
:1012E0002A2A2A2A0A00454550524F4D2069732068
:1012F000636F72727570742C20726577726974698D
:101300006E6720776974682064656661756C7473B4
:101310002E0A006C6F63616C686F73740041544DEA
:101320004547413132387266613100020000FFFEEC
:101330000000016E616E00696E660000407A10F375
:101340005A00A0724E18090010A5D4E80000E876F3
:1013500048170000E40B54020000CA9A3B0000004A
:10136000E1F505000080969800000040420F000063
:1013700000A08601000000102700000000E8030024
:101380000000006400000000000A000000000001EE
:1013900000000000002C76D888DC674F0823DFC1EE
:1013A000DFAE59E1B1B796E5E3E453C63AE65199A9
:1013B0007696E8E6C28426EB898C9B62ED407C6FD2
:1013C000FCEFBC9C9F40F2BAA56FA5F490055A2A89
:1013D000F75C936B6CF9676DC11BFCE0E40D47FE95
:1013E000F520E6B500D0ED902E030094357705008A
:1013F00080841E080000204E0A000000C80C333311
:1014000033330F986E12831141EF8D2114893BE61F
:101410005516CFFEE6DB18D1844B381BF77C1D90A8
:101420001DA4BBE424203284725E228100C9F12411
:10143000ECA1E53D274E414E494E495459494E468F
:10144000CDCCCC3D0AD7233C17B7D13877CC2B3243
:101450009595E6241FB14F0A000020410000C842C4
:1014600000401C4620BCBE4CCA1B0E5AAEC59D7423
:1014700011241FBECFEFD1E4DEBFCDBF1AE0A0E044
:10148000B2E0EEE5FCE401E00BBF02C007900D9274
:10149000A83DB107D9F72EE3A8EDBAE001C01D922F
:1014A000A433B207E1F70E94A2930C942DA60C94EA
:1014B00000008115910511F00197F1F7089581E67B
:1014C00095E09F938F930E940CA38091620290916C
:1014D0006302A0916402B09165020F900F9093FF98
:1014E00003C08BE595E002C085E595E09F938F935F
:1014F0000E940CA30F900F900895E091C51CEF730C
:10150000F0E0EA5EF24E80838091C51C8F5F80938D
:10151000C51C8091723588608093723548E452E032
:1015200061E1CA010E94DE5E80E090E00895CF9301
:10153000DF93EC018091E30A9091E40AA091E50A1F
:10154000B091E60A86FF1DC08E811F928F938D8118
:101550001F928F938C811F928F938B811F928F93F9
:101560008A811F928F9381E793E09F938F930E94CC
:10157000F8A28DB79EB70C960FB6F8949EBF0FBE1B
:101580008DBFBE0184E29BE00E941260BE0184E038
:1015900092E0DF91CF910C94865F52985A981DBAD1
:1015A000E9E6F0E0808180628083EA9A53985B9854
:1015B000EB9A808180688083E8E6F0E0808181603A
:1015C00080830895EBE7FDE1118212821082089575
:1015D000CF92DF92EF92FF920F931F93CF93DF93FF
:1015E000EC019B0180917B1D843108F0BBC0809190
:1015F0007D1D64E10E94EA9B90937D1DC090983010
:10160000D0909930E0909A30F0909B30092F10E004
:101610008DE8989FD0011124A558B24E1396CD9213
:10162000DD92ED92FC9216974115510559F0FA01A1
:101630008081FD01EA57FF4F8083FA018181A9571C
:10164000BF4F8C932097A9F089819DE8909FF0016E
:10165000919FF00D1124E558F24EDF01A657BF4FC0
:101660008C93E557FF4F88818F70808388818F70BE
:10167000808321153105E1F1D90116964C91169719
:101680005DE8509FC001519F900D11248558924EE6
:10169000FC01E757FF4F408315964C911597319702
:1016A000408334961B964D915D916D917C911E9770
:1016B000452F562F672F7727518340837C01BEE843
:1016C000EB0EF11CF9012385348545855685A4E68A
:1016D000B0E00E948D9C672F782F892F992724E6F0
:1016E00030E040E050E00E941E9CD7016D937C9357
:1016F0008DE8809FD001819FB00D1124AE57B24E6E
:10170000FE0132968FE701900D928A95E1F7809164
:101710007D1D8F5F80937D1D90917B1D9F5F9093BA
:101720007B1D4091E30A5091E40A6091E50A7091B3
:10173000E60A60FF2DC01F929F931F928F938091A6
:101740007C1D1F928F9386EB90E19F938F930E9455
:101750000CA3EDB7FEB738960FB6F894FEBF0FBED8
:10176000EDBF16C08091A8309091A930A091AA3009
:10177000B091AB300196A11DB11D8093A83090931C
:10178000A930A093AA30B093AB3080E090E002C0C3
:1017900081E090E0DF91CF911F910F91FF90EF904A
:1017A000DF90CF90089520917B1D222361F18091DD
:1017B0007C1D8F5F215020937B1D64E10E94EA9B7A
:1017C00090937C1D4091E30A5091E40A6091E50AF0
:1017D0007091E60A60FF1AC01F922F9380917D1DC1
:1017E0001F928F931F929F938FE890E19F938F9307
:1017F0000E940CA38DB79EB708960FB6F8949EBFB3
:101800000FBE8DBF03C080E090E0089581E090E0BE
:10181000089581110C94CD0A109269005A9AEA98A1
:101820005B9AEB9808951F920F920FB60F921124B6
:101830008F939F93AF93BF938091680080FF24C0E4
:101840008091413590914235A0914335B091443516
:101850000196A11DB11D8093413590934235A0930F
:101860004335B09344358091E30A9091E40AA09106
:10187000E50AB091E60A87FF07C0749882E090E01D
:1018800090938F0280938E02BF91AF919F918F9121
:101890000F900FBE0F901F9018951F920F920FB6CA
:1018A0000F9211248F939F93AF93BF938091680001
:1018B00080FF24C08091453590914635A0914735F1
:1018C000B09148350196A11DB11D80934535909387
:1018D0004635A0934735B09348358091E30A9091FF
:1018E000E40AA091E50AB091E60A90FF07C0739858
:1018F00082E090E090938F0280938E02BF91AF912F
:101900009F918F910F900FBE0F901F90189580930D
:101910007C0080917B00877F80937B0080917C009E
:10192000806C80937C0085E080937A0080917A00BF
:10193000806880937A0080917B0087FFFCCF809144
:101940007B0085FFFCCF80917A00806480937A00D1
:1019500080917A0086FDFCCF109279001092780079
:1019600084E090E060E070E020917A0020642093B1
:101970007A0020917A0026FDFCCF209178003091EA
:101980007900620F731F019779F710927C008091A4
:101990007A008F7780937A0076956795769567952C
:1019A00080E090E00E941199089580E00E94870CE9
:1019B00020918602309187024091880250918902DD
:1019C0000E940B9B21EE3AE744E95EE30E947C977C
:1019D00008950F931F93CF93DF930FE110E0CBE5B2
:1019E000DEE00093510187EC90E00E94590A80915B
:1019F000510185FD0DC00031110521F02CF0CB54B3
:101A0000D10903C0C4ECD9E0E29701501109E9CF34
:101A1000BE0180E090E00E94119920E030E04AE7AA
:101A200054E40E945F98DF91CF911F910F91089528
:101A3000CF93DF93EC0188819981009799F08237E9
:101A4000924121F01982188283E011C0623171F451
:101A50000E94E90C60939430709395308093963097
:101A60009093973082E792E19983888381E0DF91B8
:101A7000CF91089580917B00886080937B0089ECF2
:101A800080937C0085E080937A0080917A00806862
:101A900080937A0080917B0087FFFCCF80917B0050
:101AA00085FFFCCF80917A00806480937A008091DA
:101AB0007A0086FDFCCF80917A00806480937A0062
:101AC00080917A0086FDFCCF60917800709179005A
:101AD00080917A008F7780937A0080E090E00E9476
:101AE000119927ED33EA40E95FE30E940B9B26E65C
:101AF00036E648E853E40E947B970895CF92DF9240
:101B0000EF92FF921F93CF93DF93CDB7DEB7299764
:101B10000FB6F894DEBF0FBECDBF6C011092DC0A89
:101B20008FEF89878EECE82E8CE1F82E10E0898506
:101B30008823E9F11830D9F1BE016F5F7F4FCE01E4
:101B400009960E94616899859F3F11F09E3F19F4A4
:101B50009093DC0A2CC0CE010196C114D10481F40B
:101B60000E947B6880936335ABE5B5E3FE01319657
:101B700088E08E0F91919D938E13FCCF81E018C069
:101B80000E947B68F7018087FE01319620E030E0FB
:101B90008191D701A20FB31F8C932F5F3F4F283045
:101BA0003105B1F71F5FF9E0EF0EF11CC0CF812FB7
:101BB00029960FB6F894DEBF0FBECDBFDF91CF914F
:101BC0001F91FF90EF90DF90CF9008958DE890E106
:101BD0009F938F930E940CA30F900F9008952F92C4
:101BE0003F924F925F926F927F928F929F92AF92AD
:101BF000BF92CF92DF92EF92FF920F931F93CF93FA
:101C0000DF93EC015B01009711F427E003C001971B
:101C100049F426E04AE250E06BE270E089E290E0AD
:101C20000E943B67CE010E947E0D9E012352354FDC
:101C30006901D9018C93CD2B69F0CEECDCE1E12C6C
:101C4000F12C82E4282E80E1382E9EE3892E90E14B
:101C5000992E9EC08BE595E30E94AA69BC01990F5D
:101C6000880B990B0E9413996B017C01AB2869F0DA
:101C700020E030E048EC52E40E945F989F938F93FD
:101C80007F936F938BE790E1A4C0CBE5D5E306E7A4
:101C900010E189911F928F931F930F930E940CA3C1
:101CA0000F900F900F900F90B5E3C336DB0789F7C5
:101CB00020E030E048EC52E4C701B6010E945F9892
:101CC0009F938F937F936F9386E690E19F938F937B
:101CD0000E940CA30F900F900F900F900F900F90F9
:101CE00080916335811103C082E294E002C080EAF2
:101CF00093E09F938F9382E690E19F938F930E944E
:101D00000CA30F900F900F900F906DC000E010E0AB
:101D1000FE01E00FF11F80811F928F93AAE4B0E1D2
:101D2000BF93AF930E940CA30F5F1F4F0F900F90B4
:101D30000F900F900830110559F720E030E048EC83
:101D400052E4C301B2010E945F989F938F937F93E7
:101D50006F933F922F920E940CA30F900F900F90C1
:101D60000F900F900F908885811151C082E294E00E
:101D70009F938F939F928F920E940CA30E94E60DD7
:101D8000FFEFEF1AFF0A29960F900F900F900F9018
:101D9000D6018C9190E0E816F906E4F5CE010E9498
:101DA000AA69BC01990F880B990B0E9413992B010A
:101DB0003C01A114B10409F4A9CF20E030E048ECC3
:101DC00052E40E945F989F938F937F936F938FE469
:101DD00090E19F938F930E940CA30F900F900F9010
:101DE0000F900F900F90DF91CF911F910F91FF9067
:101DF000EF90DF90CF90BF90AF909F908F907F90AB
:101E00006F905F904F903F902F900C94E60D80EA7A
:101E100093E0AECFDF91CF911F910F91FF90EF90A4
:101E2000DF90CF90BF90AF909F908F907F906F90FA
:101E30005F904F903F902F900895CF93DF9300D005
:101E4000CDB7DEB7EBE5F5E38181898387818A83AE
:101E5000CE0101960E94CD5C0F900F90DF91CF9143
:101E60000895CF93DF93EC0120915B3530915C3581
:101E700040915D3550915E3560915F357091603570
:101E80008091613590916235AFEF0E94599EE1F4E7
:101E900027E04AE250E06BE270E089E290E00E94C5
:101EA0003B6780E090E00E947E0DC352D54F88834F
:101EB00049E050E06EE070E08BE595E30E9410A6EB
:101EC000DF91CF910C941D0FDF91CF9108951F9258
:101ED0000F920FB60F9211240BB60F92FF920F9331
:101EE0001F932F933F934F935F936F937F938F93A2
:101EF0009F93AF93BF93CF93DF93EF93FF93809123
:101F000072358260809372358091620286FD2B9AD1
:101F10008091620287FD2B9A80918E0290918F02B0
:101F20001816190614F4749A739A8091E30A909122
:101F3000E40AA091E50AB091E60A85FF02C0749810
:101F4000739880910202909103020197909303028B
:101F500080930202892B09F04CC18091F30A909181
:101F6000F40A01969093F40A8093F30A80919830D2
:101F700090919930A0919A30B0919B300196A11D1B
:101F8000B11D8093983090939930A0939A30B0937C
:101F90009B3080E190E09093030280930202809155
:101FA000620280FD02C01D9B05C01092E10A1092E2
:101FB000E00A06C081E090E09093E10A8093E00A95
:101FC0008091E30A9091E40AA091E50AB091E60AB3
:101FD00097FF08C08091E00A9091E10A892B49F0AF
:101FE000749A739805E71CE1CDEAD0E3FF24F394DB
:101FF00021C0739A7498F6CF8091F30A9091F40AF5
:1020000001960E94F69B892BE1F0F80160857185AD
:1020100061157105A1F5F80160857185611571057E
:1020200009F03FC0065F1F4F2596F0E3C13CDF0774
:1020300009F44CC0F801608571856115710529F3BB
:10204000DBCF4281417020E030E050E060E070E0A2
:1020500080E090E0A0E00E94599EB9F277988091CC
:10206000E30A9091E40AA091E50AB091E60A92FF92
:10207000CCCF749810928F0210928E02C6CF8091AE
:10208000F30A9091F40A01960E94F69B892B19F6A7
:102090001C821B82AE0162E180E292E00E94DE5E61
:1020A000BACF8091F30A9091F40A0E94F69B892B93
:1020B00009F0B8CFF8821A8309831C821B82AE0113
:1020C00062E18EE392E00E94DE5EACCF6091680236
:1020D0007091690261157105A1F18091F30A9091E7
:1020E000F40A0E94F69B892B61F58091413590910D
:1020F0004235A0914335B091443540918A285091A2
:102100008B2860918C2870918D28841B950BA60BD1
:10211000B70B80939D1C90939E1CA0939F1CB09323
:10212000A01C8091413590914235A0914335B091EA
:10213000443580938A2890938B28A0938C28B09361
:102140008D28609166027091670261157105A1F199
:102150008091F30A9091F40A0E94F69B892B61F515
:102160008091453590914635A0914735B0914835DD
:1021700040918E2850918F286091902870919128DD
:10218000841B950BA60BB70B8093A11C9093A21CEC
:10219000A093A31CB093A41C809145359091463523
:1021A000A0914735B091483580938E2890938F2821
:1021B000A0939028B09391288091620286FD2B987D
:1021C0008091620290916302A0916402B0916502D5
:1021D00091FF0FC00E94A2738A3119F0C1E0C80FAD
:1021E00001C0CBE00E9458728C2F0E94BA730E94EB
:1021F000A07240E050E060E080E992E00E94DE5E84
:10220000FF91EF91DF91CF91BF91AF919F918F910E
:102210007F916F915F914F913F912F911F910F91FE
:10222000FF900F900BBE0F900FBE0F901F90189550
:102230008091C51C9091AC30891B08950E941811A3
:10224000882371F0E091AC30EF73F0E0EA5EF24E7B
:10225000808190E02091AC302F5F2093AC300895C6
:102260008FEF9FEF0895CF93DF93EC011092180B3F
:102270001092170B888199810097C1F08D3E934091
:1022800021F01982188283E0BDC0613109F0B9C024
:102290000E941E1199279093130B8093120B8D307F
:1022A000910509F444C08F3F910549F40E9418112B
:1022B0008111EECF8DEE93E099838883A2C08231A5
:1022C000910509F45AC08F37910509F052C08091E9
:1022D000100B9091110B181619060CF560912E3EFB
:1022E00070912F3E88E090E00E94C0A260912E3E47
:1022F00070912F3E80E290E00E94C0A260912E3E3D
:1023000070912F3E88E090E00E94C0A28091100B57
:102310009091110B01979093110B8093100B80916A
:10232000100B9091110B8F37910509F0BFCF1092D0
:10233000AC301092C51C8091100B9091110BFC01D8
:10234000EF53FF4C10829093180B8093170B109251
:10235000110B1092100B80916435909165350097A8
:1023600009F4A4CF40E050E0609126130E94DE5EA5
:102370009DCF8830910571F5AACF60912E3E709166
:102380002F3E8DE090E00E94C0A210920F0B1092A1
:102390000E0B20910E0B30910F0B8091100B909132
:1023A000110B281739070CF0BACFF901EF53FF4C86
:1023B000808160912E3E70912F3E90E00E94C0A2DD
:1023C00080910E0B90910F0B019690930F0B8093C1
:1023D0000E0BDFCF60912E3E70912F3E0E94C0A267
:1023E0002091100B3091110B8091120BF901EF53DA
:1023F000FF4C80832F5F3F4F3093110B2093100BC6
:102400008ECF81E0DF91CF9108958091E00A909185
:10241000E10A892BD1F08091620290916302A09130
:102420006402B091650293FD10C00E94587283B798
:10243000817F866083BFF89483B7816083BF78947F
:10244000889583B78E7F83BF78940895CF93DF9369
:10245000FC01208131812115310519F0293A3241E1
:10246000A1F4EC010E9415710E94051240E050E0B9
:1024700065E880912A1390912B130E94DE5E89EA11
:1024800092E19983888381E004C0FC01118210826B
:1024900083E0DF91CF910895CF93DF9300D0CDB744
:1024A000DEB7892B81F05F934F938BE390E19F938D
:1024B0008F9369837A830E940CA30F900F900F90E3
:1024C0000F907A8169817F936F9388E390E19F9366
:1024D0008F930E940CA30F900F900F900F900F906E
:1024E0000F90DF91CF910895CF93DF9300D0CDB7B8
:1024F000DEB74A8369830E94686A6981862F0E94D9
:10250000996A4A81842F0E94996A0F900F90DF91F7
:10251000CF910C94916AAF92BF92CF92DF92EF92DB
:10252000FF920F931F93CF93DF9300D01F92CDB7ED
:10253000DEB7182F022F4A835B8369830E94686A83
:102540006981862F0E94996A812F81600E948F6A1B
:102550004A81A42E5B81B52E10E0E12CF12C68019C
:1025600081E0C81AD108E016F10689F0EC14FD04E8
:1025700019F40E94B46A02C00E94AA6AF50180831D
:10258000FFEFEF1AFF0A8FEFA81AB80AECCF0F90EF
:102590000F900F90DF91CF911F910F91FF90EF90CF
:1025A000DF90CF90BF90AF900C94916ACF92DF9262
:1025B000EF92FF920F931F93CF93DF931F92CDB7AC
:1025C000DEB70E94157180EB0E94346A81111CC035
:1025D0000E94916A8091922C9091932C81609093AB
:1025E000932C8093922C89EA93E09F938F9388E3B6
:1025F00090E19F938F930E940CA30F900F900F90E8
:102600000F9001E010E002C000E010E08EB1847095
:10261000F82E729A62E174E380E090E00E94116A01
:102620000E9415718EE40E94346A811117C00E94C5
:10263000916A8091922C9091932C82609093932C2C
:102640008093922C68018FEFC81AD80A4EE35AE0A3
:1026500061EB73E0C8010E944C128601F11001C0C9
:10266000729862E174E380E090E00E94116A0E9437
:1026700015718EEE0E94346A811159C019820E9430
:10268000916A21E030E0AE014F5F5F4F60ED70E096
:102690008EEE90E00E948B1289818535A9F480919D
:1026A000922C9091932C84609093932C8093922CF5
:1026B00078018FEFE81AF80A4EE35AE069EB73E00D
:1026C000C8010E944C12870189818835A9F4809144
:1026D000922C9091932C80619093932C8093922CC8
:1026E00078018FEFE81AF80A4EE35AE060EC73E0E5
:1026F000C8010E944C12870189818036C1F4809103
:10270000922C9091932C80629093932C8093922C96
:1027100078018FEFE81AF80A4EE35AE067EC73E0AD
:10272000C8010E944C1281E00E940778870162E193
:1027300074E380E090E00E94116A0E94157186EABD
:102740000E94346A811117C00E94916A8091922C74
:102750009091932C80649093932C8093922C780189
:102760008FEFE81AF80A4EE35AE06EEC73E0C80106
:102770000E944C12870162E174E380E090E00E94C5
:10278000116A0E9415718CE30E94346A81111FC086
:102790000E94916A8091922C9091932C80689093E2
:1027A000932C8093922C78018FEFE81AF80A4EE36D
:1027B0005AE066ED73E0C8010E944C1280E390E19C
:1027C0009F938F930E940CA30F900F90870162E15B
:1027D00074E380E090E00E94116A0E94157182ED1E
:1027E0000E94346A811117C00E94916A8091922CD4
:1027F0009091932C91609093932C8093922C7801DC
:102800008FEFE81AF80A4EE35AE06EED73E0C80164
:102810000E944C12870162E174E380E090E00E9424
:10282000116A0E94157180E80E94346A811117C0F4
:102830000E94916A8091922C9091932C9860909331
:10284000932C8093922C78018FEFE81AF80A4EE3CC
:102850005AE067EE73E0C8010E944C12870162E102
:1028600074E380E090E00E94116A0E94157180ED8F
:102870000E94346A811117C00E94916A8091922C43
:102880009091932C94609093932C8093922C780148
:102890008FEFE81AF80A4EE35AE06DEE73E0C801D4
:1028A0000E944C12870162E174E380E090E00E9494
:1028B000116A0E9415718CEE0E94346A811117C052
:1028C0000E94916A8091922C9091932C90619093A8
:1028D000932C8093922C78018FEFE81AF80A4EE33C
:1028E0005AE065EF73E0C8010E944C12870187E04F
:1028F000E82EF12C62E174E380E090E00E94116A1E
:102900000E9415718CE70E94346A811113C00E94E5
:10291000916A8091922C9091932C92609093932C39
:102920008093922C4EE35AE06CEF73E0C8010E9452
:102930004C1204C081E0E81AF108E1F60E94916AA5
:102940000E94E60D0F90DF91CF911F910F91FF90A4
:10295000EF90DF90CF900895BF92CF92DF92EF92E9
:10296000FF920F931F93CF93DF93CDB7DEB760979E
:102970000FB6F894DEBF0FBECDBFF82EE42E66234F
:10298000D9F18E010F5F1F4F80E1F80111928A95F6
:10299000E9F728E0A80168E980EB0E948B12FF208C
:1029A00041F085E094E09F938F930E94F8A20F90EE
:1029B0000F902CE0C22E24E0D22E37E0B32EB00EC2
:1029C000F80181918F011F928F93DF92CF920E9425
:1029D000F8A20F900F900F900F90B012F1CF888552
:1029E0001F928F9381E694E09F938F930E94F8A2A9
:1029F0000F900F900F900F90EE20D9F18E010F5F86
:102A00001F4F80E1F80111928A95E9F720E1A801B2
:102A100060E880EB0E948B12FF2041F081E194E09E
:102A20009F938F930E94F8A20F900F908CE0E82E56
:102A300084E0F82E9FE0D92ED00EF80181918F010D
:102A40001F928F93FF92EF920E94F8A20F900F9027
:102A50000F900F90D012F1CF88891F928F9381E64B
:102A600094E09F938F930E94F8A20F900F900F9085
:102A70000F9060960FB6F894DEBF0FBECDBFDF910A
:102A8000CF911F910F91FF90EF90DF90CF90BF906B
:102A900008950F931F93CF93DF9300D0CDB7DEB788
:102AA0001A82198222E0AE014F5F5F4F6AEA8EEE12
:102AB0000E948B1206E51DE1898190E0982F8827FE
:102AC0002A81822BF8019183808322E0AE014F5F3F
:102AD0005F4F6CEA8EEE0E948B12898190E0982FF6
:102AE00088272A81822BF8019383828322E0AE011A
:102AF0004F5F5F4F6EEA8EEE0E948B12898190E0ED
:102B0000982F88272A81822BF8019583848322E0DD
:102B1000AE014F5F5F4F60EB8EEE0E948B1289819A
:102B200090E0982F88272A81822BF801938B828B43
:102B300022E0AE014F5F5F4F62EB8EEE0E948B1280
:102B4000898190E0982F88272A81822BF801958B24
:102B5000848B22E0AE014F5F5F4F64EB8EEE0E94EC
:102B60008B12898190E0982F88272A81822BF80187
:102B7000978B868B22E0AE014F5F5F4F66EB8EEE48
:102B80000E948B12898190E0982F88272A81822BBE
:102B9000F8019783868322E0AE014F5F5F4F68EBB9
:102BA0008EEE0E948B12898190E0982F88272A81CF
:102BB000822BF8019187808722E0AE014F5F5F4F43
:102BC0006AEB8EEE0E948B12898190E0982F882705
:102BD0002A81822BF8019587848722E0AE014F5F1E
:102BE0005F4F6CEB8EEE0E948B12898190E0982FE4
:102BF00088272A81822BF8019787868722E0AE01F9
:102C00004F5F5F4F6EEB8EEE0E948B12898190E0DA
:102C1000982F88272A81822BF801918B808B0F9027
:102C20000F90DF91CF911F910F9108952F923F92B6
:102C30004F925F926F927F928F929F92AF92BF92CC
:102C4000CF92DF92EF92FF920F931F93CF93DF9378
:102C5000CDB7DEB76C970FB6F894DEBF0FBECDBF11
:102C6000182F042F2D8B19821A821B8280917A1DB6
:102C7000811107C06C8F0E94491581E080937A1DF5
:102C80006C8D662309F472C04EE264EF8EEE0E94F2
:102C9000741269E07AE180E090E00E94116A22E01B
:102CA000AE014F5F5F4F66EF8EEE0E948B1229815F
:102CB000822F90E0A0E0B0E04427582F692F7A2FB0
:102CC0008A81482B80916C1D90916D1D9A01AB01FA
:102CD000281B390B41095109A0916A1DB0916B1D48
:102CE0000E948D9C6B017C013FE0F594E794D794A2
:102CF000C7943A95D1F76091641D7091651DCB0121
:102D0000770FAA0BBB0BBC01CD014BE0660F771F01
:102D1000881F991F4A95D1F72091661D3091671D34
:102D20004901330FAA08BB08A7019601280D391DD8
:102D30004A1D5B1D0E94409CC20ED31ED092611D95
:102D4000C092601D28E0C20ED11C54E0D594C794F7
:102D50005A95E1F70D2C000CEE08FF08C0926E1D8D
:102D6000D0926F1DE092701DF092711D812F82959F
:102D7000880F880F807C8C5C8887212E312CA3E003
:102D8000B0E0012E02C0AA0FBB1F0A94E2F725E3B0
:102D900035E00E94869C9B01AC012E5F3F4F4F4F58
:102DA0005F4F29873A874B875C8780E593ECA0E0EB
:102DB000B0E09C01AD0104C0559547953795279526
:102DC0001A95D2F7298B3A8B4B8B5C8B10E0412CF8
:102DD000512C320188E090E0AC01421953095B8F1D
:102DE0004A8F101709F43EC1488564EF8EEE0E94A9
:102DF000741269857A858B859C850E94116A23E00F
:102E0000AE014F5F5F4F66EF8EEE0E948B12E09136
:102E1000601DF091611DE05AFF409F01DF010E949B
:102E20006F9C6C837D838E839F838091581D9091CE
:102E3000591D9E878D872091561D3091571D388BC7
:102E40002F8720915A1D30915B1D0E946F9C6B0152
:102E50007C01ADE0F594E794D794C794AA95D1F797
:102E6000A0915C1DB0915D1D2C813D814E815F81E3
:102E70008CE055954795379527958A95D1F70E940F
:102E8000989CBB2797FDB095AB2F8C0D9D1DAE1D5B
:102E9000BF1D0296A11DB11D32E0B595A79597956E
:102EA00087953A95D1F79C01AD0130584F4F5F4F50
:102EB000A091681DB091691D0E948D9C4B015C0121
:102EC0004FE0B694A794979487944A95D1F73981A7
:102ED0008A8190E0A0E0B0E0BA2FA92F982F882730
:102EE000A32B2B81822B9C01AD010A8C04C055952C
:102EF0004795379527950A94D2F72E8B3F8B488FAD
:102F0000598F4F8558896A01550FEE08FF0862E016
:102F1000CC0CDD1CEE1CFF1C6A95D1F7A0915E1D48
:102F2000B0915F1D2C813D814E815F810E94989CF4
:102F30009B01AC0177E155954795379527957A9593
:102F4000D1F72C833D834E835F832D853E85DF0142
:102F50000E946F9CDC01CB01EBE0B595A79597959E
:102F60008795EA95D1F72C813D814E815F81820F53
:102F7000931FA41FB51FC80ED91EEA1EFB1E022CEC
:102F800004C0CC0CDD1CEE1CFF1C0A94D2F732E00E
:102F9000C30ED11CE11CF11CF2E0F594E794D79428
:102FA000C794FA95D1F72E893F89488D598D2C19F0
:102FB0003D094E095F0969897A898B899C890E943C
:102FC000DA9B97FD0BC0660F771F881F991FA5011D
:102FD00094010E941E9C69017A010AC0A501940116
:102FE0000E941E9C69017A01CC0CDD1CEE1CFF1CAA
:102FF0009927F7FC9A958F2D7E2D6D2D9B01AC01A5
:103000000E94DA9B9B01AC01AEEDBBE00E948D9C5F
:103010004C01BB2497FCB094AB2CA3E4B3EEA70106
:1030200096010E949B9CBB2797FDB095AB2F880E05
:10303000991EAA1EBB1E4FEC840E4EE0941EA11CCE
:10304000B11C44E0B594A794979487944A95D1F71E
:10305000C80CD91CEA1CFB1C4C0C5D1C6E1C7F1C94
:103060001F5FBFCE112381F0212F30E040E050E000
:10307000C301B2010E941E9C2093721D3093731DE8
:103080004093741D5093751D5D89552389F160919E
:10309000721D7091731D8091741D9091751D611545
:1030A00071058105910521F10E94139920E836EE02
:1030B00045EC57E40E945F9821E03EED42E45EE378
:1030C0000E94789B9B01AC0160E070E080E89FE388
:1030D0000E947B972BE43AE34DEB57E30E945F9805
:1030E0006093761D7093771D8093781D9093791D62
:1030F0006C960FB6F894DEBF0FBECDBFDF91CF91B7
:103100001F910F91FF90EF90DF90CF90BF90AF9005
:103110009F908F907F906F905F904F903F902F90F7
:1031200008950F931F93CF93DF9300D000D000D06A
:10313000CDB7DEB78E010F5F1F4F86E0F801119209
:103140008A95E9F780916C1C811113C040E061E31E
:1031500086EA0E9474124AE06CE286EA0E947412C7
:1031600081E080936C1C6CE77EE380E090E00E943D
:10317000116A48E06DE286EA0E9474126CE77EE311
:1031800080E090E00E94116A26E0A80162E386EAEE
:103190000E948B1247E06DE286EA0E9474128A81D7
:1031A00090E0982F88272981822B9093671C809329
:1031B000661C2C8130E0322F22274B81242B309348
:1031C000691C2093681C4E8150E0542F44276D8168
:1031D000462B50936B1C40936A1C5F934F933F9315
:1031E0002F939F938F9385E194E09F938F930E94F9
:1031F000F8A20FB6F894DEBF0FBECDBF26960FB66D
:10320000F894DEBF0FBECDBFDF91CF911F910F911C
:103210000895CF92DF92EF92FF920F931F93CF9377
:10322000DF93CDB7DEB72A970FB6F894DEBF0FBE97
:10323000CDBF8E010F5F1F4F86E0F80111928A9576
:10324000E9F741E062E08CE30E94741248E560E037
:103250008CE30E94741262E174E380E090E00E94CB
:10326000116A26E0A80163E08CE30E948B1243E020
:1032700062E08CE30E947412098110E0102F002795
:103280008A81082BE6E4FCE111830083EB80F12CBA
:10329000FE2CEE248C81E82AF382E282CD80D12CB0
:1032A000DC2CCC248E81C82AD582C482B801012EA0
:1032B000000C880B990B0E9413999B01AC01B7017C
:1032C0000F2C000C880B990B2F83388749875A875E
:1032D0000E9413992F81388549855A850E94FB9752
:1032E00020EE3EE245E652E40E940B9B20E030E0F7
:1032F00044E353E40E947C979F938F937F936F9353
:10330000DF92CF92FF92EF921F930F9383E294E0AC
:103310009F938F930E94F8A20FB6F894DEBF0FBE62
:10332000CDBF2A960FB6F894DEBF0FBECDBFDF919A
:10333000CF911F910F91FF90EF90DF90CF90089564
:10334000CF93DF93EC01888199810097A9F18E38A2
:10335000924121F01982188283E081C08DEF9AE0BA
:103360000E948A61892B91F18091E30A9091E40A8D
:10337000A091E50AB091E60A93FD2AC08091E30A84
:103380009091E40AA091E50AB091E60A93FD51C03C
:103390008091E30A9091E40AA091E50AB091E60ACF
:1033A00094FD4FC08091E30A9091E40AA091E50A50
:1033B000B091E60A95FD4CC060E870E08DEF9AE0B0
:1033C0000E9463618EE892E19983888381E047C01F
:1033D0008091922C82FFD2CF21E048E061E083E02F
:1033E0000E9416168091791D8F938091781D8F937E
:1033F0008091771D8F938091761D8F938091751D9D
:103400008F938091741D8F938091731D8F93809102
:10341000721D8F9384EF90E19F938F930E940CA372
:103420008DB79EB70A960FB6F8949EBF0FBE8DBF9C
:10343000A5CF8091922C85FFABCF81E00E94FB78D5
:10344000A7CF8091922C86FFADCF0E949118AACF72
:103450008091922C87FFB0CF0E940919ADCFDF91E8
:10346000CF910895CF93DF93C82F8CEE0E948F6A7F
:103470008C2F0E94996A65E375E080E090E00E94DD
:10348000116A8DEE0E948F6A0E94AA6AD82F0E944C
:10349000B46AC82F0E94916A8C2F90E09D2BDF9117
:1034A000CF9108951F93CF93DF93C82F8CEE0E9486
:1034B0008F6A8C2F0E94996A62E174E380E090E049
:1034C0000E94116A8CEE0E948F6A80E00E94996AC5
:1034D00065E375E080E090E00E94116A8DEE0E9445
:1034E0008F6A0E94AA6AD82F0E94AA6A182F0E9487
:1034F000B46AC82F0E94916A812F90E0A0E0B0E0EA
:10350000BA2FA92F982F8827AD2BBC01CD016C2B8A
:10351000DF91CF911F9108952F923F924F925F922A
:103520006F927F928F929F92AF92BF92CF92DF92D3
:10353000EF92FF920F931F93CF93DF93CDB7DEB738
:10354000CB54D1090FB6F894DEBF0FBECDBF80912A
:10355000000290910102892BE1F110920102109278
:1035600000028CEE0E948F6A8EE10E94996A0E948E
:10357000916A6BE17EE480E090E00E94116A82EA49
:103580000E94321A9093F20A8093F10A84EA0E9410
:10359000321A9093F00A8093EF0A86EA0E94321A58
:1035A0009093EE0A8093ED0A88EA0E94321A909373
:1035B000EC0A8093EB0A8AEA0E94321A9093EA0A94
:1035C0008093E90A8CEA0E94321A9093E80A809369
:1035D000E70A88E40E94521A6DAB7EAB8FAB98AFBE
:1035E00088E50E94521A4B015C018091E90A909192
:1035F000EA0A8C0120E030E040E050E0BA01229677
:103600008FAF229723961FAF239724962FAF24972F
:1036100025963FAF259726964FAF269727965FAF03
:10362000279728966FAF289729967FAF29979C01F7
:1036300040E050E060E070E080E090E008E00E9450
:10364000FB9D0E94B49D3901B42FA52FF62FE72FC3
:103650008C019401A50160E070E080E090E05301EE
:10366000CB2EDA2EEF2EFE2E0E94329E2CA33BA3F1
:1036700049835A831B012C01C201315041095F4F1C
:103680006F4F7F4F8F4F9F4F88248394912C21152C
:103690003F4F4F4F5140610571058105910509F07C
:1036A00010F4812C912C34010091E70A1091E80A62
:1036B0005801C12CD12CE12CF12C00E010E02CA100
:1036C0003BA149815A81B101C2010E94A09CF22E06
:1036D000032F142FB52FF62FE72FD82EE92EA0E0B9
:1036E0000E94599E84F42150310940485F4F6F4F2A
:1036F0007F4F8F4F9F4FF22E032F142FB52FF62F92
:10370000E72FD82EE92E2F2D302F412F5B2F6F2F33
:103710007E2F8D2D9E2D07E10E94149E2B8F3C8FB6
:103720004D8F5E8F6F8F78A389A39AA32053384F54
:103730004F4F5F4F6F4F7F4F8F4F9F4F2B8B3C8B68
:103740004D8B5E8B6F8B788F898F9A8F2056304F81
:103750004F4F5F4F6F4F7F4F8F4F9F4F243D3043F1
:1037600041055105610571058105910529F020F09C
:103770003401BFEF6B1A7B0A8090EF0A9090F00A39
:10378000940140E050E060E070E080E090E000E113
:103790000E94FB9D2B833C834D835E836F837887E0
:1037A0004C014091EB0A5091EC0AACA0BBA0C9803F
:1037B000DA80710182019A0140E050E060E070E03F
:1037C00080E090E00E94A09CF22E032F142FB52FD2
:1037D000F62FE72FD82EE92EA0E00E94599E5CF428
:1037E000AFE70E943B9EF22E032F142FB52FF62F2A
:1037F000E72FD82EE92E2F2D302F412F5B2F6F2F43
:103800007E2F8D2D9E2D07E00E94149E59016A0186
:103810007B018C012B813C814D815E816F8178859C
:10382000C4010E94329E2B833C834D835E836F8351
:1038300078878F87988B2E5F3F4F434051096E4F9B
:103840007F4F8F4F9F4F22303105494F5F4F64406C
:1038500071058105910521F018F0FFEF6F1A7F0ABD
:103860006091F10A7091F20A80E090E020E030E887
:1038700040E050E00E94F99C29873A874B875C879B
:103880006D877E874C014091ED0A5091EE0AACA005
:10389000BBA0C980DA80710182019A0140E050E04A
:1038A00060E070E080E090E00E94A09CF22E032F88
:1038B000142FB52FF62FE72FD82EE92EA0E00E9467
:1038C000599E84F421503F4F4F4F5F4F6F4F7F4FB2
:1038D0008F4F9F4FF22E032F142FB52FF62FE72F68
:1038E000D82EE92E2F2D302F412F5B2F6F2F7E2FBB
:1038F0008D2D9E2D08E00E94149E59016A017B01C6
:103900008C0129853A854B855C856D857E85C40152
:103910000E94329E29873A874B875C876D877E8716
:10392000898B9A8B2F5F3F4F414051096109710983
:1039300081099109213030484C4F5F476140710542
:103940008105910521F018F01FEF611A710A2B898A
:103950003C894D895E896F89788D898D9A8D2F3C40
:10396000374041055105610571058105910511F04B
:103970000CF09CC1ACA0BBA0C980DA8071018201AF
:103980009501A601B101C2010E94A09CA12CB12CFD
:10399000C12CE0E8DE2EE12CF12C00E010E00E94CA
:1039A000269D29AF3AAF4BAF5CAF6DAF7EAF8FAF07
:1039B00021969FAF2197AB8CBC8CCD8CDE8CEF8C8D
:1039C000F8A009A11AA19501A601B701C8010E949A
:1039D000A09C59016A017B01E82F192F02E00E9487
:1039E000FB9D0E2F0E94329E7901142F452EF62F3B
:1039F000E72F6C01922EAF2CB42E052F362EB72F49
:103A0000582E8D2CA0E00E94599E5CF4A1E00E94EB
:103A10003B9E922EA32EB42E052F362EB72F582E56
:103A2000892E292D3A2D4B2D502F632D7B2F852D3F
:103A3000982D01E00E94149E29A73AA74A012C96CE
:103A40006FAF2C972B967FAF2B978BA79CA72983C3
:103A50003A834BA39CA26DA37EA38FA398A7B42DFA
:103A60009701412F542D6F2F7E2FC601A0E00E9499
:103A7000599E4CF4A3E00E943B9E7901142FB52F70
:103A8000F62FE72F6C019701412F5B2F6F2F7E2FB1
:103A9000C60102E00E94149E2DA73EA74FA758AB77
:103AA00069AB7AAB8BAB9CAB2901B42FA52F2296C7
:103AB0006FAF2297F72F1C012B893C894D895E89B6
:103AC0006F89788D898D9A8D24323A4F4F4F5F4F91
:103AD0006F4F7F4F8F4F9F4F0CF08BC02B8D3C8DC6
:103AE0004D8D5E8D6F8D78A189A19AA12455324F9D
:103AF0004F4F5F4F6F4F7F4F8F4F9F4F59016A015D
:103B00007B018C010E94A09C19012A01B62FA72FCE
:103B1000FC0103E00E94FB9D51016201EB2EFA2E95
:103B20008F010E94479E59016A017B018C0129A5E2
:103B30003AA5A4012C966FAD2C972B967FAD2B97B1
:103B40008BA59CA50E94329E29833A834BA35CA33C
:103B50006DA37EA38FA398A79101A2016B2F7A2F4B
:103B6000CF0102E00E94FB9D51016201EB2EFA2E73
:103B70008F010E94479E02E00E94FB9D0E2F0E9433
:103B8000479E122FD32EE42EB52FF62FE72FF82EB7
:103B9000092FA0E00E94599E5CF4A1E00E943B9E88
:103BA000122FD32EE42EB52FF62FE72FF82E092F44
:103BB000212F3D2D4E2D5B2F6F2F7E2F8F2D902F80
:103BC00001E00E94149E59016A017B018C012DA520
:103BD0003EA54FA558A969A97AA98BA99CA90E94BD
:103BE000329E2901B42FA52F22966FAF2297F72F6F
:103BF0001C012B813C814D815E816F8178858F8591
:103C00009889A980BA80CBA0DCA0EDA0FEA00FA16E
:103C100018A50E94479E2B833C834D835E836F8350
:103C200078878F87988B29853A854B855C856D854C
:103C30007E8589899A895201CB2EDA2E2296EFACA5
:103C40002297FF2E81010E94479E29873A874B8742
:103C50005C876D877E87898B9A8B2B893C894D8900
:103C60005E896F89788D898D9A8DA9ACBAACCBAC01
:103C7000DCACEDACFEAC0FAD21961FAD21970E94E0
:103C8000479E2056304F4F4F5F4F6F4F7F4F8F4FA4
:103C90009F4F243D30434105510561057105810564
:103CA000910521F018F00FEF601A700A4DA95EA976
:103CB0006FA978AD9A01AB0160E070E0CB0122966C
:103CC0002FAF229723963FAF239724964FAF249789
:103CD00025965FAF259726966FAF269727967FAFDD
:103CE000279728968FAF289729969FAF2997A98461
:103CF000BA84CB84DC84ED84FE8409891A8960E06F
:103D000070E080E090E00E94A09C122FD32EE42E61
:103D1000B52FF62FE72FF82E092FA0E00E94599E0D
:103D200084F421503109404E5F4F6F4F7F4F8F4FCA
:103D30009F4F122FD32EE42EB52FF62FE72FF82EFC
:103D4000092F212F3D2D4E2D5B2F6F2F7E2F8F2D75
:103D5000902F05E10E94149EAB80BC80CD80DE8058
:103D6000EF80F8840F8518890E94479E122FD32E6A
:103D7000E42EB52FF62FE72FF82E092FA0E00E9492
:103D8000599E84F4215030484F4F5F4F6F4F7F4F03
:103D90008F4F9F4F122FD32EE42EB52FF62FE72FE4
:103DA000F82E092F212F3D2D4E2D5B2F6F2F7E2FAB
:103DB0008F2D902F0FE00E94149E59016A017B0104
:103DC0008C01322E5B2CB42FAD2DF62F4F2C4C01D5
:103DD000285E33404109510961097109810991093E
:103DE000283D304D41405105610571058105910522
:103DF00009F010F4672869F09501A601B701C80120
:103E00000E94B49D322E532EB42FA52FF62F472E8D
:103E10004C01232D352D4B2F5A2F6F2F742DC4019C
:103E20000E940B9920E030E048EC52E40E945F9839
:103E3000C55BDF4F0FB6F894DEBF0FBECDBFDF917D
:103E4000CF911F910F91FF90EF90DF90CF90BF9097
:103E5000AF909F908F907F906F905F904F903F902A
:103E60002F9008954F925F926F927F928F929F92C0
:103E7000AF92BF92CF92DF92EF92FF922B013C0163
:103E800069017A0123EC35EF4CE851E4C701B60132
:103E90000E940B9B4B015C0128EB3EE143E753E49E
:103EA000C701B6010E947C979B01AC01C501B4011A
:103EB0000E945F980E94D9984B015C0120E030E09D
:103EC00048EC52E4C301B2010E945F9821E835E951
:103ED00043EC50E40E940B9BA50194010E940B9BB4
:103EE0004B015C0123E333E948E853E4C701B60121
:103EF0000E947C979B01AC01C501B4010E945F98B0
:103F000023E333EB48E553E40E940B9BFF90EF90D3
:103F1000DF90CF90BF90AF909F908F907F906F90E9
:103F20005F904F9008954F925F926F927F928F9221
:103F30009F92AF92BF92CF92DF92EF92FF92690170
:103F40007A010E947F9A20E030E040E050E40E9435
:103F50007B9722E93CE54EED5EE30E945F984B01C2
:103F60005C0123EC35EF4CE851E4C701B6010E9437
:103F70000B9B2B013C0128EB3EE143E753E4C701D7
:103F8000B6010E947C979B01AC01C301B2010E9463
:103F90005F989B01AC01C501B4010E947C976B0145
:103FA0007C0128EB3EE143E753E40E940B9B4B016D
:103FB0005C01A701960163EC75EF8CE891E40E9427
:103FC0007B979B01AC01C501B4010E945F98FF90F3
:103FD000EF90DF90CF90BF90AF909F908F907F90A9
:103FE0006F905F904F9008954F925F926F927F9283
:103FF0008F929F92AF92BF92CF92DF92EF92FF92F9
:104000002B013C0169017A0123EC35EF4CE851E4C6
:10401000C701B6010E940B9B4B015C0128EB3EE1FE
:1040200043E753E4C701B6010E947C979B01AC01B2
:10403000C501B4010E945F980E94D9984B015C01B0
:1040400020E030E048EC52E4C301B2010E945F98E6
:10405000A50194010E940B9B20E030E040E251E476
:104060000E947B9724EE38E34EE05FE30E940B9BB7
:104070009B01AC01C701B6010E947C97FF90EF90B5
:10408000DF90CF90BF90AF909F908F907F906F9078
:104090005F904F90089580E80E948F6A81110DC053
:1040A0008EEF0E94996A811108C06BE17EE480E086
:1040B00090E00E94116A0C94916A0E94916A80912A
:1040C000A4309091A530A091A630B091A730019670
:1040D000A11DB11D8093A4309093A530A093A6306C
:1040E000B093A7300895FC01DC01AC014E5F5F4F37
:1040F00090E031E38D91982788E0292F220F97FFD8
:1041000003C0922F932701C0922F8150B1F7A417BB
:10411000B50781F721E030E08281981711F020E0A7
:1041200030E0C9010895DF92EF92FF920F931F9341
:10413000CF93DF930E944B2080E80E948F6A811109
:104140006DC08AEF0E94996A811168C08FE00E9459
:10415000996A811163C065E375E080E090E00E9498
:10416000116A81E80E948F6A811158C00E94AA6A70
:10417000D82F0E94AA6A0E94AA6A182F0E94AA6ACF
:104180000E94AA6A082F0E94AA6A0E94B46AF82EA6
:1041900080E80E948F6A811141C08CEF0E94996A69
:1041A00081113CC089EC0E94996A811137C065E396
:1041B00075E080E090E00E94116A81E80E948F6AB9
:1041C0000E94AA6AE82E0E94AA6AD82E0E94AA6AB1
:1041D0000E94AA6AC82F0E94B46A1F92DF921F929F
:1041E000EF921F92FF921F920F931F921F931F92A5
:1041F000DF931F928F931F92CF9388E394E09F9356
:104200008F930E94F8A20E94916A8DB79EB7429642
:104210000FB6F8949EBF0FBE8DBF17C00E94916A63
:104220008091A4309091A530A091A630B091A73094
:104230000196A11DB11D8093A4309093A530A09349
:10424000A630B093A7300E944B2020E030E040E041
:1042500050E060E070E080E090E0DF91CF911F914E
:104260000F91FF90EF90DF900895EF92FF920F93E0
:104270001F93CF93DF9300D01F92CDB7DEB78C0191
:1042800080E80E948F6A811154C00115110551F018
:1042900085EE0E94996A81114CC061E077E980E067
:1042A00090E009C083EE0E94996A811142C069E9D9
:1042B0007AEB81E090E00E94116A81E80E948F6AA7
:1042C000811137C00E94AA6AE82E89830E94AA6AD7
:1042D000F82E8A830E94B46A8B830E94916ACE0171
:1042E00001960E947320892B21F16F2D70E07E29A9
:1042F0006C7F80E090E0012B69F00E94119920E032
:1043000030E04AEF5AE30E940B9B20E030E040ECA3
:1043100050E40CC00E94119922E538EB4FE25BE3B8
:104320000E940B9B26E636E64BE352E40E947B9705
:104330001BC00E94916A8091A4309091A530A091F9
:10434000A630B091A7300196A11DB11D8093A43075
:104350009093A530A093A630B093A7300E944B2035
:1043600060EF7FEF89E794E40F900F900F90DF915B
:10437000CF911F910F91FF90EF9008950F931F938E
:10438000CF93DF93729A8091620283FF08C08EE41C
:104390000E94346A811165C0C0E5D0E009C0C0E563
:1043A000D0E087EE93E00E94590A2197D1F7EFCF32
:1043B00087EE93E00E94590A2197D1F78FE40E947B
:1043C000346A0E94AA6AD82FDF730E94AA6A082F53
:1043D0000E94AA6AC82F0E94B46A182F0E94916A8C
:1043E0008091620283FF72986D2F70E0762F6627AE
:1043F000600F711D80E090E00E94119920E134E08F
:1044000048EC5BE30E940B9B60938628709387289F
:1044100080938828909389286C2F70E0762F6627E8
:10442000610F711D769567957695679580E090E0B0
:104430000E94119924EA3CEF44E25CE30E940B9B4A
:1044400020E030E040E252E40E947B9760937335B5
:1044500070937435809375359093763580E090E055
:1044600002C081E090E0DF91CF911F910F910895FC
:104470007298729A8EE40E94346A80EA0E94996A65
:1044800080E00E94996A80E00E94996A8FE40E940D
:10449000346A0E94AA6A8EE40E94346A80E80E940C
:1044A000996A80E00E94996A80E00E94996A0E945D
:1044B000916A80E090E0089583E290E19F938F936A
:1044C0000E940CA380917D020F900F90882361F0D1
:1044D0001F928F9380E290E19F938F930E940CA391
:1044E0000F900F900F900F9008958BEF9FE09F9388
:1044F0008F930E940CA383ED9FE09F938F930E9464
:104500000CA38CEA9FE09F938F930E940CA381E7FA
:104510009FE09F938F930E940CA385E39FE09F935E
:104520008F930E940CA383E09FE09F938F930E9440
:104530000CA387EC9EE09F938F930E940CA381EACB
:104540009EE09F938F930E940CA38BE69EE09F9327
:104550008F930E940CA38091922C9091932C827047
:1045600098702DB73EB72E5E3F4F0FB6F8943EBF02
:104570000FBE2DBF892B41F08BE39EE09F938F935D
:104580000E940CA30F900F908FE09EE09F938F935B
:104590000E940CA383ED9DE09F938F930E940CA338
:1045A0008AEA9DE09F938F930E940CA38EE79DE083
:1045B0009F938F930E940CA38FE49DE09F938F9312
:1045C0000E940CA38DE19DE09F938F930E940CA30A
:1045D0008CEE9CE09F938F930E940CA382EB9CE057
:1045E0009F938F930E940CA38CE79CE09F938F93E3
:1045F0000E940CA38CE49CE09F938F930E940CA3D9
:1046000080E29CE09F938F930E940CA381EF9BE03C
:104610009F938F930E940CA388EB9BE09F938F93B3
:104620000E940CA38FE79BE09F938F930E940CA3A3
:1046300088E49BE09F938F930E940CA38AE19BE008
:104640009F938F930E940CA38DB79EB780960FB651
:10465000F8949EBF0FBE8DBF86EE9AE09F938F9316
:104660000E940CA385EB9AE09F938F930E940CA36A
:1046700086E89AE09F938F930E940CA387E59AE0C7
:104680009F938F930E940CA380E39AE09F938F9354
:104690000E940CA38AEF99E09F938F930E940CA332
:1046A00084EC99E09F938F930E940CA38EE899E08D
:1046B0009F938F930E940CA385E699E09F938F931D
:1046C0000E940CA38DE299E09F938F930E940CA30C
:1046D00082E099E09F938F930E940CA32DB73EB781
:1046E0002A5E3F4F0FB6F8943EBF0FBE2DBF089510
:1046F00087E694E00C9434A34F925F926F927F927E
:104700008F929F92AF92BF92CF92DF92EF92FF92E1
:10471000CF93DF93CDB7DEB728970FB6F894DEBFFF
:104720000FBECDBF8091983090919930A0919A3072
:10473000B0919B3089839A83AB83BC83409098303F
:104740005090993060909A3070909B308091983062
:1047500090919930A0919A30B0919B308D839E8337
:10476000AF83B887609198307091993080919A307A
:1047700090919B302CE3822E912CA12CB12CA50181
:1047800094010E941E9C7F936F9330E1C32E3EE004
:10479000D32EE12CF12C6D817E818F819885A7012C
:1047A00096010E941E9CA50194010E941E9C3F93AD
:1047B0002F9340E8842E41E5942EAA24A394B12C93
:1047C000C301B201A50194010E941E9CA70196019C
:1047D0000E941E9C3F932F9369817A818B819C81DB
:1047E000A50194010E941E9C3F932F938CED98E0AD
:1047F0009F938F930E940CA30FB6F894DEBF0FBE59
:10480000CDBF28960FB6F894DEBF0FBECDBFDF91A7
:10481000CF91FF90EF90DF90CF90BF90AF909F909F
:104820008F907F906F905F904F900895E4E3FEE348
:10483000808191818234924479F0E453FE43FF9366
:10484000EF938EEB98E09F938F930E940CA30F90B1
:104850000F900F900F9008953A96E53F81E4F80786
:1048600038F30895CF93DF93EC018C9A0E94D50C16
:104870009F938F937F936F9382EB98E09F938F9397
:104880000E940CA30F900F900F900F900F900F901D
:10489000209719F00E94E60D08C080EB98E09F93E6
:1048A0008F930E940CA30F900F9081E00E94870CC1
:1048B00020918202309183024091840250918502BE
:1048C0000E940B9B9F938F937F936F9384EA98E052
:1048D0009F938F930E940CA30F900F900F900F90B7
:1048E0000F900F90209719F00E94E60D08C082EA01
:1048F00098E09F938F930E940CA30F900F9082E0FB
:104900000E94870C20917E0230917F0240918002AC
:10491000509181020E940B9B9F938F937F936F9383
:1049200086E998E09F938F930E940CA30F900F90BD
:104930000F900F900F900F90209719F00E94E60DA6
:1049400008C084E998E09F938F930E940CA30F9076
:104950000F9083E00E94870C9F938F937F936F93B8
:1049600085E898E09F938F930E940CA38C980F90FA
:104970000F900F900F900F900F90209719F00E94BA
:10498000E60D08C083E898E09F938F930E940CA3E4
:104990000F900F908091922C9091932C92FF83C056
:1049A00021E042E161E080ED0E94FB6B9F938F93D9
:1049B0007F936F9386E798E09F938F930E940CA359
:1049C0000F900F900F900F900F900F90209719F06D
:1049D0000E94E60D08C084E798E09F938F930E94A1
:1049E0000CA30F900F9021E042E162E080ED0E9465
:1049F000FB6B9F938F937F936F9387E698E09F93D2
:104A00008F930E940CA30F900F900F900F900F9018
:104A10000F90209719F00E94E60D08C085E698E0F7
:104A20009F938F930E940CA30F900F9021E042E17F
:104A300063E080ED0E94FB6B9F938F937F936F9356
:104A400088E598E09F938F930E940CA30F900F909E
:104A50000F900F900F900F90CD2B19F00E94E60D44
:104A600008C086E598E09F938F930E940CA30F9057
:104A70000F9021E042E164E080ED0E94FB6B9F9388
:104A80008F937F936F9389E498E09F938F930E9415
:104A90000CA30F900F900F900F900F900F90DF913D
:104AA000CF910C94E60DCD2BD1F3DF91CF910895EA
:104AB0000F931F93CF93DF93882389F049E050E051
:104AC0006FEF70E08BE595E30E9446A249E050E06D
:104AD0006EE070E08BE595E30E9410A613C0CBE575
:104AE000D5E304E418E089911F928F931F930F93ED
:104AF0000E940CA30F900F900F900F9085E3C33688
:104B0000D80789F7DF91CF911F910F910C94E60D93
:104B1000882311F0299A089529980895882311F07F
:104B20002A9A08952A980895882311F02B9A0895B7
:104B30002B980895CF92DF92EF92FF92CF93DF935D
:104B40006B017C0160FF11C084EA94E09F938F9316
:104B500088E390E19F938F930E940CA30F900F9096
:104B60000F900F9081E090E002C080E090E0C1FEE5
:104B700009C0EC0121964EE35AE069EA74E00E9414
:104B80004C12CE01C2FE09C0EC0121964EE35AE060
:104B900061EB74E00E944C12CE01C3FE09C0EC012F
:104BA00021964EE35AE069EB74E00E944C12CE016C
:104BB000C4FE09C0EC0121964EE35AE065E476E0BC
:104BC0000E944C12CE01C5FE09C0EC0121964EE3B5
:104BD0005AE06DEB74E00E944C12CE01C6FE09C093
:104BE000EC0121964EE35AE061EC74E00E944C1215
:104BF000CE01C7FE09C0EC0121964EE35AE067ECF6
:104C000074E00E944C12CE01D0FE09C0EC01219646
:104C10004EE35AE06FEC74E00E944C12CE01D1FEDC
:104C200009C0EC0121964EE35AE067ED74E00E9462
:104C30004C12CE01D2FE09C0EC0121964EE35AE09F
:104C40006BED74E00E944C12CE012091922C3091B9
:104C5000932C24703071232B59F0D3FE09C0EC0142
:104C600021964EE35AE061EE74E00E944C12CE01B0
:104C70002091922C26FF0BC0D4FE09C0EC01219696
:104C80004EE35AE066EE74E00E944C12CE01209191
:104C9000922C27FF0BC0D5FE09C0EC0121964EE3F4
:104CA0005AE06CEE74E00E944C12CE01D6FE09C0B0
:104CB000EC0121964EE35AE064EF74E00E944C123E
:104CC000CE01D7FE09C0EC0121964EE35AE06FEF0A
:104CD00074E00E944C12CE01E0FE0CC04EE35AE09C
:104CE00060E175E0DF91CF91FF90EF90DF90CF9082
:104CF0000C944C12CD28CE28CF2841F48FE398E0B5
:104D00009F938F930E940CA30F900F90DF91CF91F0
:104D1000FF90EF90DF90CF900895CF92DF92EF92C7
:104D2000FF92CF93DF93EC01C12CD12C7601209719
:104D300009F4A3C06AE378E0CE010E9425A2892B82
:104D400011F46894C0F862E378E0CE010E9425A2D5
:104D5000892B11F46894C1F86AE278E0CE010E94D0
:104D600025A2892B11F46894C2F866E278E0CE019E
:104D70000E9425A2892B11F46894C3F863E278E0BD
:104D8000CE010E9425A2892B11F46894C4F86FE12A
:104D900078E0CE010E9425A2892B11F46894C5F811
:104DA00069E178E0CE010E9425A2892B11F4689474
:104DB000C6F861E178E0CE010E9425A2892B11F4AA
:104DC0006894C7F869E078E0CE010E9425A2892B9B
:104DD00011F46894D0F865E078E0CE010E9425A235
:104DE000892B11F46894D1F86FEF77E0CE010E941F
:104DF00025A2892B11F46894D2F86AEF77E0CE01EE
:104E00000E9425A2892B11F46894D3F864EF77E00F
:104E1000CE010E9425A2892B11F46894D4F86CEE7F
:104E200077E0CE010E9425A2892B11F46894D5F871
:104E300061EE77E0CE010E9425A2892B11F46894DF
:104E4000D6F860ED77E0CE010E9425A2892B11F4FF
:104E50006894D7F86BEC77E0CE010E9425A2892BED
:104E600011F46894E0F860917B0270917C0280E01C
:104E700090E00E9439A2EC015ACFC701B601DF9140
:104E8000CF91FF90EF90DF90CF900895AF92BF92B7
:104E9000CF92DF92EF92FF920F931F93CF93DF9306
:104EA000D22FC32F8A01F62EC72ED82EE92E2170BD
:104EB00030E040E050E060E070E080E090E0A0E0B2
:104EC0000E94599E89F085E195E09F938F9388E336
:104ED00090E19F938F930E940CA30F900F900F90DF
:104EE0000F90E1E0F0E002C0E0E0F0E08091922C71
:104EF00080FF19C02D2F247030E040E050E060E0CA
:104F000070E080E090E0A0E00E94599E61F05F01B7
:104F10008FEFA81AB80A4EE35AE069E175E0CF01B5
:104F20000E944C12F5012D2F227030E040E050E03D
:104F300060E070E080E090E0A0E00E94599E61F0A7
:104F40005F018FEFA81AB80A4EE35AE06DE175E0F1
:104F5000CF010E944C12F5012D2F287030E040E067
:104F600050E060E070E080E090E0A0E00E94599E98
:104F700061F05F018FEFA81AB80A4EE35AE065E3CB
:104F800075E0CF010E944C12F5012D2F207130E009
:104F900040E050E060E070E080E090E0A0E00E943F
:104FA000599E61F05F018FEFA81AB80A4EE35AE0EC
:104FB00060E275E0CF010E944C12F5012D2F2072A6
:104FC00030E040E050E060E070E080E090E0A0E0A1
:104FD0000E94599E61F05F018FEFA81AB80A4EE354
:104FE0005AE063E275E0CF010E944C12F5012D2FCB
:104FF000207430E040E050E060E070E080E090E05D
:10500000A0E00E94599E61F05F018FEFA81AB80AD4
:105010004EE35AE069E275E0CF010E944C12F501BF
:105020002D2F207830E040E050E060E070E080E03C
:1050300090E0A0E00E94599E61F05F018FEFA81AF6
:10504000B80A4EE35AE06FE275E0CF010E944C12BD
:10505000F50120E03C2F317040E050E060E070E06E
:1050600080E090E0A0E00E94599E61F05F018FEF28
:10507000A81AB80A4EE35AE062E375E0CF010E9435
:105080004C12F50120E03C2F327040E050E060E02F
:1050900070E080E090E0A0E00E94599E61F05F0126
:1050A0008FEFA81AB80A4EE35AE067E375E0CF0124
:1050B0000E944C12F50120E03C2F347040E050E09B
:1050C00060E070E080E090E0A0E00E94599E61F016
:1050D0005F018FEFA81AB80A4EE35AE06EE375E05D
:1050E000CF010E944C12F50120E03C2F387040E0C7
:1050F00050E060E070E080E090E0A0E00E94599E07
:1051000061F05F018FEFA81AB80A4EE35AE061E43C
:1051100075E0CF010E944C12F50120E03C2F307168
:1051200040E050E060E070E080E090E0A0E00E94AD
:10513000599E61F05F018FEFA81AB80A4EE35AE05A
:1051400066E475E0CF010E944C12F50120E03C2F8F
:10515000307240E050E060E070E080E090E0A0E07D
:105160000E94599E61F05F018FEFA81AB80A4EE3C2
:105170005AE06DE475E0CF010E944C12F50120E089
:1051800030E040E050E06F2D647070E080E090E02F
:10519000A0E00E94599E61F05F018FEFA81AB80A43
:1051A0004EE35AE064E575E0CF010E944C12F50130
:1051B0008091922C81FF19C020E03C2F307440E098
:1051C00050E060E070E080E090E0A0E00E94599E36
:1051D00061F05F018FEFA81AB80A4EE35AE068E564
:1051E00075E0CF010E944C12F5018091922C9091B4
:1051F000932C93FF19C020E030E040E0512F507114
:1052000060E070E080E090E0A0E00E94599E61F0D4
:105210005F018FEFA81AB80A4EE35AE06BE575E01C
:10522000CF010E944C12F5018091922C9091932C09
:1052300093FF19C020E030E040E0512F507260E051
:1052400070E080E090E0A0E00E94599E61F05F0174
:105250008FEFA81AB80A4EE35AE06EE575E0CF0169
:105260000E944C12F5018091922C9091932C93FF07
:1052700019C020E030E040E0512F507460E070E051
:1052800080E090E0A0E00E94599E61F05F018FEF06
:10529000A81AB80A4EE35AE064E675E0CF010E940E
:1052A0004C12F50120E03C2F307840E050E060E007
:1052B00070E080E090E0A0E00E94599E61F05F0104
:1052C0008FEFA81AB80A4EE35AE06FE675E0CF01F7
:1052D0000E944C12F50120E030E0402F417050E078
:1052E00060E070E080E090E0A0E00E94599E61F0F4
:1052F0005F018FEFA81AB80A4EE35AE064E775E041
:10530000CF010E944C12F50120E030E0402F4270A6
:1053100050E060E070E080E090E0A0E00E94599EE4
:1053200061F05F018FEFA81AB80A4EE35AE067E711
:1053300075E0CF010E944C12F50120E030E040E022
:1053400050E06F2D687070E080E090E0A0E00E9477
:10535000599E61F05F018FEFA81AB80A4EE35AE038
:105360006AE775E0CF010E944C12F50120E030E0C1
:1053700040E050E06F2D607170E080E090E0A0E0D0
:105380000E94599E61F05F018FEFA81AB80A4EE3A0
:105390005AE06EE775E0CF010E944C12F501809152
:1053A000922C9091932C92FF19C020E030E0402F76
:1053B000487050E060E070E080E090E0A0E00E9483
:1053C000599E61F05F018FEFA81AB80A4EE35AE0C8
:1053D00062E875E0CF010E944C12F5018091922C99
:1053E0009091932C92FF19C020E030E0402F407143
:1053F00050E060E070E080E090E0A0E00E94599E04
:1054000061F05F018FEFA81AB80A4EE35AE066E830
:1054100075E0CF010E944C12F5018091922C909181
:10542000932C92FF19C020E030E0402F407250E0F2
:1054300060E070E080E090E0A0E00E94599E61F0A2
:105440005F018FEFA81AB80A4EE35AE06AE875E0E8
:10545000CF010E944C12F5018091922C9091932CD7
:1054600092FF19C020E030E0402F407450E060E02F
:1054700070E080E090E0A0E00E94599E61F05F0142
:105480008FEFA81AB80A4EE35AE06EE875E0CF0134
:105490000E944C12F5018091922C82FF19C020E0ED
:1054A00030E0402F407850E060E070E080E090E035
:1054B000A0E00E94599E61F05F018FEFA81AB80A20
:1054C0004EE35AE068ED76E0CF010E944C12F50100
:1054D0008091922C82FF19C020E030E040E0512FF3
:1054E000517060E070E080E090E0A0E00E94599E82
:1054F00061F05F018FEFA81AB80A4EE35AE062E943
:1055000075E0CF010E944C12F5018091922C909190
:10551000932C93FF19C020E030E040E0512F5270EF
:1055200060E070E080E090E0A0E00E94599E61F0B1
:105530005F018FEFA81AB80A4EE35AE065E975E0FB
:10554000CF010E944C12F5018091922C9091932CE6
:1055500093FF19C020E030E040E0512F547060E02C
:1055600070E080E090E0A0E00E94599E61F05F0151
:105570008FEFA81AB80A4EE35AE06DE975E0CF0143
:105580000E944C12F5018091922C9091932C94FFE3
:1055900019C020E030E040E0512F587060E070E02A
:1055A00080E090E0A0E00E94599E61F05F018FEFE3
:1055B000A81AB80A4EE35AE066EA75E0CF010E94E5
:1055C0004C12F5018091922C85FF19C020E030E04B
:1055D00040E050E06F2D607270E080E090E0A0E06D
:1055E0000E94599E61F05F018FEFA81AB80A4EE33E
:1055F0005AE06FEA75E0CF010E944C12F5018091EC
:10560000922C85FF19C020E030E040E050E06F2D83
:10561000607470E080E090E0A0E00E94599E61F02C
:105620005F018FEFA81AB80A4EE35AE068EB75E005
:10563000CF010E944C12F5018091922C85FF1EC073
:1056400020E030E040E050E06F2D607870E080E0D6
:1056500090E0A0E00E94599E89F04EE35AE062EC8F
:1056600075E0CF01DF91CF911F910F91FF90EF90E7
:10567000DF90CF90BF90AF900C944C122D2F3C2F09
:10568000A8016F2D7C2D8D2D9E2DA0E00E94599E8E
:1056900041F486EC97E09F938F930E940CA30F90A8
:1056A0000F90DF91CF911F910F91FF90EF90DF90BE
:1056B000CF90BF90AF900895AF92BF92DF92EF92DC
:1056C000FF920F931F93CF93DF93EC015B01FB01DC
:1056D000108261EC77E00E9425A2892B89F58091E8
:1056E000922C1DE440E8F42E82FF03C034E8E32E40
:1056F00002C024E0E22E00E0D12C81FF02C090EC39
:10570000F92E26E04AE250E06BE270E089E290E098
:105710000E943B6781E090E00E947E0D81111DE5B3
:105720008091922C9091932C93FF02C0177F06E0FA
:1057300094FD086085FF09C0177F80EED82E05C054
:1057400010E0F12CE12C00E0D12C6FEB77E0CE01E2
:105750000E9425A2892B61F481E0F501808360918C
:105760007B0270917C0280E090E00E9439A2EC0103
:105770006DEB77E0CE010E9425A2892B61F48FEFBB
:10578000F501808360917B0270917C0280E090E063
:105790000E9439A2EC01209709F456C169EB77E029
:1057A000CE010E9425A2892B09F4116065EB77E0F8
:1057B000CE010E9425A2892B09F4146062EB77E0E8
:1057C000CE010E9425A2892B09F4126060EB77E0DC
:1057D000CE010E9425A2892B09F418606DEA77E0BA
:1057E000CE010E9425A2892B09F4106167EA77E0B7
:1057F000CE010E9425A2892B09F4106261EA77E0AC
:10580000CE010E9425A2892B09F410646EE977E08D
:10581000CE010E9425A2892B09F4106869E977E07E
:10582000CE010E9425A2892B19F4FF2DF160FF2ED5
:1058300062E977E0CE010E9425A2892B19F48F2D11
:105840008260F82E6FE877E0CE010E9425A2892BB6
:1058500019F4EF2DE460FE2E6AE877E0CE010E9495
:1058600025A2892B19F4FF2DF860FF2E63E877E05D
:10587000CE010E9425A2892B19F48F2D8061F82E6C
:105880006CE777E0CE010E9425A2892B19F4EF2D59
:10589000E062FE2E68E777E0CE010E9425A2892B08
:1058A00019F4FD2DF460DF2E65E777E0CE010E944C
:1058B00025A2892B19F48F2D8064F82E60E777E0FC
:1058C000CE010E9425A2892B19F4EF2DE068FE2E4F
:1058D0006DE677E0CE010E9425A2892B19F4FE2DFA
:1058E000F160EF2E6AE677E0CE010E9425A2892BB7
:1058F00019F48E2D8260E82E67E677E0CE010E94D3
:1059000025A2892B19F4EE2DE460EE2E63E677E0F4
:10591000CE010E9425A2892B19F4FE2DF860EF2EEE
:105920006FE577E0CE010E9425A2892B19F48E2D18
:105930008061E82E6BE577E0CE010E9425A2892BDD
:1059400019F4EE2DE062EE2E67E577E0CE010E94BD
:1059500025A2892B19F4FE2DF064EF2E65E577E082
:10596000CE010E9425A2892B19F48E2D8068E82E85
:1059700062E577E0CE010E9425A2892B09F401603F
:105980006AE477E0CE010E9425A2892B09F4026027
:1059900061E477E0CE010E9425A2892B09F404601E
:1059A00068E377E0CE010E9425A2892B09F4086004
:1059B00065E377E0CE010E9425A2892B09F40061FE
:1059C0006FE277E0CE010E9425A2892B09F40062E4
:1059D00064E277E0CE010E9425A2892B09F40064DD
:1059E00060E277E0CE010E9425A2892B19F4ED2D0B
:1059F000E860DE2E6CE177E0CE010E9425A2892BC3
:105A000019F4FD2DF061DF2E63E177E0CE010E94F5
:105A100025A2892B19F48D2D8062D82E69E077E0BC
:105A2000CE010E9425A2892B19F4ED2DE064DE2E13
:105A300060E077E0CE010E9425A2892B09F0A2CE7A
:105A4000FD2DF068DF2E9ECE212F3F2D4E2D502FA5
:105A50006D2D70E080E090E0DF91CF911F910F916C
:105A6000FF90EF90DF90BF90AF9008955F926F929C
:105A70007F928F929F92AF92BF92CF92DF92EF92DE
:105A8000FF920F931F93CF93DF93782EC5E7DCE14E
:105A900000E010E08AEFE82E86E0F82E872D817076
:105AA000582E872D8270682E95EEC92E96E0D92E3D
:105AB0002DEEA22E26E0B22E3BEE832E36E0932E64
:105AC000772051F01F930F93FF92EF920E940CA347
:105AD0000F900F900F900F905520A1F089858F9314
:105AE00088858F93BF92AF920E940CA30F900F9066
:105AF0000F900F906620C1F09F928F920E940CA38E
:105B00000F900F90662081F0DF92CF920E940CA33D
:105B1000288139814A815B816C817D818E819F8161
:105B20000E9446270F900F900E94E60D0F5F1F4FB7
:105B30002A960430110521F6DF91CF911F910F9124
:105B4000FF90EF90DF90CF90BF90AF909F908F909D
:105B50007F906F905F90089580EE96E09F938F9373
:105B60000E940CA38091822890918328A091842880
:105B7000B09185280F900F90813027EA92072EE18F
:105B8000A207B10519F482ED96E01DC0823026EA25
:105B900092072EE1A207B10519F485EC96E013C037
:105BA000823027EA92072EE1A207B10519F487EBAC
:105BB00096E009C0823028EA92072EE1A207B105DB
:105BC00049F489EA96E09F938F930E940CA30F906B
:105BD0000F900895BF93AF939F938F9383EA96E0BE
:105BE0009F938F930E940CA30F900F900F900F9094
:105BF0000F900F90089583E996E09F938F930E94F2
:105C00000CA30E9478230E94AC2D0E94E60D8CE527
:105C10009CE19F938F938BE896E09F938F930E94D4
:105C20000CA360915C0270915D0280915E02909184
:105C30005F0228EE33E040E050E00E941E9C5F933C
:105C40004F933F932F938BE796E09F938F930E9400
:105C50000CA382E796E09F938F930E940CA30E946F
:105C6000D6128091922C2DB73EB7225F3F4F0FB6D0
:105C7000F8943EBF0FBE2DBF80FF05C041E061E03C
:105C800081E00E94AC148EE696E09F938F930E9471
:105C90000CA380E00E9458250E947C238091610221
:105CA0001F928F9385E696E09F938F930E940CA39B
:105CB0008091DF0A1F928F938CE596E09F938F93DC
:105CC0000E940CA380918D028F9380918C028F9300
:105CD00080918B028F9380918A028F938EE496E05D
:105CE0009F938F930E940CA31F9280E48F9386E36F
:105CF00096E09F938F930E940CA3809178351F921A
:105D00008F93809177351F928F9383E296E09F93D4
:105D10008F930E940CA3809160021F928F938AE15F
:105D200096E09F938F930E940CA3809162029091C2
:105D30006302A0916402B09165022DB73EB7225E66
:105D40003F4F0FB6F8943EBF0FBE2DBF96FD03C068
:105D50008EEC95E002C08BEC95E09F938F9380E1F1
:105D600096E09F938F930E940CA383E00E94362DB0
:105D70000F900F900F900F901D9903C08EEC95E03F
:105D800002C08BEC95E09F938F9384E096E09F9305
:105D90008F930E940CA38AEF95E09F938F930E94AC
:105DA0000CA3809162020F900F900F900F900F90B4
:105DB0000F9081FF09C084EF95E09F938F930E941D
:105DC0000CA30F900F9013C080FD03C08EEC95E0E4
:105DD00002C08BEC95E09F938F9380EF95E09F93AB
:105DE0008F930E940CA30F900F900F900F908091B3
:105DF000620290916302A0916402B091650297FDE6
:105E000003C08EEC95E002C08BEC95E09F938F93DE
:105E100087EE95E09F938F930E940CA380EE95E010
:105E20009F938F930E940CA36091E30A7091E40A00
:105E30008091E50A9091E60A0E949A250E94E60D5B
:105E40000F900F900F900F900F900F90779B03C0C3
:105E50008EEC95E002C08BEC95E09F938F9387EDDD
:105E600095E09F938F930E940CA30E945F0A0E946B
:105E70003A0D9F938F937F936F9389EC95E09F9357
:105E80008F930E940CA30E94E90C9F938F937F93A2
:105E90006F938BEB95E09F938F930E940CA381E00F
:105EA00090E00E9432248091413590914235A0913A
:105EB0004335B0914435BF93AF939F938F938DEA51
:105EC00095E09F938F930E940CA3809156358F93FA
:105ED000809155358F93809154358F9380915335B0
:105EE0008F9389E995E09F938F930E940CA38091F3
:105EF000453590914635A0914735B0914835BF93CF
:105F0000AF939F938F938BE895E09F938F930E941D
:105F10000CA38DB79EB782960FB6F8949EBF0FBEA6
:105F20008DBF80915A358F93809159358F93809191
:105F300058358F93809157358F9387E795E09F93DE
:105F40008F930E940CA361E070E080E090E00E94DB
:105F5000EF0D61E070E081E090E00E94EF0D0F90A6
:105F60000F900F900F900F900F90299903C08EEC17
:105F700095E002C08BEC95E09F938F938FE695E0C0
:105F80009F938F930E940CA30F900F900F900F90F0
:105F90002A9903C08EEC95E002C08BEC95E09F93AC
:105FA0008F9387E695E09F938F930E940CA30F90A9
:105FB0000F900F900F900895F89491E2E0E0F0E0D8
:105FC000909357008491E2E0F0E090935700249181
:105FD000E4E0F0E090935700E49190E0A0E0B0E0BE
:105FE000BC0155274427822F90E0A0E0B0E0BA2FF3
:105FF000A92F982F8827840F951FA61FB71F8E0FD4
:10600000911DA11DB11D8093822890938328A09398
:106010008428B093852878940895CF93DF93CDB7E3
:10602000DEB761970FB6F894DEBF0FBECDBF48E272
:1060300050E062E270E085E79CE10E94F2A52091C9
:10604000751C3091761C4091771C5091781C6091A2
:10605000791C70917A1C80917B1C90917C1CAFEF15
:106060000E94599E09F05DC08DE48093751C80E804
:106070008093761C84E08093771C1092781C109299
:10608000791C10927A1C10927B1C10927C1C8CE361
:1060900090E090937E1C80937D1C10927F1C109248
:1060A000801C1092811C1092821C1092831C1092F2
:1060B000841C1092851C1092861C1092881C1092D1
:1060C000871C1092891C10928A1C10928B1C1092B3
:1060D0008C1C10928D1C10928E1C10928F1C109292
:1060E000901C1092921C1092911C1092931C109272
:1060F000941C1092951C1092961C1092971C109252
:10610000981C1092991C10929A1C10929C1C109230
:106110009B1C48E250E062E270E085E79CE10E944F
:1061200010A644E050E06EE170E0CE010B960E94B4
:10613000F2A58B859C85AD85BE858F3F2FEF92079D
:10614000A207B207A9F48AE090E4A0E0B0E080934F
:10615000620290936302A0936402B093650244E0EC
:1061600050E06EE170E082E692E00E9410A608C066
:106170008093620290936302A0936402B0936502DD
:106180008091620290916302A0916402B0916502D5
:10619000A2FF02C02A9A03C080E00E948E2544E03C
:1061A00050E06AE570E0CE010B960E94F2A58B8567
:1061B0009C85AD85BE858F3F2FEF9207A207B20762
:1061C00089F41092E30A1092E40A1092E50A109200
:1061D000E60A44E050E06AE570E083EE9AE00E944F
:1061E00010A608C08093E30A9093E40AA093E50AFE
:1061F000B093E60A49E050E06EE070E08BE595E38D
:106200000E94F2A50E941D0F44E050E06EE470E091
:10621000CE010B960E94F2A58B859C85AD85BE852F
:1062200044E050E06EE470E08F3F9F4FAF4FBF4FB0
:1062300029F482E892E00E9410A604C082E892E06D
:106240000E94F2A544E050E06AE470E0CE010B96B3
:106250000E94F2A58B859C85AD85BE8544E050E00B
:106260006AE470E08F3F9F4FAF4FBF4F29F48EE736
:1062700092E00E9410A604C08EE792E00E94F2A570
:1062800044E050E062E570E0CE010B960E94F2A57A
:106290008B859C85AD85BE8544E050E062E570E06D
:1062A0008F3F9F4FAF4FBF4F29F486E892E00E9487
:1062B00010A604C086E892E00E94F2A541E050E0FA
:1062C0006DE170E0CE0141960E94F2A5898941E01E
:1062D00050E06DE170E08F3F29F48FED9AE00E946D
:1062E00010A604C08FED9AE00E94F2A541E050E0B4
:1062F0006CE170E0CE0141960E94F2A5898941E0EF
:1063000050E06CE170E08F3F29F481E692E00E945A
:1063100010A604C081E692E00E94F2A541E050E0A0
:106320006BE170E0CE0141960E94F2A5898941E0BF
:1063300050E06BE170E08F3F29F480E692E00E942C
:1063400010A604C080E692E00E94F2A54AE050E068
:1063500064E070E0CE0101960E94F2A589814AE0D6
:1063600050E064E070E08F3F29F48CE59CE10E94EE
:1063700010A604C08CE59CE10E94F2A544E050E028
:1063800066E570E0CE010B960E94F2A58B859C8598
:10639000AD85BE8544E050E066E570E08F3F9F4FDD
:1063A000AF4FBF4F29F48AE892E00E9410A604C0C4
:1063B0008AE892E00E94F2A544E050E067E170E0D4
:1063C000CE010B960E94F2A58B859C85AD85BE857E
:1063D00044E050E067E170E08F3F9F4FAF4FBF4F09
:1063E00029F48CE592E00E9410A604C08CE592E0AE
:1063F0000E94F2A580915C0290915D02A0915E02E4
:10640000B0915F0281389A41A640B105A0F086EEB6
:1064100091E09F938F930E940CA380E197E2A0E00C
:10642000B0E080935C0290935D02A0935E02B09313
:106430005F020F900F9060915C0270915D028091FD
:106440005E0290915F020E941E6A42E050E062E0AC
:1064500070E0CE010F960E94F2A58F85988942E0E8
:1064600050E062E070E08F3F910529F48AED9AE0F8
:106470000E9410A604C08AED9AE00E94F2A542E0B4
:1064800050E060E070E0CE010F960E94F2A58F858B
:10649000988942E050E060E070E08F3F910529F478
:1064A00088ED9AE00E9410A604C088ED9AE00E9450
:1064B000F2A561960FB6F894DEBF0FBECDBFDF9197
:1064C000CF910895CF92DF92EF92FF9260917B027D
:1064D00070917C0280E090E00E9439A262ED75E04C
:1064E0000E944DA2892B09F03BC18DE48093751C5D
:1064F00080E88093761C84E08093771C1092781C4F
:106500001092791C10927A1C10927B1C10927C1CA9
:106510008CE390E090937E1C80937D1C10927F1CF6
:106520001092801C1092811C1092821C1092831C6D
:106530001092841C1092851C1092861C1092881C4C
:106540001092871C1092891C10928A1C10928B1C2E
:1065500010928C1C10928D1C10928E1C10928F1C0D
:106560001092901C1092921C1092911C1092931CED
:106570001092941C1092951C1092961C1092971CCD
:106580001092981C1092991C10929A1C10929C1CAC
:1065900010929B1C48E250E062E270E085E79CE1CB
:1065A0000E9410A68AE090E4A0E0B0E0809362022E
:1065B00090936302A0936402B093650244E050E0BC
:1065C0006EE170E082E692E00E9410A61092E30A6B
:1065D0001092E40A1092E50A1092E60A44E050E0B4
:1065E0006AE570E083EE9AE00E9410A682E2C82E6F
:1065F000DD24DA948CECE82E8BE3F82EC092820234
:10660000D0928302E0928402F092850244E050E04E
:106610006EE470E082E892E00E9410A6C0927E02D2
:10662000D0927F02E0928002F092810244E050E03A
:106630006AE470E08EE792E00E9410A687ED94E392
:10664000AFEEBCE38093860290938702A09388020A
:10665000B093890244E050E062E570E086E892E0A1
:106660000E9410A68AE999E9A9E1B0E480938A0220
:1066700090938B02A0938C02B0938D0244E050E083
:1066800066E570E08AE892E00E9410A61092DF0AA8
:1066900080E00E94FD7441E050E06DE170E08FED1C
:1066A0009AE00E9410A68AE1809361020E94A5737D
:1066B00041E050E06CE170E081E692E00E9410A6BB
:1066C0008FE08093600241E050E06BE170E080E693
:1066D00092E00E9410A68AE0ECE5FCE1DF011D9249
:1066E0008A95E9F74AE050E064E070E0CF010E944B
:1066F00010A680E197E2A0E0B0E080935C02909366
:106700005D02A0935E02B0935F0244E050E067E157
:1067100070E08CE592E00E9410A61092DB0A1092C5
:10672000DA0A42E050E062E070E08AED9AE00E940E
:1067300010A61092D90A1092D80A42E050E060E008
:1067400070E088ED9AE00E9410A681E00E94582532
:1067500080E090E0FF90EF90DF90CF900C94310FAD
:10676000FF90EF90DF90CF9008950E94FB706C9A9D
:106770006B9A6A9A6F9A729A749A739A779A8098B7
:1067800080B3897F80BB8398849887E080937E0064
:10679000549A0E94DC2F0E940D300E94CD0A80E0A6
:1067A00090E00E94310F60915C0270915D028091D7
:1067B0005E0290915F020E941E6A0E94E90C609343
:1067C0009430709395308093963090939730809169
:1067D000620286FD239A219A229A239A0E94E20A53
:1067E0001D9B05C01092E10A1092E00A089581E015
:1067F00090E09093E10A8093E00A0895CF93DF93AD
:1068000090E04091E30A5091E40A6091E50A7091AA
:10681000E60A41FD08C02091620220FD04C021FF6C
:106820008CC01D9B8AC02DE8289FE001299FD00DB8
:106830001124CE018E57924E9F938F9389ED95E050
:106840009F938F930E94F8A2FE01E558F24EDF015C
:10685000AA57BF4F2C910F900F900F900F9043812C
:106860005481658176818091983090919930A09182
:106870009A30B0919B30841B950BA60BB70B22234B
:10688000D1F1BF93AF939F938F93DF01A257BF4F77
:1068900011968C9111978F938C918F9312971196DB
:1068A0008C9111978F938C918F9313978C911F924A
:1068B0008F9311978C911F928F9313968C911F92A7
:1068C0008F9311978C911F928F93E957FF4F80817F
:1068D0001F928F931F922F938FED95E09F938F932D
:1068E0000E94F8A28DB79EB746960FB6F8949EBF49
:1068F0000FBE8DBF10C0BF93AF939F938F9386E25F
:1069000096E09F938F930E94F8A20F900F900F90A4
:106910000F900F900F900E94E60D80917D028823CA
:1069200061F01F928F9383EE91E09F938F930E946B
:106930000CA30F900F900F900F90DF91CF910895BF
:1069400080917B1D882341F080917C1D90E00E9406
:10695000FE330E94D30BF4CF0895CF93DF93EC0165
:106960008881998185332FE09207E9F018F4892B0B
:10697000B9F048C08D332FE0920709F449C0813443
:106980009F4009F03FC085EF9AE00E948A61892B01
:10699000E9F185EF9AE00E946D6180E00E94882510
:1069A00085E39FE02CC0623189F5299A6091D80A6D
:1069B0007091D90A7695762F66277795679585EF3A
:1069C0009AE00E9463618091E30A9091E40AA091A9
:1069D000E50AB091E60AA0FF10C08091D90A8F9312
:1069E0008091D80A8F938DED90E19F938F930E94B1
:1069F0000CA30F900F900F900F908DE39FE0998361
:106A0000888304C01982188283E017C081E015C012
:106A100085EF9AE00E948A61892BC1F385EF9AE0A5
:106A20000E946D610E94A03460E270E085EF9AE000
:106A30000E94636181E49FE0E2CFDF91CF910895EE
:106A40002F923F924F925F926F927F928F929F927E
:106A5000AF92BF92CF92DF92EF92FF920F931F936C
:106A6000CF93DF93CDB7DEB72B970FB6F894DEBF89
:106A70000FBECDBF9B878A873A01FC01808191813F
:106A8000892B11F00C94CE4960917B0270917C02AD
:106A9000CA010E9439A260E870E0C3010E946CA2A2
:106AA000009759F460912E3E70912F3E8AE090E05D
:106AB0000E94C0A281E00C94D3498130910561F419
:106AC000F3011081912E990C9908892C092D292CFC
:106AD000392C492C592CB9C082309105B9F4F301F5
:106AE0008081082E000C990B982F88272181820F16
:106AF000911D27FD9A95182F992E892E880C8808AC
:106B0000082D282C382C482C582C9FC083309105F8
:106B1000B1F5F3012081922F990F990B392F492F4D
:106B2000592F692F792F892F00E10E94FB9D1901B0
:106B30002A014B01B82FA92F2181922F990F990B70
:106B4000392F492F592F692F792F892F08E00E945B
:106B5000FB9D59016A017B018C019101A201B401E5
:106B60008B2F9A2F0E94329EA2801A2D110F110B8B
:106B7000B12EC12ED12EE12EF12E012F55C004973A
:106B80000CF45BC0F3012081922F990F990B392FE0
:106B9000492F592F692F792F892F08E10E94FB9DDA
:106BA00019012A014B01B82FA92F2181922F990F8A
:106BB000990B392F492F592F692F792F892F00E1F0
:106BC0000E94FB9D59016A017B018C019101A20188
:106BD000B4018B2F9A2F0E94329EA3801A2D110F81
:106BE000110BB12EC12ED12EE12EF12E012F0E94BC
:106BF000329E19012A014B01B82FA92F2281922F11
:106C0000990F990B392F492F592F692F792F892FD8
:106C100008E00E94FB9D59016A017B018C019101F2
:106C2000A201B4018B2F9A2F0E94329E122F932E15
:106C3000842E052F1B012C0108C01AE0912C812CF9
:106C400000E0212C312C412C512C0E94E60D212FEB
:106C5000392D482D502FB101C2012537F3E63F07EA
:106C6000FDE64F075105610571058105910511F498
:106C70000C9443442537E3E63E07EDE64E07510505
:106C8000610571058105910511F008F0B2C1233746
:106C9000F2E73F0741055105610571058105910541
:106CA00011F40C94DC462337E2E73E074105510519
:106CB000610571058105910511F008F0B9C025360F
:106CC000F4E63F0741055105610571058105910510
:106CD00009F4DBC72536E4E63E07410551056105A9
:106CE00071058105910511F008F041C0A6E70E94E9
:106CF000599E11F40C94C7400E94599E09F070F4FB
:106D0000A8E60E94599E11F40C94963EA5E70E94B5
:106D1000599E11F40C94B1400C94CC49212F392D7B
:106D2000482D502FB101C2012436F1E63F0741053D
:106D30005105610571058105910511F40C94044715
:106D40002537E2E63E0741055105610571058105DC
:106D5000910509F431C52A333642410551056105D3
:106D600071058105910509F430C30C94CC49212F9C
:106D7000392D482D502FB101C2012737EFE63E07CC
:106D800041055105610571058105910511F40C94CA
:106D9000A9442737FFE63F07410551056105710505
:106DA0008105910509F0C8F42436E9E63E0741055E
:106DB0005105610571058105910511F40C948A4016
:106DC00025363E4641055105610571058105910550
:106DD00011F40C94DD440C94CC49212F392D482D0D
:106DE000502FB101C2012536E2E73E0741055105AA
:106DF000610571058105910511F40C94A9452936A9
:106E0000F2E73F07410551056105710581059105CF
:106E100011F40C948B46233331474105510561052C
:106E200071058105910511F00C94CC490C9404472F
:106E3000212F392D482D502FB101C2012236F5E600
:106E40003F07F4E64F07510561057105810591057E
:106E500009F41BC72236E5E63E07E4E64E07510576
:106E6000610571058105910511F008F05BC02133C2
:106E7000F4E63F07F1E64F0751056105710581050D
:106E8000910509F4B6C22133E4E63E07E1E64E0778
:106E90005105610571058105910509F0C0F423379D
:106EA000F3E73F074105510561057105810591052E
:106EB00011F40C94F046283734474105510561051B
:106EC00071058105910509F480C20C94CC49212FEC
:106ED000392D482D502FB101C2012837F4E63F0764
:106EE000F1E64F075105610571058105910509F42A
:106EF0007CC22C36E5E73E07E2E64E075105610508
:106F000071058105910509F457C42336344641467D
:106F10005105610571058105910511F00C94CC496D
:106F20000C940447212F392D482D502FB101C20157
:106F30002D36E5E73E07E8E64E0751056105710588
:106F40008105910511F40C941A472D36F5E73F079A
:106F5000F8E64F075105610571058105910509F0B6
:106F6000E0F42237E2E73E07E5E64E07510561050A
:106F700071058105910511F40C94F44323363D46C7
:106F800048465105610571058105910511F00C9484
:106F9000CC490E9409190C94CE49212F392D482D36
:106FA000502FB101C2012436E3E63E07ECE64E075E
:106FB0005105610571058105910511F40C94574344
:106FC0002736FFE63F07FCE64F07510561057105CF
:106FD0008105910511F40C945A43233632434946F6
:106FE0005105610571058105910511F00C94CC499D
:106FF00020C2212F392D482D502FB101C201203739
:10700000FCE63F07F5E64F07F8E65F076105710507
:107010008105910509F48AC62037ECE63E07E5E6CE
:107020004E07E8E65E07610571058105910511F0DF
:1070300008F0E0C02437F8E73F07F4E74F075105B1
:10704000610571058105910511F40C9433412437D4
:10705000E8E73E07E4E74E07510561057105810544
:10706000910511F008F05DC02033F1E33F07F1E72F
:107070004F075105610571058105910511F40C94C7
:10708000F4432033E1E33E07E1E74E075105610594
:1070900071058105910509F0C0F42133F2E63F073F
:1070A000F0E74F075105610571058105910509F468
:1070B00098C222333246404751056105710581056A
:1070C000910509F4E3C20C94CC49212F392D482DA8
:1070D000502FB101C2012037F5E63F07F2E74F0715
:1070E0005105610571058105910511F40C94A945BF
:1070F0002C36E4E73E074E07510561057105810511
:10710000910511F40C94F248213331434147510564
:10711000610571058105910511F00C94CC490C9421
:107120004344212F392D482D502FB101C2012B3658
:10713000ECE63E07E5E74E07E2E65E07610571050E
:107140008105910509F438C32B36FCE63F07F5E7C6
:107150004F07F2E65F07610571058105910509F0AA
:10716000E0F42437E4E63E07E7E74E075105610502
:1071700071058105910511F40C94404924373F466F
:107180004F465246610571058105910511F00C9439
:10719000CC490C9400000C94CE49212F392D482D58
:1071A000502FB101C2012E36E1E63E07E8E64E0758
:1071B000E3E65E07610571058105910511F40C9404
:1071C00007412633F9E63F07F5E74F07F5E65F0786
:1071D000610571058105910509F4ACC529363C4668
:1071E00041465346610571058105910511F00C94E6
:1071F000CC4989C3212F392D482D502FB101C2010F
:107200002437F3E73F07F5E64F07F2E75F0761052D
:1072100071058105910511F40C9459452437E3E774
:107220003E07E5E64E07E2E75E0761057105810569
:10723000910511F008F062C02337F5E63F07F2E749
:107240004F07F0E75F07610571058105910511F4AE
:107250000C94CA472337E5E63E07E2E74E07E0E72E
:107260005E07610571058105910509F0D0F42136AD
:10727000FDE63F07F5E74F07F8E65F076105710593
:107280008105910511F40C94C744223737474047D4
:107290005047610571058105910509F45CC20C94A4
:1072A000CC49212F392D482D502FB101C201243650
:1072B000FDE63F07F3E64F07F2E75F07610571055B
:1072C0008105910509F441C62136ECE63E07E5E665
:1072D0004E07E2E75E07610571058105910509F436
:1072E00046C5233732474747504761057105810539
:1072F000910511F00C94CC490C945C45212F392D4B
:10730000482D502FB101C2012437E2E73E07E1E6E4
:107310004E07E5E75E07610571058105910509F4F2
:107320006FC62437F2E73F07F1E64F07F5E75F073F
:10733000610571058105910509F0C8F42437E3E77B
:107340003E07E5E64E07E4E75E0761057105810546
:10735000910509F4B3C727373047484754476105BB
:1073600071058105910509F428C70C94CC49212F9A
:10737000392D482D502FB101C2012F36ECE63E07C2
:10738000EFE54E07E6E75E076105710581059105AA
:1073900009F486C52C36F1E63F07F4E74F07F8E716
:1073A0005F07610571058105910511F40C94BC48D6
:1073B00022373746404755476105710581059105DC
:1073C00011F00C94CC490C94334383E080934935FD
:1073D00010924B3510924A3549E455E362E18EE351
:1073E00092E00E94DE5E0C94CE490E9491180C94AB
:1073F000CE4921E042E161E080ED0E94FB6B21E09B
:1074000042E161E080ED0E94FB6B21E042E161E03E
:1074100080ED0E94FB6B21E042E161E080ED0E9483
:10742000FB6B21E042E161E080ED0E94FB6B0C947C
:10743000CE4960917B0270917C0280E090E00E94D6
:1074400039A262E376E00E944DA2892B09F0C5C003
:1074500060917B0270917C0280E090E00E9439A2F2
:107460008C01009709F497C06AEF73E00E944DA267
:10747000892BE1F488EE93E0A0E0B0E080935C0219
:1074800090935D02A0935E02B0935F0268EE73E09A
:1074900080E090E00E941E6A44E050E067E170E006
:1074A0008CE592E00E9410A60C94CE4968E376E049
:1074B000C8010E944DA2892BE1F480E197E2A0E08F
:1074C000B0E080935C0290935D02A0935E02B09363
:1074D0005F0260E177E280E090E00E941E6A44E093
:1074E00050E067E170E08CE592E00E9410A60C94F9
:1074F000CE496BE376E0C8010E944DA2892BE1F4EE
:1075000080EA96E8A1E0B0E080935C0290935D028F
:10751000A0935E02B0935F0260EA76E881E090E0BB
:107520000E941E6A44E050E067E170E08CE592E062
:107530000E9410A60C94CE496FE376E0C8010E9429
:107540004DA2892BE1F480E89AE1A6E0B0E08093B7
:107550005C0290935D02A0935E02B0935F0260E8CC
:107560007AE186E090E00E941E6A44E050E067E124
:1075700070E08CE592E00E9410A60C94CE4981E95F
:1075800093E09F938F930E940CA30E94E60D0F90AF
:107590000F900C94CE4960915C0270915D028091D5
:1075A0005E0290915F0228EE33E040E050E00E94DE
:1075B0001E9C5F934F933F932F938DE893E09F938F
:1075C0008F930E940CA30E94E60D0F900F900F90D6
:1075D0000F900F900F900C94CE490E94D6120C94ED
:1075E000CE4960917B0270917C0280E090E00E9425
:1075F00039A28C016BEC75E00E944DA2892BA1F49D
:107600008091620290916302A0916402B091650240
:10761000A2608093620290936302A0936402B0938D
:107620006502299A0C94CE496EEC75E0C8010E945F
:107630004DA2892BB1F48091620290916302A091D6
:107640006402B0916502AD7F809362029093630201
:10765000A0936402B093650280E00E9488250C9498
:10766000CE49299903C08EEC95E002C08BEC95E0E1
:107670009F938F9385E893E09F938F930E940CA331
:107680000F900F900F900F900C94CE4960917B0259
:1076900070917C0280E090E00E9439A28C016BEC3A
:1076A00075E00E944DA2892BE1F4809162029091D5
:1076B0006302A0916402B0916502A46080936202AB
:1076C00090936302A0936402B09365022A9A44E007
:1076D00050E06EE170E082E692E00E9410A60C9409
:1076E000CE496EEC75E0C8010E944DA2892BF1F4E1
:1076F0008091620290916302A0916402B091650250
:10770000AB7F8093620290936302A0936402B09374
:10771000650280E00E948E2544E050E06EE170E05A
:1077200082E692E00E9410A60C94CE492A9903C0EA
:107730008EEC95E002C08BEC95E09F938F938DE7E4
:1077400093E09F938F930E940CA30F900F900F9044
:107750000F900C94CE4960917B0270917C0280E086
:1077600090E00E9439A28C016BEC75E00E944DA262
:10777000892B19F477980C94CE496EEC75E0C8010A
:107780000E944DA2892B19F4779A0C94CE49779BCD
:1077900003C08EEC95E002C08BEC95E09F938F9335
:1077A00081E595E09F938F930E940CA30F900F901B
:1077B0000F900F900C94CE4960917B0270917C02E7
:1077C00080E090E00E9439A28C0163E476E00E94A0
:1077D0004DA2892BD1F480917B1D1F928F938091B4
:1077E0007D1D1F928F9380917C1D1F928F931F92FE
:1077F00084E18F9383E593E09F938F930E940CA382
:107800000FB6F894DEBF0FBECDBF68E476E0C801C6
:107810000E944DA2892B19F40E94A03470C060E52B
:1078200076E0C8010E944DA2892B09F047C0609103
:107830007B0270917C0280E090E00E9439A2009768
:1078400009F45DC00E9426A18531910570F59093E1
:10785000DB0A8093DA0A42E050E062E070E08AEDF1
:107860009AE00E9410A660917B0270917C0280E0F9
:1078700090E00E9439A2009709F441C00E9426A11D
:107880009093D90A8093D80A42E050E060E070E01B
:1078900088ED9AE00E9410A660917B0270917C02B4
:1078A00080E090E00E9439A22AC081E493E09F9397
:1078B0008F930E940CA30F900F9021C08091DB0A40
:1078C0008F938091DA0A8F9388E393E09F938F934D
:1078D0000E940CA30E94E60D8091D90A8F9380919B
:1078E000D80A8F9389E293E09F938F930E940CA311
:1078F0000E94E60D0FB6F894DEBF0FBECDBF0E940A
:10790000E60D0C94CE4960917B0270917C0280E080
:1079100090E00E9439A28C0164E775E00E944DA2BC
:10792000892B09F077C060917B0270917C0280E026
:1079300090E00E9439A28C01009711F40C94CE497A
:107940006EE476E00E944DA2892BB1F482E29FEFB3
:10795000ACECBBE38093820290938302A0938402F9
:10796000B093850244E050E06EE470E082E892E07B
:107970000E9410A60C94CE4964E576E0C8010E94EE
:107980004DA2892BB1F482E29FEFACECBAE3809375
:10799000820290938302A0938402B093850244E014
:1079A00050E06EE470E082E892E00E9410A60C9431
:1079B000CE49C8010E9422A12B013C0120E030E009
:1079C000A9010E945A988823D9F081E00E94870C6F
:1079D0009B01AC01C301B2010E945F9860938202D7
:1079E00070938302809384029093850244E050E078
:1079F0006EE470E082E892E00E9410A60C94CE49FA
:107A00008CE193E09F938F930E940CA30F900F90B3
:107A10000C94CE4967E775E0C8010E944DA2892BFE
:107A200009F077C060917B0270917C0280E090E069
:107A30000E9439A28C01009711F40C94CE496EE497
:107A400076E00E944DA2892BB1F482E29FEFACEC6C
:107A5000BBE380937E0290937F02A0938002B09359
:107A6000810244E050E06AE470E08EE792E00E9418
:107A700010A60C94CE4964E576E0C8010E944DA2A0
:107A8000892BB1F482E29FEFACECBAE380937E02E3
:107A900090937F02A0938002B093810244E050E073
:107AA0006AE470E08EE792E00E9410A60C94CE4942
:107AB000C8010E9422A12B013C0120E030E0A90175
:107AC0000E945A988823D9F082E00E94870C9B017B
:107AD000AC01C301B2010E945F9860937E02709373
:107AE0007F02809380029093810244E050E06AE438
:107AF00070E08EE792E00E9410A60C94CE498FE0D1
:107B000093E09F938F930E940CA30F900F900C947F
:107B1000CE496FE675E0C8010E944DA2892B09F09D
:107B200073C060917B0270917C0280E090E00E94C3
:107B300039A28C01009711F40C94CE496EE476E0E2
:107B40000E944DA2892BB1F487ED94E3AFEEBCE324
:107B50008093860290938702A0938802B093890253
:107B600044E050E062E570E086E892E00E9410A6F2
:107B70000C94CE4964E576E0C8010E944DA2892BA1
:107B800051F480E093E09F938F930E940CA30F9099
:107B90000F900C94CE49C8010E9422A12B013C01F8
:107BA00020E030E0A9010E945A98882319F180E072
:107BB0000E94870C4B015C0121EE3AE744E95EE349
:107BC000C301B2010E947B97A50194010E945F98B6
:107BD0006093860270938702809388029093890253
:107BE00044E050E062E570E086E892E00E9410A672
:107BF0000C94CE4983EF92E09F938F930E940CA345
:107C00000F900F900C94CE490E94D50C9F938F93A8
:107C10007F936F938CEE92E09F938F930E940CA3BF
:107C200082E00E94870C20917E0230917F02409179
:107C30008002509181020E940B9B162F072FF82E75
:107C4000E92E81E00E94870CEF92FF920F931F9321
:107C500020918202309183024091840250918502EA
:107C60000E940B9B9F938F937F936F9380EE92E084
:107C70009F938F930E940CA30E94E60D0FB6F89479
:107C8000DEBF0FBECDBF0C94CE4960917B027091D8
:107C90007C0280E090E00E9439A2009711F10E94DE
:107CA0008D260091E30A1091E40A2091E50A3091B3
:107CB000E60A601771078207930739F16093E30AB8
:107CC0007093E40A8093E50A9093E60A44E050E05A
:107CD0006AE570E083EE9AE00E9410A68AE495E0DF
:107CE00002C083E495E09F938F930E940CA3609160
:107CF000E30A7091E40A8091E50A9091E60A0E94F5
:107D00009A250E94E60D0F900F9088E395E09F93CF
:107D10008F930E940CA36FEF7FEFCB010E949A25F7
:107D20000E94E60D0F900F900C94CE490E94752290
:107D30000C94CE49F3018481843329F440E061E05E
:107D400080E00E94AC1480917D02882311F40C9491
:107D5000CE491F928F9385E395E09F938F930E9466
:107D60000CA30F900F900F900F900C94CE49F3013D
:107D70008481893709F080C060917B0270917C0218
:107D800080E090E00E9439A28C016BEC75E00E94CB
:107D90004DA2892B51F48091620290916302A091CF
:107DA0006402B0916502906410C06EEC75E0C80189
:107DB0000E944DA2892BD1F48091620290916302BE
:107DC000A0916402B09165029F7B809362029093C0
:107DD0006302A0936402B093650244E050E06EE158
:107DE00070E082E692E00E9410A646C069E576E067
:107DF000C8010E944DA2892B21F58091741C8F939C
:107E00008091731C8F938091721C8F938091711C51
:107E10008F938091701C8F9380916F1C8F938091B2
:107E20006E1C8F9380916D1C8F9385EB92E09F93D6
:107E30008F930E940CA30FB6F894DEBF0FBECDBF88
:107E40001BC08091620290916302A0916402B09184
:107E5000650296FD03C08EEC95E002C08BEC95E0C8
:107E60009F938F9381EB92E09F938F930E940CA33B
:107E70000F900F900F900F9080917D02882311F446
:107E80000C94CE491F928F9382E395E09F938F933A
:107E90000E940CA30F900F900F900F900C94CE495E
:107EA000F30184818737E9F560917B0270917C0250
:107EB00080E090E00E9439A20097D9F00E9422A1B0
:107EC0002B013C0120E030E0A9010E945A98882350
:107ED00081F040928A0250928B0260928C027092E2
:107EE0008D0244E050E066E570E08AE892E00E948E
:107EF00010A680918D028F9380918C028F93809138
:107F00008B028F9380918A028F9383EA92E09F93F2
:107F10008F930E940CA30F900F900F900F900F90D3
:107F20000F9080917D02882311F40C94CE491F920A
:107F30008F938FE295E09F938F930E940CA30F90F5
:107F40000F900F900F900C94CE4960917B0270912E
:107F50007C0280E090E00E9439A28C016BEC75E01D
:107F60000E944DA2409062025090630260906402B1
:107F700070906502892B19F4689457F809C06EEC6B
:107F800075E0C8010E944DA2892B99F4E89457F836
:107F900040926202509263026092640270926502A3
:107FA00044E050E06EE170E082E692E00E9410A6AC
:107FB00013C057FC03C08EEC95E002C08BEC95E03B
:107FC0009F938F938FE992E09F938F930E940CA3CE
:107FD0000F900F900F900F9080917D02882311F4E5
:107FE0000C94CE491F928F938CE295E09F938F93D0
:107FF0000E940CA30F900F900F900F900C94CE49FD
:1080000060917B0270917C0280E090E00E9439A236
:108010008C016FE576E00E944DA2892B11F489E175
:1080200008C063E676E0C8010E944DA2892B49F49E
:1080300080E18093C4001092C50082E08093C0006C
:1080400055C067E676E0C8010E944DA2892B11F465
:1080500088E0EFCF6CE676E0C8010E944DA2892B44
:1080600039F061E776E0C8010E944DA2892B11F436
:1080700083E0DFCF8091C400893141F48AE992E046
:108080009F938F930E940CA30F900F908091C40038
:10809000803141F485E992E09F938F930E940CA375
:1080A0000F900F908091C400883041F48FE892E0E7
:1080B0009F938F930E940CA30F900F908091C40008
:1080C000833041F489E892E09F938F930E940CA340
:1080D0000F900F908091C400883041F483E892E0C3
:1080E0009F938F930E940CA30F900F9080917D021D
:1080F000882311F40C94CE491F928F9389E295E066
:108100009F938F930E940CA30F900F900F900F904E
:108110000C94CE4960917B0270917C0280E090E0EB
:108120000E9439A26EE476E00E944DA2892B11F4E0
:1081300081E001C080E00E94582580917D02882363
:1081400011F40C94CE491F928F9386E295E09F9391
:108150008F930E940CA30F900F900F900F900C9490
:10816000CE490E947C2380917D02882311F40C94D7
:10817000CE491F928F9383E295E09F938F930E9445
:108180000CA30F900F900F900F900C94CE490E946B
:10819000782380917D02882311F40C94CE491F929C
:1081A0008F9380E295E09F938F930E940CA30F9092
:1081B0000F900F900F900C94CE4960917B027091BC
:1081C0007C0280E090E00E9439A20E9426A18031CA
:1081D00070F48093DF0A0E94FD7441E050E06DE18D
:1081E00070E08FED9AE00E9410A60C94CE49809129
:1081F000DF0A1F928F9389E792E09F938F930E94EB
:108200000CA30F900F900F900F900C94CE4960919B
:108210007B0270917C0280E090E00E9439A20E9473
:1082200026A195EF980F903170F4809361020E941F
:10823000A57341E050E06CE170E081E692E00E94BD
:1082400010A60C94CE49809161021F928F9380E713
:1082500092E09F938F930E940CA30F900F900F902A
:108260000F900C94CE4960917B0270917C0280E06B
:1082700090E00E9439A2009789F04AE050E0BC01EA
:108280008CE59CE10E945DA24AE050E064E070E071
:108290008CE59CE10E9410A60C94CE498CE59CE1F3
:1082A0009F938F9386E796E09F938F930E94F8A207
:1082B0000F900F900F900F900C94CE4960917B021D
:1082C00070917C0280E090E00E9439A28C016AEFFC
:1082D00073E00E944DA2892BE1F4219A8091620201
:1082E00090916302A0916402B091650280618093D5
:1082F000620290936302A0936402B093650244E02B
:1083000050E06EE170E082E692E00E9410A60C94CC
:10831000CE4968E775E0C8010E944DA2892BE1F4BF
:10832000229A8091620290916302A0916402B091BE
:10833000650280628093620290936302A09364025C
:10834000B093650244E050E06EE170E082E692E0B6
:108350000E9410A60C94CE496CED73E0C8010E94F7
:108360004DA2892BE1F4239A8091620290916302DD
:10837000A0916402B0916502806480936202909340
:108380006302A0936402B093650244E050E06EE1A2
:1083900070E082E692E00E9410A60C94CE496BE158
:1083A00075E0C8010E944DA2892BE1F4239A8091C7
:1083B000620290916302A0916402B09165028068AC
:1083C0008093620290936302A0936402B09365026B
:1083D00044E050E06EE170E082E692E00E9410A678
:1083E0000C94CE4967E87AE0C8010E944DA2892B1F
:1083F00071F581E08093AD3085E79CE19093AF30DB
:108400008093AE301092B1301092B0308091620201
:1084100090916302A0916402B09165029160809393
:10842000620290936302A0936402B093650244E0F9
:1084300050E06EE170E082E692E00E9410A64DEA04
:1084400050E362E18EE392E00E94DE5EA7C763E044
:1084500074E0C8010E944DA2892B11F5E5EAFCE108
:10846000119211922CE1E53CF207D1F78091620262
:1084700090916302A0916402B09165029260809332
:10848000620290936302A0936402B093650244E099
:1084900050E06EE170E082E692E00E9410A67EC796
:1084A0006EEC75E0C8010E944DA2409162025091AD
:1084B00063026091640270916502892BC1F44F7070
:1084C0005C7F4093620250936302609364027093F6
:1084D00065022B9A44E050E06EE170E082E692E0A3
:1084E0000E9410A6809152350E94BA7357C744FD6E
:1084F00003C08EEC95E002C08BEC95E09F938F93C8
:1085000085E692E09F938F930E940CA38091620274
:108510000F900F900F900F9085FD03C08EEC95E0AB
:1085200002C08BEC95E09F938F938AE592E09F9336
:108530008F930E940CA3809162020F900F900F9076
:108540000F9086FD03C08EEC95E002C08BEC95E0A9
:108550009F938F938FE492E09F938F930E940CA33D
:10856000809162020F900F900F900F9087FD03C0D3
:108570008EEC95E002C08BEC95E09F938F9384E4A2
:1085800092E09F938F930E940CA38091620290913E
:108590006302A0916402B09165020F900F900F905A
:1085A0000F9090FD03C08EEC95E002C08BEC95E03F
:1085B0009F938F9389E392E09F938F930E940CA3E4
:1085C0008091620290916302A0916402B091650271
:1085D0000F900F900F900F9091FD03C08EEC95E0DF
:1085E00002C08BEC95E09F938F938EE292E09F9375
:1085F0008F930E940CA38091620290916302A091DC
:108600006402B09165020F900F900F900F9091FF50
:10861000C5C68EE796E00E9434A395EAE92E9CE158
:10862000F92E00E010E026E8822E26E0922EF701D7
:1086300080819181F2E0EF0EF11C9F938F93C8012E
:108640000B969F938F939F928F920E94F8A20F5F39
:108650001F4F0F900F900F900F900F900F900031C1
:10866000110529F79BC68CE195E09F938F930E949B
:108670000CA380917D020F900F90882361F01F92D0
:108680008F9389E195E09F938F930E940CA30F90A5
:108690000F900F900F90F89498E088E10FB6F8943F
:1086A000A895809360000FBE90936000FFCF0E945A
:1086B000AC6B74C660917B0270917C0280E090E0AC
:1086C0000E9439A28C016BEC75E00E944DA2892BAF
:1086D000E9F40E94A0728091620290916302A091DD
:1086E0006402B09165028D7F8160809362029093F5
:1086F0006302A0936402B093650244E050E06EE12F
:1087000070E082E692E00E9410A648C66EEC75E02A
:10871000C8010E944DA2892BE1F40E9458728091F9
:10872000620290916302A0916402B09165028C7F15
:108730008093620290936302A0936402B0936502F7
:1087400044E050E06EE170E082E692E00E9410A604
:1087500025C661E976E0C8010E944DA2892BE9F4A3
:108760000E9458728091620290916302A09164020B
:10877000B09165028E7F8260809362029093630263
:10878000A0936402B093650244E050E06EE170E0B3
:1087900082E692E00E9410A601C68091620281FFEB
:1087A0000FC081E996E09F938F938AE292E09F93B6
:1087B0008F930E940CA30F900F900F900F90EEC517
:1087C00080FD03C08EEC95E002C08BEC95E09F939A
:1087D0008F9386E292E09F938F930E940CA30F9059
:1087E0000F900F900F90DAC58091AB308F938091EE
:1087F000AA308F938091A9308F938091A8308F9366
:108800008091A7308F938091A6308F938091A5306F
:108810008F938091A4308F938091A3308F93809118
:10882000A2308F938091A1308F938091A0308F934D
:1088300080919F308F9380919E308F9380919D3057
:108840008F9380919C308F938DEE94E09F938F93C4
:108850000E940CA30E94E60D80917D020FB6F89451
:10886000DEBF0FBECDBF882309F498C51F928F933A
:108870008AEE94E09F938F930E940CA30F900F9029
:108880000F900F908BC5F89489E021E030E0F9015A
:1088900080935700C895E02C20E030E0F9018093E8
:1088A0005700C895F02C7894F89423E030E0F90153
:1088B00080935700C895002D22E030E0F9018093A5
:1088C0005700C895102D7894809185288F938091BA
:1088D00084288F93809183288F93809182288F930F
:1088E00080EE94E09F938F930E940CA31F92EF92CF
:1088F0001F92FF921F920F931F921F9389EB94E098
:108900009F938F930E940CA30E941624809166006F
:108910001F928F938DEA94E09F938F930E940CA3F4
:108920000E94E60D80917D020FB6F894DEBF0FBE67
:10893000CDBF882309F432C51F928F938AEA94E051
:108940009F938F930E940CA30F900F900F900F9006
:1089500025C560E070E080E090E00E94EF0D60E0EF
:1089600070E081E090E00E94EF0D80917D0288230D
:1089700009F414C51F928F9387EA94E09F938F9315
:108980000E940CA30F900F900F900F9007C50E94AC
:1089900038220E94E60D80917D02882309F4FEC4EE
:1089A0001F928F9384EA94E09F938F930E940CA36D
:1089B0000F900F900F900F90F1C460917B02709117
:1089C0007C0280E090E00E9439A268E476E00E9498
:1089D0004DA2892B31F5F89484E29BE00E94CD5F93
:1089E0008C01892B69F0C8010F960E94D562B801ED
:1089F00084E092E00E94865FC8010E947960F0CF17
:108A000084E29BE00E945E60892B29F084E29BE077
:108A10000E940660F5CF84E29BE00E94C95F7894D3
:108A200036C084E29BE00E94CD5F8C0186E9E82E8F
:108A300086E0F82E0115110551F1F80186811F928B
:108A40008F9380851F928F9385811F928F9381854D
:108A50001F928F9387811F928F9384811F928F9390
:108A600083811F928F9382811F928F9382851F92A1
:108A70008F93FF92EF920E94F8A2C8010E94796042
:108A80008C010FB6F894DEBF0FBECDBFD3CF80915F
:108A90007D02882309F482C41F928F9381EA94E0B7
:108AA0009F938F930E940CA30F900F900F900F90A5
:108AB00075C40E94623272C460917B0270917C0224
:108AC00080E090E00E9439A28C0165ED76E00E9482
:108AD0004DA2892BD1F48091620290916302A09102
:108AE0006402B0916502977F809362029093630263
:108AF000A0936402B093650244E050E06EE170E040
:108B000082E692E00E9410A649C464E576E0C801BE
:108B10000E944DA2892BD1F4809162029091630250
:108B2000A0916402B0916502986080936202909374
:108B30006302A0936402B093650244E050E06EE1EA
:108B400070E082E692E00E9410A628C40E945F0AAC
:108B500025C460917B0270917C0280E090E00E94CD
:108B600039A2FC0120812332C1F44AE050E060E0E8
:108B700070E001960E94BF9E7B836A8360917B02B6
:108B800070917C0280E090E00E9439A22A813B81B2
:108B9000243031050CF096C002C01B821A82009767
:108BA00009F490C01982BE016F5F7F4F0E945C2B59
:108BB00019013A014B01B82FA92F8AE02A813B8184
:108BC000829FF001839FF00D1124EB58F34E4080FB
:108BD000518032813C8383818D8394819E83258162
:108BE0002F8336813887878189879101A301B4015A
:108BF0008B2F9A2F5201CC80DD80EE80FF8008857C
:108C000019850E94509E09F460C08981811103C0BA
:108C1000208231822AC0181684F4422853289C816D
:108C2000692A2D81722A3E81832A8F81982A98850C
:108C3000B92B2985A22B408217C0209430946094D0
:108C4000709480949094B095A095242053203C81FA
:108C500063228D8178229E8189222F8192223885FC
:108C6000B3238985A8232082518262827382848201
:108C70009582B683A78348E250E062E270E085E720
:108C80009CE10E9410A689E994E09F938F930E9433
:108C90000CA38AE02A813B81829FF001839FF00D23
:108CA0001124EB58F34E208131814281538164813C
:108CB0007581868197810E9446270E94E60D0F905C
:108CC0000F9003C082E00E94362D8DE894E09F93C0
:108CD0008F930E940CA32FEF3FEF4FEF5FEF6FEFEB
:108CE0007FEF8FEF9FEF0E9446270E94E60D809155
:108CF0007D020F900F90882309F450C31F928F9329
:108D00008AE894E09F938F930E940CA30F900F909A
:108D10000F900F9043C360917B0270917C0280E0C2
:108D200090E00E9439A2FC0120812332A1F44AE0A4
:108D300050E060E070E001960E94BF9E8B01609160
:108D40007B0270917C0280E090E00E9439A20430A6
:108D50001105ECF402C000E010E00097C1F04AE019
:108D600050E060E070E00E94EA9F2AE0209FF0015E
:108D7000219FF00D1124EB58F34E7187608748E274
:108D800050E062E270E085E79CE10E9410A681E07D
:108D90000E94362D80917D02882309F4FFC21F9224
:108DA0008F9387E894E09F938F930E940CA30F907A
:108DB0000F900F900F90F2C20E940D6380917D0280
:108DC000882309F4EBC21F928F9384E894E09F9369
:108DD0008F930E940CA30F900F900F900F90DEC204
:108DE0000E94FB2D80917D02882309F4D7C21F9237
:108DF0008F9381E894E09F938F930E940CA30F9030
:108E00000F900F900F90CAC280E090E00E94322431
:108E100080917D02882309F4C1C21F928F938EE74F
:108E200094E09F938F930E940CA30F900F900F904C
:108E30000F90B4C28091922C81FF2DC00E94BE2160
:108E4000892B49F5809189288F93809188288F9369
:108E5000809187288F93809186288F9383E794E071
:108E60009F938F930E940CA3809176358F9380916E
:108E700075358F93809174358F93809173358F936F
:108E800086E694E09F938F930E940CA30FB6F8940C
:108E9000DEBF0FBECDBF0E94E60D8091922C909157
:108EA000932C93FF63C081E090E00E9435217B0109
:108EB0001C0180E090E00E9435214B018C010E9452
:108EC00093203F922F92FF92EF9285E594E09F933B
:108ED0008F930E940CA31F930F939F928F9285E410
:108EE00094E09F938F930E940CA324013801940176
:108EF000A80147018101B701C1010E94321F9F9360
:108F00008F937F936F938AE394E09F938F930E9454
:108F10000CA3242D352D462D572D6E2D792D822D08
:108F2000912F0E94931F9F938F937F936F938CE257
:108F300094E09F938F930E940CA3242D352D462DF2
:108F4000572D6E2D792D822D912F0E94F41F9F9306
:108F50008F937F936F9389E194E09F938F930E9407
:108F60000CA30FB6F894DEBF0FBECDBF0E94E60D76
:108F700080917D02882309F411C21F928F9386E1AC
:108F800094E09F938F930E940CA30F900F900F90EB
:108F90000F9004C28091922C82FF3FC021E048E0F4
:108FA00061E083E00E9416168091791D8F93809175
:108FB000781D8F938091771D8F938091761D8F936D
:108FC0008091751D8F938091741D8F938091731D77
:108FD0008F938091721D8F938FEF93E09F938F9368
:108FE0000E940CA30E94E60D8091711D8F938091C9
:108FF000701D8F9380916F1D8F9380916E1D8F9345
:1090000081EF93E09F938F930E940CA30E94E60D43
:109010000FB6F894DEBF0FBECDBF8091922C85FFB6
:1090200058C081E00E94FB78609166357091673589
:1090300080916835909169350E94139920E030E065
:1090400048EC52E40E945F989F938F937F936F93B5
:109050008AED96E09F938F930E94F8A260916A3503
:1090600070916B3580916C3590916D350E9411999E
:1090700020E030E040E85AE30E940B9B9F938F93DF
:109080007F936F9389EE96E09F938F930E94F8A24F
:1090900060916E3570916F3580917035909171351A
:1090A0000E94119920E030E040E85BE30E940B9BB6
:1090B0009F938F937F936F938AEF96E09F938F9305
:1090C0000E94F8A20E94E60D0FB6F894DEBF0FBE14
:1090D000CDBF8091922C9091932C94FF3BC00E9425
:1090E0008C1A20E030E048EC52E4162F072FF82EBF
:1090F000E92E0E940B9B20E836EE45EC57E40E94D7
:109100005F9821E03EED42E45EE30E94789B9B0184
:10911000AC0160E070E080E89FE30E947B972BE465
:109120003AE34DEB57E30E945F989F938F937F93B1
:109130006F93EF92FF920F931F9388ED93E09F93AD
:109140008F930E940CA30E94E60D0FB6F894DEBF29
:109150000FBECDBF80917D02882309F41FC11F92ED
:109160008F9385ED93E09F938F930E940CA30F90B4
:109170000F900F900F9012C160917B0270917C0252
:1091800080E090E00E9439A26AE077E00E944DA260
:10919000892BB1F460917B0270917C0280E090E0B9
:1091A0000E9439A2009709F4F9C00E9426A18031DB
:1091B00008F0F4C090915201892B80935201EEC0C7
:1091C000809152018F701F928F9389E192E09F935B
:1091D0008F930E940CA30E94E60D0F900F900F90AA
:1091E0000F90DCC060917B0270917C0280E090E087
:1091F0000E9439A2009711F14AE050E060E070E06F
:109200000E94BF9E603198F4609360021F926F933A
:1092100088EC93E09F938F930E940CA341E050E071
:109220006BE170E080E692E00E9410A611C0809190
:1092300060021F928F938FEB93E006C080916002D3
:109240001F928F9386EB93E09F938F930E940CA3C2
:109250000F900F900F900F900E94E60D80917D026D
:10926000882309F49BC01F928F9383EB93E09F9315
:109270008F930E940CA30F900F900F900F908EC0B1
:1092800060917B0270917C0280E090E00E9439A2A4
:109290008C016BEC75E00E944DA2892BE1F40E94D9
:1092A0000A718091620290916302A0916402B09170
:1092B000650290618093620290936302A0936402BE
:1092C000B093650244E050E06EE170E082E692E027
:1092D0000E9410A663C06EEC75E0C8010E944DA20A
:1092E000892B99F5F8940E9417710FB6F894A895F8
:1092F00080916000886180936000109260000FBED2
:1093000084B7877F84BF809160008861809360000C
:109310001092600078948091620290916302A09113
:109320006402B09165029F7E809362029093630213
:10933000A0936402B093650244E050E06EE170E0F7
:1093400082E692E00E9410A629C06FE077E0C80193
:109350000E944DA2409162025091630260916402AA
:1093600070916502892B21F454FF18C0F894FFCF47
:1093700054FD03C08EEC95E002C08BEC95E09F930A
:109380008F9385E192E09F938F930E940CA30F909F
:109390000F900F900F9002C00E945C22EA85FB851F
:1093A0001182108283E02B960FB6F894DEBF0FBEB9
:1093B000CDBFDF91CF911F910F91FF90EF90DF9084
:1093C000CF90BF90AF909F908F907F906F905F9065
:1093D0004F903F902F900895CF93DF93EC018881B9
:1093E0009981009741F08736924109F490C0198223
:1093F000188283E097C00E94B5338091620280FD9D
:1094000005C081FF01C01D9B0E94587280917000B1
:109410008C7F809370008091B60080628093B6004C
:109420001092B20082E08093B1008091B600877004
:10943000E1F7809170008160809370006DE77AE0C1
:1094400080E090E00E94E4700E94782380E00E9417
:10945000582589E091E19F938F930E940CA30E946D
:10946000D6128091922C9091932C0F900F9091FD99
:109470000E94586B8091922C9091932C93FD0E94A6
:109480004B208091922C9091932C92FF06C021E06A
:109490004CE061E080ED0E94FB6B8091DF0A0E944E
:1094A000FD74809161020E94A5730E94A273809353
:1094B000140B809161020E94A5738091DF0A1F92B4
:1094C0008F938091140B1F928F9384E197E09F9369
:1094D0008F930E94F8A21092160B1092150B0F900A
:1094E0000F900F900F900F900F9082E592E0909365
:1094F00065358093643583E290E0909327138093E1
:10950000261387E692E19983888381E00BC063325A
:10951000E1F741EC50E360E070E085E19BE00E9400
:109520002035E3CFDF91CF9108950F931F93CF9311
:10953000DF93EC018A0188819981009711F18C37C2
:10954000924121F01982188283E020C06231E9F44F
:10955000A80162E170E085E19BE00E94203584E093
:109560008093493510924B3510924A3510934D3502
:1095700000934C3549E455E362E18EE392E00E94AA
:10958000DE5E8CE792E19983888381E0DF91CF9161
:109590001F910F910895AF92BF92CF92DF92EF92F9
:1095A000FF920F931F93CF93DF93EC018091E30A17
:1095B0009091E40AA091E50AB091E60A81FD08C005
:1095C0009091620290FD04C091FF57C01D9B55C051
:1095D0005A018B01FB01C384D484E584F684A4E69C
:1095E000B0E0A70196010E948D9C672F782F892FEC
:1095F000992724E630E040E050E00E941E9C7F93D3
:109600006F93CD2CDE2CEF2CFF24DF92CF92F8014C
:1096100086811F928F9385811F928F9388818F708F
:109620001F928F9389811F928F93F50181811F92E1
:109630008F9380811F928F932296DF93CF9386E240
:1096400097E09F938F930E94F8A280917D02EDB7DF
:10965000FEB774960FB6F894FEBF0FBEEDBF882319
:1096600061F01F928F9380EE91E09F938F930E9401
:109670000CA30F900F900F900F90DF91CF911F913F
:109680000F91FF90EF90DF90CF90BF90AF90089533
:109690008436910514F19F938F938AE697E09F9308
:1096A0008F930E94F8A280919C3090919D30A09160
:1096B0009E30B0919F300196A11DB11D80939C30CA
:1096C00090939D30A0939E30B0939F300F900F9059
:1096D0000F900F9081E090E0089580E090E0089571
:1096E0002F923F924F925F926F927F928F929F92B2
:1096F000AF92BF92CF92DF92EF92FF920F931F93A0
:10970000CF93DF93CDB7DEB7CC59D1090FB6F8941C
:10971000DEBF0FBECDBFCB56DF4F99838883C559BF
:10972000D0408A01633871F489E19BE0C456DF4F71
:109730006883CC59D0400E941D5DC456DF4F6881BC
:10974000CC59D040CB56DF4FA881B981C559D04004
:109750002D913C912431B2E13B0709F483C440F4DC
:109760002115310581F02531304109F4C5C4B9C452
:10977000263242E1340709F495C42D32324111F406
:109780000C94445AAEC444EF52E061E870E089E1C1
:109790009BE00E94025D85E190E15BC45A01E3E039
:1097A000F0E0EC0FFD1FE40FF51F1082CA010E94CC
:1097B000484B892B81F720E030E040E050E0CC5668
:1097C000DF4F6881C459D040627070E080E090E063
:1097D000A0E00E94599E09F039C7CE56DF4F28817C
:1097E000C259D040287030E040E050E060E070E0C6
:1097F00080E090E0A0E00E94599E99F127E04AE2C3
:1098000050E06BE270E089E290E00E943B678BE5FC
:1098100095E30E94AA69BC01990F880B990B0E94DD
:10982000139920E030E048EC52E40E945F989F9347
:109830008F937F936F938EE997E09F938F931F92FF
:1098400087E78F93CE018A0D9B1D03969F938F937D
:109850000E9464A3A80EB91E0FB6F894DEBF0FBE17
:10986000CDBFCE56DF4F2881C259D040207130E0A5
:1098700040E050E060E070E080E090E0A0E00E9416
:10988000599EE9F126E04AE250E06BE270E089E29D
:1098900090E00E943B6781E090E00E947E0D809303
:1098A000DE0A8EEC9CE10E94AA69BC01990F880B2C
:1098B000990B0E94139920E030E048EC52E40E949A
:1098C0005F989F938F937F936F9388EA97E09F931E
:1098D0008F931F9287E78F93C501029621E030E0B6
:1098E0002C0F3D1F820F931F9F938F930E9464A3A1
:1098F000A80EB91E0FB6F894DEBF0FBECDBFC2577B
:10990000DF4F2881CE58D04030E040E050E060E0AA
:1099100070E080E090E0A0E00E94599E01F10E947A
:109920003A0D9F938F937F936F9383EB97E09F9371
:109930008F931F9287E78F93C5010296A1E0B0E055
:10994000AC0FBD1F8A0F9B1F9F938F930E9464A330
:10995000A80EB91E0FB6F894DEBF0FBECDBFCE560F
:10996000DF4F2881C259D040207430E040E050E001
:1099700060E070E080E090E0A0E00E94599E31F14C
:10998000809197308F93809196308F93809195300E
:109990008F93809194308F9381EC97E09F938F9376
:1099A0001F9287E78F93C501029621E030E02C0FCC
:1099B0003D1F820F931F9F938F930E9464A3A80E55
:1099C000B91E0FB6F894DEBF0FBECDBFCE56DF4F27
:1099D0002881C259D040207830E040E050E060E07B
:1099E00070E080E090E0A0E00E94599E41F1F89480
:1099F0008091413590914235A0914335B0914435E5
:109A00007894BF93AF939F938F938FEC97E09F933E
:109A10008F931F9287E78F93C5010296A1E0B0E074
:109A2000AC0FBD1F8A0F9B1F9F938F930E9464A34F
:109A3000A80EB91E0FB6F894DEBF0FBECDBF20E052
:109A4000312F317040E050E060E070E080E090E065
:109A5000A0E00E94599E09F00BC620E0312F327021
:109A600040E050E060E070E080E090E0A0E00E9424
:109A7000599E09F07BC620E0312F347040E050E061
:109A800060E070E080E090E0A0E00E94599E09F064
:109A90009EC620E0312F387040E050E060E070E07A
:109AA00080E090E0A0E00E94599E09F0C0C620E04E
:109AB000312F307140E050E060E070E080E090E0F5
:109AC000A0E00E94599E09F030C720E0312F30728B
:109AD00040E050E060E070E080E090E0A0E00E94B4
:109AE000599E09F052C720E030E040E050E0CC56EB
:109AF000DF4F6881C459D040647070E080E090E02E
:109B0000A0E00E94599E09F06EC720E0C856DF4FC2
:109B10003881C859D04040E050E060E070E080E01B
:109B200090E0A0E00E94599E09F0CAC720E0C75605
:109B3000DF4F3881C959D04040E050E060E070E02C
:109B400080E090E0A0E00E94599E09F0E8C7502F05
:109B50005170952E20E030E0452F50E060E070E03D
:109B600080E090E0A0E00E94599E11F00C94BE5558
:109B700020E030E0402F427050E060E070E080E094
:109B800090E0A0E00E94599E11F00C94F25520E064
:109B900030E0C657DF4F4881CA58D04050E060E0FF
:109BA00070E080E090E0A0E00E94599E11F00C94DB
:109BB000265620E030E040E050E0CC56DF4F688190
:109BC000C459D040687070E080E090E0A0E00E944E
:109BD000599E11F00C94515620E030E040E050E0E6
:109BE000CC56DF4F6881C459D040607170E080E08E
:109BF00090E0A0E00E94599E11F00C947D5620E068
:109C000030E0402F487050E060E070E080E090E08D
:109C1000A0E00E94599E11F00C94A95620E030E07B
:109C2000402F407150E060E070E080E090E0A0E004
:109C30000E94599E11F00C94DE5620E030E0402F37
:109C4000407250E060E070E080E090E0A0E00E94B0
:109C5000599E11F00C94135720E030E0402F4074CF
:109C600050E060E070E080E090E0A0E00E94599E4B
:109C700011F00C944857F02FF0787F2E20E030E060
:109C80004F2F50E060E070E080E090E0A0E00E94A4
:109C9000599E11F00C947D57CD56DF4F2881C35942
:109CA000D0402170622E20E030E040E0562D60E090
:109CB00070E080E090E0A0E00E94599E11F40C94C6
:109CC000575A8091922C82FD02C00C94C55721E016
:109CD00046E061E083E00E94161620E030E0472D68
:109CE00050E060E070E080E090E0A0E00E94599ECB
:109CF00011F40C94C5578091922C82FF02C00C94F1
:109D00008A5720E030E040E0CD56DF4F5881C359FC
:109D1000D040527060E070E080E090E0A0E00E94EF
:109D2000599E11F00C94FA5720E030E040E0CD56F7
:109D3000DF4F5881C359D040547060E070E080E03C
:109D400090E0A0E00E94599E11F00C942D5820E064
:109D500030E040E0CD56DF4F5881C359D0405071BC
:109D600060E070E080E090E0A0E00E94599E11F079
:109D70000C94605820E030E040E0CD56DF4F588131
:109D8000C359D040507260E070E080E090E0A0E005
:109D90000E94599E11F00C949F5820E030E040E062
:109DA000CD56DF4F5881C359D040507460E070E009
:109DB00080E090E0A0E00E94599E11F00C94DE58E3
:109DC00020E030E040E0CD56DF4F5881C359D0400D
:109DD000587060E070E080E090E0A0E00E94599E42
:109DE00011F00C941D5920E030E040E050E0CC56DA
:109DF000DF4F6881C459D040607270E080E090E02D
:109E0000A0E00E94599E11F40C944E598091922C1E
:109E100085FD02C00C944E5981E00E94FB78609150
:109E200066357091673580916835909169350E94EB
:109E3000139920E030E048EC52E40E945F989F9331
:109E40008F937F936F9388E599E09F938F931F92F1
:109E500087E78F93C501029641E050E04C0F5D1FEC
:109E6000840F951F9F938F930E9464A3A80EB91E21
:109E7000C5010E94484B0FB6F894DEBF0FBECDBFA0
:109E8000892B09F088CCE1E020E030E040E050E0B0
:109E9000CC56DF4F6881C459D040607470E080E0D8
:109EA00090E0A0E00E94599E11F00C94515920E0DE
:109EB00030E040E050E0CC56DF4F6881C459D040DC
:109EC000607870E080E090E0A0E00E94599E11F080
:109ED0000C94945920E030E040E0C656DF4F5881A2
:109EE000CA59D04060E070E080E090E0A0E00E94BD
:109EF000599E11F00C94D65920E030E0492D50E0E5
:109F000060E070E080E090E0A0E00E94599E11F0D7
:109F10000C94065ACE56DF4F2881C259D040312FBB
:109F2000402FCD56DF4F5881C359D040CC56DF4F1C
:109F30006881C459D040722D832DC956DF4F988156
:109F4000C759D040A0E00E94599E11F00C94115ABC
:109F5000809160028061898380910D0B8A83FE016C
:109F6000EA0DFB1D13828091E30A9091E40AA0910F
:109F7000E50AB091E60A85010D5F1F4F80FF0CC016
:109F80001F930F9383EA99E09F938F930E94F8A207
:109F90000F900F900F900F90B801CE0101960E9484
:109FA00032668091620282FF0AC021E431E3A80197
:109FB000BE016F5F7F4F8BE692E00E94BE6A809188
:109FC000E30A9091E40AA091E50AB091E60A82FDC5
:109FD00073980E94A07289E19BE00E941F5D8091AE
:109FE000620290916302A0916402B091650290FFB9
:109FF00040C05FEFA51AB50A0E94A273F82E89E14E
:10A000000E94BA738091620290916302A0916402EF
:10A01000B091650290FF29C0739880910D0B8F5FFE
:10A0200080930D0B8A83B5016F5F7F4FCE01019640
:10A030000E94326689E19BE00E941F5D40E050E093
:10A0400065E880912A1390912B130E94DE5E84E1D3
:10A0500092E1CB56DF4FA881B981C559D0408D938D
:10A060009C933CC0A12CB12CCDCF8F2D0E94BA73F4
:10A07000739A8091E00A9091E10A892B11F00E9475
:10A08000587280910D0B8F5F80930D0B8091E30AC6
:10A090009091E40AA091E50AB091E60A82FF7BCB99
:10A0A000739A79CB85E09BE00E948A61892BB1F09D
:10A0B0000E94A0728091620287FD2B9860E470E09C
:10A0C00085E09BE00E9463618DE292E1CB56DF4F19
:10A0D000E881F981C559D0409183808381E00C9457
:10A0E000675ACB56DF4FA881B981C559D0401D9220
:10A0F0001C9283E00C94675A623181F7809062026F
:10A1000090906302A0906402B090650291FC43CBF2
:10A11000F8018081813021F50180F281E02D2081DC
:10A12000CE56DF4F2883C259D0401181028133813E
:10A13000CD56DF4F3883C359D0404481CC56DF4FD2
:10A140004883C459D040258036805781C956DF4F97
:10A150005883C759D040C084D184E12CF12C55C01C
:10A160008230C1F4E380F480C12CD12CB1E0CE5612
:10A17000DF4FB883C259D04010E000E0E0E8CD5690
:10A18000DF4FE883C359D040CC56DF4F1882C45903
:10A19000D04034C08330D9F0843009F0FCCAC12CDF
:10A1A000D12CE12CF12CF5E0CE56DF4FF883C259CB
:10A1B000D04010E000E0CD56DF4F1882C359D040A8
:10A1C00022E0CC56DF4F2883C459D04017C0C12CA1
:10A1D000D12CE12CF12C35E0CE56DF4F3883C2591B
:10A1E000D04010E000E0CD56DF4F1882C359D04078
:10A1F00041E0CC56DF4F4883C459D040212C312C4C
:10A20000C956DF4F1882C759D040409094305090C3
:10A210009530609096307090973080918A0290913E
:10A220008B02A0918C02B0918D02C657DF4F8883BC
:10A230009983AA83BB83CA58D0402DEC3CEC4CE4F4
:10A240005EE3BC01CD010E947C979B01AC01C30180
:10A25000B2010E94389A87FD0BC0E894A0F8809262
:10A26000620290926302A0926402B092650247C0BB
:10A27000C657DF4F288139814A815B81CA58D04057
:10A28000C301B2010E945A9887FF39C08091A03063
:10A290009091A130A091A230B091A3300196A11D60
:10A2A000B11D8093A0309093A130A093A230B093C1
:10A2B000A330A0FC70CA6894A0F8809262029092C9
:10A2C0006302A0926402B092650295E4CE56DF4F1D
:10A2D0009883C259D04010E200E0CD56DF4F18827B
:10A2E000C359D040A4E0CC56DF4FA883C459D04016
:10A2F000212C312CC956DF4F1882C759D040B02FBE
:10A30000B470C657DF4FB883CA58D04020E030E061
:10A310004B2F50E060E070E080E090E0A0E00E9411
:10A32000599E09F08C9ACE56DF4FE881C259D04031
:10A33000E072C257DF4FE883CE58D0402E2F30E076
:10A3400040E050E060E070E080E090E0A0E00E943B
:10A35000599E11F00E943A0DF12FF074C856DF4F4C
:10A36000F883C859D04020E03F2F40E050E060E043
:10A3700070E080E090E0A0E00E94599E11F00E9401
:10A38000BE21212F2078C756DF4F2883C959D040DE
:10A3900020E0C756DF4F3881C959D04040E050E037
:10A3A00060E070E080E090E0A0E00E94599E51F0F3
:10A3B0000E94D50C60934E3570934F358093503585
:10A3C00090935135CE56DF4F2881C259D04021702D
:10A3D00030E040E050E060E070E080E090E0A0E03D
:10A3E0000E94599EF1F08CE59CE19F938F938EE73C
:10A3F00097E09F938F931F9287E78F93CE010396E9
:10A400009F938F930E9464A34C010E94484B0FB608
:10A41000F894DEBF0FBECDBF892B09F0BCC9540133
:10A4200002C0A12CB12CCE56DF4F2881C259D0409A
:10A43000227030E040E050E060E070E080E090E0CA
:10A44000A0E00E94599ED1F1C501029666E877E02E
:10A45000A1E0B0E0AC0FBD1F8A0F9B1F0E9456A267
:10A46000B3E0AB0EB11C2BE5622E25E3722E3CE06F
:10A47000832E34E0932E47E7542EF30181913F0160
:10A480001F928F939F928F921F925F92C5010296A7
:10A4900021E030E02C0F3D1F820F931F9F938F937D
:10A4A0000E9464A3A80EB91E0FB6F894DEBF0FBEBB
:10A4B000CDBF53E6651655E37506F9F6CE56DF4F68
:10A4C0002881C259D040247030E040E050E060E084
:10A4D00070E080E090E0A0E00E94599E09F450C036
:10A4E000C50102966AE877E0A1E0B0E0AC0FBD1FBD
:10A4F0008A0F9B1F0E9456A2B4E0AB0EB11C2E0126
:10A50000EAE74E0E511C80E1D2011D928A95E9F7CF
:10A5100028E0A20168E980EB0E948B123201B8E0CA
:10A520006B0E711C9CE0892E94E0992E27E7F201B6
:10A5300081912F011F928F939F928F921F922F9341
:10A54000C501029641E050E04C0F5D1F840F951F3E
:10A550009F938F93C556DF4F2883CB59D0400E94DD
:10A5600064A3A80EB91E0FB6F894DEBF0FBECDBF10
:10A57000C556DF4F2881CB59D04046145704B9F651
:10A58000CD56DF4F9881C359D0409078C656DF4FE3
:10A590009883CA59D04020E030E040E0592F60E075
:10A5A00070E080E090E0A0E00E94599EE1F480918C
:10A5B000E00A9091E10A9F938F938FE897E09F9331
:10A5C0008F931F9287E78F93CE018A0D9B1D039671
:10A5D0009F938F930E9464A3A80EB91E0FB6F894A0
:10A5E000DEBF0FBECDBF20E030E040E050E0CC56F3
:10A5F000DF4F6881C459D040617070E080E090E026
:10A60000A0E00E94599E09F4D6C8E3E0F0E0EC0F08
:10A61000FD1FEA0DFB1D80E28083A50183E090E031
:10A620008A199B09FC01E40FF51FEF53FF4C2081B1
:10A630004F5F5F4F222309F4B1C82081E1E0F0E0D1
:10A64000EC0FFD1FE40FF51F2283ECCFCE018A0D26
:10A650009B1D66E977E003960E9456A2B7E0AB0E19
:10A66000B11CC5010E94484B892B09F094C8B5C89C
:10A67000C114D10409F4F1C9F894409041355090C7
:10A680004235609043357090443578948091C61C73
:10A690009091C71CA091C81CB091C91CA301920144
:10A6A000281B390B4A0B5B0BCA01B9010E94119997
:10A6B000C257DF4F688379838A839B83CE58D0400B
:10A6C000B60180E090E00E9411999B01AC01C25755
:10A6D000DF4F688179818A819B81CE58D0400E946A
:10A6E0005F984C019F928F937F936F938AED97E0D1
:10A6F0009F938F931F9287E78F939E012A0D3B1D97
:10A700002D5F3F4F3F932F93C456DF4F6883CC5943
:10A71000D040C556DF4F7883CB59D0400E9464A308
:10A72000A80EB91EC456DF4F6881CC59D040C5561B
:10A73000DF4F7881CB59D040862F972FA82DB92D88
:10A740008093533590935435A0935535B093563537
:10A750004092C61C5092C71C6092C81C7092C91CC3
:10A760000FB6F894DEBF0FBECDBF77C9C114D104B8
:10A7700009F481C9F89480919D1C90919E1CA09130
:10A780009F1CB091A01C78949F938F938091690235
:10A790008F93809168028F9387EE97E09F938F93BA
:10A7A0001F9287E78F93C5010296A1E0B0E0AC0F3E
:10A7B000BD1F8A0F9B1F9F938F930E9464A3A80EB7
:10A7C000B91E0FB6F894DEBF0FBECDBF54C9F894C2
:10A7D0008091453590914635A0914735B0914835E7
:10A7E0007894BF93AF939F938F9387EF97E09F9356
:10A7F0008F931F9287E78F93C501029621E030E087
:10A800002C0F3D1F820F931F9F938F930E9464A371
:10A81000A80EB91EC5010E94484B0FB6F894DEBFC2
:10A820000FBECDBF892B11F00C94CB4B32C9C11494
:10A83000D10409F43CC9F894409045355090463510
:10A84000609047357090483578948091CA1C9091FB
:10A85000CB1CA091CC1CB091CD1CA3019201281B54
:10A86000390B4A0B5B0BCA01B9010E941199C257FF
:10A87000DF4F688379838A839B83CE58D040B601AB
:10A8800080E090E00E9411999B01AC01C257DF4F1C
:10A89000688179818A819B81CE58D0400E945F98DF
:10A8A0004C019F928F937F936F9382E098E09F93E8
:10A8B0008F931F9287E78F939E012A0D3B1D2D5F7B
:10A8C0003F4F3F932F93C456DF4F6883CC59D040FE
:10A8D000C556DF4F7883CB59D0400E9464A3A80EA1
:10A8E000B91EC456DF4F6881CC59D040C556DF4FE2
:10A8F0007881CB59D040862F972FA82DB92D8093E2
:10A90000573590935835A0935935B0935A354092A6
:10A91000CA1C5092CB1C6092CC1C7092CD1C0FB6FE
:10A92000F894DEBF0FBECDBFC2C8CD2809F4CDC894
:10A93000F8948091A11C9091A21CA091A31CB091AD
:10A94000A41C78949F938F93809167028F9380913A
:10A9500066028F938FE098E09F938F931F9287E713
:10A960008F93C5010296A1E0B0E0AC0FBD1F8A0F26
:10A970009B1F9F938F930E9464A3A80EB91E0FB6CE
:10A98000F894DEBF0FBECDBFA0C8809198309091E3
:10A990009930A0919A30B0919B30BF93AF939F9321
:10A9A0008F938FE198E09F938F931F9287E78F9308
:10A9B000C501029621E030E02C0F3D1F820F931F4E
:10A9C0009F938F930E9464A3A80EB91EC5010E9495
:10A9D000484B0FB6F894DEBF0FBECDBF892B11F0E8
:10A9E0000C94CB4B80C88091A3308F938091A23080
:10A9F0008F938091A1308F938091A0308F9380911D
:10AA00009F308F9380919E308F9380919D308F9354
:10AA100080919C308F938AE298E09F938F931F924E
:10AA200087E7982E9F92C5010296A1E0B0E0AC0F97
:10AA3000BD1F8A0F9B1F9F938F930E9464A3A80E34
:10AA4000B91EC5010E94484B0FB6F894DEBF0FBE79
:10AA5000CDBF892B11F00C94CB4B8091922C90910F
:10AA6000932C93FF52C88091A7308F938091A6308A
:10AA70008F938091A5308F938091A4308F938EE433
:10AA800098E09F938F931F929F92C501029621E0B9
:10AA900030E02C0F3D1F820F931F9F938F930E94D6
:10AAA00064A3A80EB91EC5010E94484B0FB6F894C6
:10AAB000DEBF0FBECDBF892B11F00C94CB4B25C848
:10AAC000809189288F93809188288F9380918728FF
:10AAD0008F93809186288F9380E698E09F938F9341
:10AAE0001F9287E78F93C5010296A1E0B0E0AC0FFB
:10AAF000BD1F8A0F9B1F9F938F930E9464A3A80E74
:10AB0000B91EC5010E94484B0FB6F894DEBF0FBEB8
:10AB1000CDBF892B11F00C94CB4B0C94964D8091AA
:10AB200051358F93809150358F9380914F358F930E
:10AB300080914E358F938BE698E09F938F931F9271
:10AB400087E78F93C501029621E030E02C0F3D1F6F
:10AB5000820F931F9F938F930E9464A3A80EB91E28
:10AB6000C5010E94484B0FB6F894DEBF0FBECDBFA3
:10AB7000892B11F00C94CB4B0C94A74D81E00E94D3
:10AB8000870C20918202309183024091840250917F
:10AB900085020E940B9B9F938F937F936F9388E70F
:10ABA00098E09F938F931F9287E78F93C50102963A
:10ABB000A1E0B0E0AC0FBD1F8A0F9B1F9F938F9346
:10ABC0000E9464A3A80EB91EC5010E94484B0FB68F
:10ABD000F894DEBF0FBECDBF892B11F00C94CB4B88
:10ABE0000C94B84D82E00E94870C20917E02309137
:10ABF0007F0240918002509181020E940B9B9F93A3
:10AC00008F937F936F9385E898E09F938F931F9224
:10AC100087E78F93C501029621E030E02C0F3D1F9E
:10AC2000820F931F9F938F930E9464A3A80EB91E57
:10AC3000C5010E94484B0FB6F894DEBF0FBECDBFD2
:10AC4000892B11F00C94CB4B0C94C74D83E00E94E0
:10AC5000870C9F938F937F936F9382E998E09F93E4
:10AC60008F931F9287E78F93C5010296A1E0B0E012
:10AC7000AC0FBD1F8A0F9B1F9F938F930E9464A3ED
:10AC8000A80EB91E8C98C5010E94484B0FB6F894C7
:10AC9000DEBF0FBECDBF892B11F00C94CB4B0C94B3
:10ACA000D94D299903C08EEC95E002C08BEC95E05C
:10ACB0009F938F938FE998E09F938F931F9287E7DD
:10ACC0008F93C501029621E030E02C0F3D1F820FCB
:10ACD000931F9F938F930E9464A3A80EB91EC50172
:10ACE0000E94484B0FB6F894DEBF0FBECDBF892B34
:10ACF00011F00C94CB4B0C94EC4D2A9903C08EECC4
:10AD000095E002C08BEC95E09F938F9387EA98E0E3
:10AD10009F938F931F9287E78F93C5010296A1E0BF
:10AD2000B0E0AC0FBD1F8A0F9B1F9F938F930E94B3
:10AD300064A3A80EB91EC5010E94484B0FB6F89433
:10AD4000DEBF0FBECDBF892B11F00C94CB4B0C9402
:10AD5000FF4D8091922C9091932C92FD02C00C9407
:10AD60000E4E21E042E161E080ED0E94FB6B9F937B
:10AD70008F937F936F938FEA98E09F938F931F92A7
:10AD800087E78F93C501029621E030E02C0F3D1F2D
:10AD9000820F931F9F938F930E9464A3A80EB91EE6
:10ADA000C5010E94484B0FB6F894DEBF0FBECDBF61
:10ADB000892B11F00C94CB4B0C940E4E8091922C5D
:10ADC0009091932C92FD02C00C941D4E21E042E123
:10ADD00062E080ED0E94FB6B9F938F937F936F9354
:10ADE0008DEB98E09F938F931F9287E78F93C50118
:10ADF0000296A1E0B0E0AC0FBD1F8A0F9B1F9F938E
:10AE00008F930E9464A3A80EB91EC5010E94484BEF
:10AE10000FB6F894DEBF0FBECDBF892B11F00C9496
:10AE2000CB4B0C941D4E8091922C9091932C92FDC3
:10AE300002C00C942C4E21E042E163E080ED0E94C0
:10AE4000FB6B9F938F937F936F938BEC98E09F9313
:10AE50008F931F9287E78F93C501029621E030E020
:10AE60002C0F3D1F820F931F9F938F930E9464A30B
:10AE7000A80EB91EC5010E94484B0FB6F894DEBF5C
:10AE80000FBECDBF892B11F00C94CB4B0C942C4EE4
:10AE90008091922C9091932C92FD02C00C943B4E89
:10AEA00021E042E164E080ED0E94FB6B9F938F9371
:10AEB0007F936F9389ED98E09F938F931F9287E71D
:10AEC0008F93C5010296A1E0B0E0AC0FBD1F8A0FC1
:10AED0009B1F9F938F930E9464A3A80EB91EC50168
:10AEE0000E94484B0FB6F894DEBF0FBECDBF892B32
:10AEF00011F00C94CB4B0C943B4E8091922C82FD24
:10AF000002C00C944C4E46E061E083E00E941616AD
:10AF10000C944C4E8091751D8F938091741D8F936E
:10AF20008091731D8F938091721D8F9387EE98E0AF
:10AF30009F938F931F9287E78F93C501029641E0FD
:10AF400050E04C0F5D1F840F951F9F938F930E94BD
:10AF500064A3A80EB91EC5010E94484B0FB6F89411
:10AF6000DEBF0FBECDBF892B11F00C94CB4B20E080
:10AF700030E040E0562D60E070E080E090E0A0E03E
:10AF80000E94599E11F40C94814E8091922C82FD66
:10AF900002C00C94814E8091791D8F938091781D11
:10AFA0008F938091771D8F938091761D8F938FEE75
:10AFB00098E09F938F931F9287E78F93C501029626
:10AFC000E1E0F0E0EC0FFD1F8E0F9F1F9F938F932A
:10AFD0000E9464A3A80EB91EC5010E94484B0FB67B
:10AFE000F894DEBF0FBECDBF892B11F00C94CB4B74
:10AFF0000C94814E8091922C9091932C93FD02C0E1
:10B000000C94944E80E090E00E9435219F938F93A2
:10B010007F936F938AEF98E09F938F931F9287E7B8
:10B020008F93C501029641E050E04C0F5D1F840FE5
:10B03000951F9F938F930E9464A3A80EB91EC5010C
:10B040000E94484B0FB6F894DEBF0FBECDBF892BD0
:10B0500011F00C94CB4B0C94944E8091922C9091C7
:10B06000932C93FD02C00C94A74E81E090E00E94C7
:10B0700035219F938F937F936F938AE099E09F93FD
:10B080008F931F9287E78F93C5010296E1E0F0E06E
:10B09000EC0FFD1F8E0F9F1F9F938F930E9464A341
:10B0A000A80EB91EC5010E94484B0FB6F894DEBF2A
:10B0B0000FBECDBF892B11F00C94CB4B0C94A74E37
:10B0C0008091922C9091932C93FD02C00C94BA4ED7
:10B0D00081E090E00E9435212B013C0180E090E06E
:10B0E0000E9435219B01AC01C301B2010E94321FB5
:10B0F0009F938F937F936F938BE199E09F938F93AF
:10B100001F9287E78F93C501029641E050E04C0FF4
:10B110005D1F840F951F9F938F930E9464A3A80EB9
:10B12000B91EC5010E94484B0FB6F894DEBF0FBE92
:10B13000CDBF892B11F00C94CB4B0C94BA4E80915F
:10B14000922C9091932C93FD02C00C94CD4E81E0F3
:10B1500090E00E9435212B013C0180E090E00E94AC
:10B1600035219B01AC01C301B2010E94931F9F9343
:10B170008F937F936F9386E299E09F938F931F92B3
:10B1800087E78F93C5010296E1E0F0E0EC0FFD1F29
:10B190008E0F9F1F9F938F930E9464A3A80EB91ECA
:10B1A000C5010E94484B0FB6F894DEBF0FBECDBF5D
:10B1B000892B11F00C94CB4B0C94CD4E8091922C9A
:10B1C0009091932C93FD02C00C94E04E81E090E0AE
:10B1D0000E9435212B013C0180E090E00E94352146
:10B1E0009B01AC01C301B2010E94F41F9F938F9396
:10B1F0007F936F9384E399E09F938F931F9287E7E8
:10B200008F93C501029641E050E04C0F5D1F840F03
:10B21000951F9F938F930E9464A3A80EB91EC5012A
:10B220000E94484B0FB6F894DEBF0FBECDBF892BEE
:10B2300011F00C94CB4B0C94E04E8091922C909199
:10B24000932C94FD02C00C94F34E0E948C1A9F9391
:10B250008F937F936F9387E499E09F938F931F92CF
:10B2600087E78F93C5010296E1E0F0E0EC0FFD1F48
:10B270008E0F9F1F9F938F930E9464A3A80EB91EE9
:10B28000C5010E94484B0FB6F894DEBF0FBECDBF7C
:10B29000892B11F00C94CB4B0C94F34EE0E00C9402
:10B2A000444F8091922C85FD02C00C94574FE111C0
:10B2B00003C081E00E94FB7860916A3570916B3524
:10B2C00080916C3590916D350E94119920E030E0AD
:10B2D00040E85AE30E940B9B9F938F937F936F9359
:10B2E00089E699E09F938F931F9287E78F93C5011B
:10B2F0000296E1E0F0E0EC0FFD1F8E0F9F1F9F9381
:10B300008F930E9464A3A80EB91EC5010E94484BEA
:10B310000FB6F894DEBF0FBECDBF892B11F00C9491
:10B32000CB4BE1E00C94574F8091922C85FD02C0ED
:10B330000C946A4FE11103C081E00E94FB78609198
:10B340006E3570916F3580917035909171350E9496
:10B35000119920E030E040E85BE30E940B9B9F9353
:10B360008F937F936F938BE799E09F938F931F92B7
:10B3700087E78F93C501029641E050E04C0F5D1FB7
:10B38000840F951F9F938F930E9464A3A80EB91EEC
:10B39000C5010E94484B0FB6F894DEBF0FBECDBF6B
:10B3A000892B11F00C94CB4B0C946A4FF7018681DA
:10B3B0001F928F9385811F928F9383811F928F930A
:10B3C00082811F928F938CE899E09F938F931F92B5
:10B3D00087E78F93C501029621E030E02C0F3D1FD7
:10B3E000820F931F9F938F930E9464A3A80EB91E90
:10B3F000C5010E94484B0FB6F894DEBF0FBECDBF0B
:10B40000892B11F00C94CB4B0C947C4F779A809144
:10B41000E30A9091E40AA091E50AB091E60A92FD50
:10B42000749A8091E30A9091E40AA091E50AB091A0
:10B43000E60A82FD0CC08091620280FD08C081FD99
:10B4400002C00C94A84F1D9902C00C94A84F40E074
:10B4500050E060E070E0CE0101960E94E80A809121
:10B460007B1D90E02091DA0A3091DB0A8217930766
:10B4700010F40C94A84F40E050E062E18CE092E0C0
:10B480000E94DE5E0C94A84F85E09BE00E948A61DA
:10B49000892B11F40C946E500E94587280916202B4
:10B4A00087FD02C00C94CB4B2B9A0C94CB4B20E025
:10B4B00030E0472D50E060E070E080E090E0A0E0F8
:10B4C0000E94599E11F00C947B4E0C94814EC456F0
:10B4D000DF4F0FB6F894DEBF0FBECDBFDF91CF9127
:10B4E0001F910F91FF90EF90DF90CF90BF90AF90A2
:10B4F0009F908F907F906F905F904F903F902F9094
:10B5000008950C94475D4F925F926F927F92AF9235
:10B51000BF92CF92DF92EF92FF920F931F93CF9340
:10B52000DF93CDB7DEB760970FB6F894DEBF0FBEDE
:10B53000CDBF6B010E94A273E82FF0E0EE0FFF1F5A
:10B54000E157F34E808191810196918380838091B0
:10B55000E30A9091E40AA091E50AB091E60A81FD20
:10B560007498409062025090630260906402709000
:10B5700065020E9484657C01FC018081982F929570
:10B580009F70913099F48F7051F48091731C909159
:10B59000741C01969093741C8093731C3AC1B6017D
:10B5A00087E795E30E94BB5C892B51F08091711C69
:10B5B0009091721C01969093721C8093711C29C10A
:10B5C000D301C2013EE0B695A795979587953A9528
:10B5D000D1F7F82FF170AF2E84E29BE00E94CD5F8F
:10B5E0008C01892B09F448C0B601C80102960E945B
:10B5F000BB5C892BE9F1980147E95AE060E074E609
:10B60000C8010F960E945162F7019181F80184816F
:10B61000981321C082858F5F828780916F1C9091E3
:10B62000701C01969093701C80936F1C84E00E94A4
:10B63000A366F801208530E02817390708F079C1A2
:10B6400084E00E94A366F8018087F70180818F70F3
:10B65000F8018187DEC0F801128684E00E94A366AB
:10B66000F8018087F70180818F70F801818762C1BE
:10B67000C8010E947960B4CF84E092E00E94615FCB
:10B680008C01892B09F4C5C0B601C80102960E943D
:10B69000B25CF70181818150F801848380E091E000
:10B6A000A0E0B0E083879487A587B687128684E000
:10B6B0000E94A366F8018087F70180818F70F801EE
:10B6C0008187B80184E29BE00E943160980147E9DC
:10B6D0005AE060E074E6C8010F960E945162BB24F4
:10B6E000B394F7018181F8018483F70180818F7021
:10B6F000F801878384E00E94A366F801858383E0D4
:10B700000E94A366F801868387818F3009F0B12CEF
:10B71000F7014180F8018481481A512C612C712C69
:10B7200086E0440C551C661C771C8A95D1F723854E
:10B73000348545855685A0ECB0E00E948D9CBB27E2
:10B74000A92F982F872F480E591E6A1E7B1E4386ED
:10B75000548665867686A601B801C7010E94E80A6C
:10B7600080917B1D90E02091DA0A3091DB0A8217EC
:10B77000930738F040E050E062E18CE092E00E94F4
:10B78000DE5E8091DA0A9091DB0A029708F44DC0E0
:10B790008091922C9091932C91FF2AC00E944A6B29
:10B7A000C70105960E94166BF70181811F928F9346
:10B7B000F80186811F928F9385811F928F9384EB6E
:10B7C00099E09F938F931F9280E18F93CE01019612
:10B7D0006C019F938F930E9464A382E00E94306B60
:10B7E000C6010E94166B0FB6F894DEBF0FBECDBF28
:10B7F0008091620290916302A0916402B09165020F
:10B8000097FD4DC08091DA0A9091DB0A029708F407
:10B810007AC08091E30A9091E40AA091E50AB09180
:10B82000E60A81FF89C0749A87C080916202909174
:10B830006302A0916402B091650296FFA9CFAA208D
:10B8400009F4A6CFF7018081982F9F709230E8F01D
:10B850009150807F892B808389E19BE00E94815AEF
:10B8600080916D1C90916E1C019690936E1C80933C
:10B870006D1C8091E30A9091E40AA091E50AB091D1
:10B88000E60A96FF85CF739883CF8091731C9091C1
:10B89000741C01969093741C8093731C79CF8CE573
:10B8A0009CE120915C1C222309F4ACCF9F938F93E1
:10B8B00087EC99E09F938F93CE0101963C019F9373
:10B8C0008F930E94A1A36C01B301C70102960E944D
:10B8D00077A20F900F900F900F900F900F900097FE
:10B8E00009F490CFEFEFCE1ADE0A8C0D9D1DAC014E
:10B8F0000196FA0120812032D1F362E186E192E0E3
:10B900000E94DE5E7FCFBB2009F483CF82E080936C
:10B91000AD301092AF301092AE301093B130009332
:10B92000B0304DEA50E362E18EE392E00E94DE5EC9
:10B9300070CFA12CB12CD5CE60960FB6F894DEBF97
:10B940000FBECDBFDF91CF911F910F91FF90EF9070
:10B95000DF90CF90BF90AF907F906F905F904F90AF
:10B9600008950895FB012081FC012083FB012181C2
:10B97000FC0121830895FC019081DB018C919813D7
:10B9800009C021E090E0318111968C91381320E0BC
:10B99000822F089580E090E00895BC0187E795E349
:10B9A0000C94B25CDC011996ED91FC911A9702801F
:10B9B000F381E02D309709F0099408950F931F93B8
:10B9C000CF93DF9300D0CDB7DEB78C0188E10E9422
:10B9D000B666BC01CE0101960E94B25CD8011996F0
:10B9E000ED91FC911A970190F081E02DBE016F5FFF
:10B9F0007F4FC80109950F900F90DF91CF911F9154
:10BA00000F910895EF92FF920F931F93CF93DF93BF
:10BA10008C01EB017A014EE053E00E942C5DF801AD
:10BA2000F286E18662E173E0CE01DF91CF911F9152
:10BA30000F91FF90EF900C94865D0C94455DCF9331
:10BA4000DF93EC0167E775E388E10E94AC66CE0105
:10BA5000DF91CF910C94475DEF92FF920F931F936C
:10BA6000CF93DF938C01EB017A010E94625DF801B4
:10BA7000F086E78266E173E0CE01DF91CF911F91FE
:10BA80000F91FF90EF900C94865D0C946A5D0C947E
:10BA9000417DDC011796ED91FC9118970190F081A2
:10BAA000E02D0994DC011796ED91FC911897028026
:10BAB000F381E02D309709F00994089588E293E12D
:10BAC0000C94C95FFC0173836283BC0188E293E13B
:10BAD0000C943160BC0188E293E10C941260CF9326
:10BAE000DF93EC0188E293E10E94CD5F009749F07B
:10BAF000FC01228133812C173D0729F00E947960D7
:10BB0000F5CF80E090E0DF91CF9108950F931F93E0
:10BB1000CF93DF938B010E946F5DEC01892B31F095
:10BB20001D830C83C8010E946F7F8E83DF91CF91AC
:10BB30001F910F9108951F93CF93DF93DC0114960B
:10BB4000ED91FC9115973097E1F0162FEC01909351
:10BB50002B1380932A1382E08887CD0106960995DE
:10BB6000082E000C990B0297029710F0133839F445
:10BB7000BE01CE01DF91CF911F910C94CB5D81E08E
:10BB80008887DF91CF911F910895FC01208520FDCA
:10BB90000C949B5D0895CF92DF92EF92FF920F93EA
:10BBA0001F93CF93DF93E0902A13F0902B13C09054
:10BBB0002C13D0902D13F601E817F90739F03097C0
:10BBC00009F44BC00190F081E02DF6CF009709F405
:10BBD00044C08B01EC018885882309F11886C114C3
:10BBE000D10461F0CC15DD0529F0AE0167E8C6018E
:10BBF0000E94C55DF601C080D180F1CFEC81FD814E
:10BC0000309769F0C017D10751F0D0932B13C09330
:10BC10002A1340E050E063E8CE0106960995E091D2
:10BC20002C13F0912D13CE17DF0741F488819981F1
:10BC300090932D1380932C130CC0FC01309749F086
:10BC4000808191818C179D07C1F7888199819183AB
:10BC50008083F0922B13E0922A13DF91CF911F91F2
:10BC60000F91FF90EF90DF90CF9008951F93CF93A7
:10BC7000DF9310923613C0912C13D0912D1311E045
:10BC8000209779F08985882341F01887198640E04C
:10BC900050E062E8CE010E949B5D0990D881C02DE2
:10BCA000EFCFDF91CF911F9108958091D91391E04B
:10BCB000980F9093D913089560912A1370912B13C4
:10BCC0000C94CB5D8AE88093D9131092D71310920D
:10BCD000D81310922D1310922C1310922B13109234
:10BCE0002A1308958091361381110E94365E509177
:10BCF000D813552309F452C0E091D7132E2F30E00A
:10BD000085E0E89FF0011124E95CFC4E60816093BE
:10BD10003513A181B281B0933413A093331383817F
:10BD2000948190933213809331132F5F3F4F2F7183
:10BD300033272093D71351505093D813009731F5E0
:10BD400080912C1390912D139093301380932F1387
:10BD500080912F1390913013892B01F1809136132C
:10BD600081110E94365E40913313509134136091DB
:10BD7000351380912F13909130130E94C55DE0918F
:10BD80002F13F091301380819181DECF613819F447
:10BD900021E0FC012087AD010E94C55D8091361332
:10BDA0002091D81390E0820F911D08958091361351
:10BDB0002091D81390E0820F911D08959C019091DD
:10BDC000D8139032B9F0E091D713E90FEF71E093F7
:10BDD0002E1385E0E89FF0011124E95CFC4E60839E
:10BDE00052834183348323839F5F9093D81380E0F1
:10BDF00090E0089581E090E00895CF93DF93C091A3
:10BE00002A13D0912B130E94C55DD0932B13C0939E
:10BE10002A13DF91CF910895AB0130912C1320911B
:10BE20002D13E32FF22FE817F907B1F0309721F027
:10BE30000190F081E02DF7CF009771F0FC01308385
:10BE4000218390932D1380932C1321E02087178258
:10BE5000168261E80C94FD5E0895009749F0FC019C
:10BE600020852150223020F421E0218720933613B1
:10BE7000089521E030E0FC018085811102C020E0BE
:10BE800030E0C9010895CF93DF93EC014A815B81D3
:10BE900060E070E08C819D810E9446A22A813B81F6
:10BEA00088819981289FA001299F500D389F500DAE
:10BEB000112460E070E08E819F81DF91CF910C941E
:10BEC00046A2FC018281938120E030E028173907E7
:10BED000D1F0A481B581A20FB31F4C91411110C0C4
:10BEE00081E08C9380819181289FA001299F500D32
:10BEF000389F500D112486819781840F951F0895D6
:10BF00002F5F3F4FE3CF80E090E00895FC018681F2
:10BF100097814281538120E030E024173507D1F02A
:10BF20008617970781F4A481B581A20FB31F8C9166
:10BF3000181614F481508C9384819581FC01E20FD2
:10BF4000F31F80810895A081B1818A0F9B1F2F5F0D
:10BF50003F4FE3CF8FEF0895FC01268137816217B1
:10BF60007307A0F0A081B18142815381A49FC001D9
:10BF7000A59F900DB49F900D1124280F391F81E0CB
:10BF800090E06217730720F080E0089580E090E071
:10BF90000895FC01118210820895FC018081918135
:10BFA0000895FB0120813181FC01318320830895B4
:10BFB000DC01ED91FC91309741F0808191810097F7
:10BFC00011F0FC01FACFCF01089580E090E00895D0
:10BFD000DC01ED91FC9111973097A9F0208131811E
:10BFE000232B21F41D921C92CF010895A081B181D1
:10BFF0008D919C911197892B11F0FD01F7CF118242
:10C000001082CD01089580E090E00895DC01ED916B
:10C01000FC911197309721F0208131812D933C9331
:10C02000CF010895DC01ED91FC913097C9F0A0E0BB
:10C03000B0E0E617F70761F4FB012081318110972A
:10C0400009F4DC012D933C93FB01118210820895C9
:10C0500020813181DF012115310511F0F901E9CF8E
:10C0600008950F931F93CF93DF938C01EB010E94F0
:10C07000126019821882C8010E94D85F009711F4DB
:10C08000F80101C0FC01D183C083DF91CF911F91E2
:10C090000F9108950F931F93CF93DF93EC018B01C2
:10C0A0000E94126088819981F801918380831983AD
:10C0B0000883DF91CF911F910F910895DC01ED91DD
:10C0C000FC9180E090E0309729F001960190F0819A
:10C0D000E02DF9CF0895FB01309719F4BA010C94C3
:10C0E0004A6080819181DA018D939C9351834083D2
:10C0F0000895009721F0FC0180819181089580E0EE
:10C1000090E008958091DC139091DD13892B29F440
:10C110001092DB131092DA1308950E94A06FE09141
:10C12000DC13F091DD132281338140815181240F92
:10C13000351F281B390B0480F581E02D309769F0FD
:10C140006281738140815181460F571F481B590BF3
:10C150004217530780F79A01EECF820F931F9093F7
:10C16000DB138093DA13089580E992E00C942D5F3D
:10C17000EF92FF920F931F93CF93DF938C01FC01FB
:10C1800080819181009799F08A359105D9F0F80165
:10C190001182108283E068C0868197818417950799
:10C1A00009F049C00480F581E02D3097A9F710927D
:10C1B000DD131092DC138AE590E0F801918380830F
:10C1C00081E052C0673891F16238A9F7C091DC1361
:10C1D000D091DD13E12CF12C209769F3CE010E9460
:10C1E0003883892BF1F0AE0168E88E819F810E942F
:10C1F000DE5E892BA1F41F821E828C819D81E11459
:10C20000F10421F0F7019583848304C09093DD133A
:10C210008093DC131D821C820E948260D7CF0E9413
:10C22000B4607E010C80DD81C02DD6CFE091DC139F
:10C23000F091DD13BACFF093DD13E093DC13A4810A
:10C24000B581109709F4B7CF16968D919C911797E9
:10C250008417950739F414968D919C9115979583C1
:10C260008483EDCFFD01EBCFDF91CF911F910F9133
:10C27000FF90EF900895CF93DF93EC010E94B4609C
:10C280002E813F819091DC138091DD13232B59F097
:10C29000E92FF82F309739F0EC17FD0781F0048073
:10C2A000F581E02DF7CF20912A1330912B133F8396
:10C2B0002E839C838D83D093DD13C093DC13DF9199
:10C2C000CF910C948260CF93DF93EC010E9418838E
:10C2D000CE01DF91CF910C943B61CF93DF93EC01C2
:10C2E0000E942483CE01DF91CF910C943B61CF93C8
:10C2F000DF93EC010E942E83CE01DF91CF910C944D
:10C300003B61FC0120813181620F731F7183608367
:10C310000C94826021E030E0FC0186819781892BBA
:10C3200011F020E030E0C9010895FC012281338141
:10C3300080819181820F931F0895FC0180819181FA
:10C34000089581E090E02091DC133091DD13232BE0
:10C3500011F480E090E008958091DC139091DD135A
:10C36000892B29F08091DA139091DB13089580E0F6
:10C3700090E00895CF93DF93EC01E091DC13F0910E
:10C38000DD138E179F0769F48C819D819093DD13D7
:10C390008093DC130DC0848195818C179D0721F05B
:10C3A000FC013097C1F706C08C819D819583848301
:10C3B0000E9482601D821C821F821E82DF91CF91AB
:10C3C0000895EF92FF920F931F93CF93DF938C0109
:10C3D0007A01FC0180819181009741F08B349105B5
:10C3E00001F1F8011182108283E048C08FED93E1E2
:10C3F0000E94CD5FEC01209751F06C817D81CE01D0
:10C4000002960E9463610990D881C02DF4CF81E02B
:10C410008093DE138BE490E0F8019183808381E0C8
:10C420002DC06838E1F78FED93E10E94CD5FEC01FC
:10C43000209781F3CE010296E816F906D9F4BE01E1
:10C440008FED93E10E941260E0902A13F0902B137D
:10C450008A859B8590932B1380932A13EC85FD8509
:10C46000309719F08E859F850995F0922B13E092F5
:10C470002A13D0CF0990D881C02DDACFDF91CF9188
:10C480001F910F91FF90EF9008951092DE138FEDA2
:10C4900093E10E94C95F60E070E08AE992E00C9449
:10C4A0000C5F0F931F93CF93DF93EC0100912A133E
:10C4B00010912B131B870A875D874C873F872E8738
:10C4C0008091DE13882379F08AE992E090932B1310
:10C4D00080932A13CE0102960E94636110932B135E
:10C4E00000932A1302C07D836C83BE018FED93E11C
:10C4F0000E941260BE018FED93E1DF91CF911F91F9
:10C500000F910C9431600F931F93CF93DF93EC0145
:10C510008091DE13882391F000912A1310912B1340
:10C520008AE992E090932B1380932A13CE0102960E
:10C530000E946D6110932B1300932A13BE018FED9F
:10C5400093E10E941260BE018FED93E1DF91CF91E4
:10C550001F910F910C9431600F931F93CF93DF9332
:10C56000EC018091DE13882391F000912A13109141
:10C570002B138AE992E090932B1380932A13CE0118
:10C5800002960E94776110932B1300932A13BE0129
:10C590008FED93E10E941260BE018FED93E1DF9178
:10C5A000CF911F910F910C943160CF93DF93EC01E9
:10C5B0008091DE13882329F0CE0102960E94BA6191
:10C5C00004C01F821E8219861886BE018FED93E17A
:10C5D000DF91CF910C941260CF93DF932091DE1303
:10C5E000222329F00296DF91CF910C948A61EC010D
:10C5F0008FED93E10E94CD5F009739F08C179D0776
:10C6000039F0FC0180819181F7CF81E090E002C098
:10C6100080E090E0DF91CF9108952F923F924F926A
:10C620005F926F927F928F929F92AF92BF92CF92C2
:10C63000DF92EF92FF920F931F93CF93DF93CDB7CB
:10C64000DEB7E8970FB6F894DEBF0FBECDBFE6E6C3
:10C65000F7E3AAEAB7E32C9111963C911197129651
:10C660004C91129713965C91A6EAB7E35C901196F1
:10C670004C90119712963C90129713962C9094AC74
:10C680008090A3377090A4376090A53780AD8983E0
:10C6900091AD9A8382AD8B8393AD9C8384A98D8366
:10C6A00095A99E8386A98F8397A9988780A9898752
:10C6B00091A99A8782A98B8793A99C8784A58D8746
:10C6C00095A59E8786A58F8797A5988B80A5898B32
:10C6D00091A59A8B82A58B8B93A59C8B84A18D8B26
:10C6E00095A19E8B86A18F8B97A1988F80A1898F12
:10C6F00091A19A8F82A18B8F93A19C8F848D8D8F16
:10C70000958D9E8F868D8F8F978D98A3808D89A311
:10C71000918D9AA3828D8BA3938D9CA384898DA3E5
:10C7200095899EA386898FA3978998A7808989A7D1
:10C7300091899AA782898BA793899CA784858DA7C5
:10C7400095859EA786858FA7978598AB808589ABB1
:10C7500091859AABB284A384F480E580D680C780AB
:10C7600080818FAB918198AF128103812BAB3CAB61
:10C770004DAB5EAB0E94CC6F5EA95F934DA94F930A
:10C780003CA93F932BA92F932F923F924F925F92F8
:10C790006F927F928F929F922C812F932B812F9358
:10C7A0002A812F9329812F9328852F932F812F93CF
:10C7B0002E812F932D812F932C852F932B852F93B3
:10C7C0002A852F9329852F9328892F932F852F939F
:10C7D0002E852F932D852F932C892F932B892F9383
:10C7E0002A892F9329892F93288D2F932F892F936F
:10C7F0002E892F932D892F932C8D2F932B8D2F9353
:10C800002A8D2F93298D2F9328A12F932F8D2F932E
:10C810002E8D2F932D8D2F932CA12F932BA12F9302
:10C820002AA12F9329A12F9328A52F932FA12F93CE
:10C830002EA12F932DA12F932CA52F932BA52F93B2
:10C840002AA52F9329A52F9328A92F932FA52F939E
:10C850002EA52F932DA52F93AF92BF922AA92F9388
:10C8600029A92F93CF92DF92EF92FF920F931F93FC
:10C8700028AD2F932FA92F939F938F937F936F931F
:10C88000809178351F928F93E7E7F5E380811F92BF
:10C890008F938EE791E19F938F930E940CA3EEEA12
:10C8A000F7E324A535A546A557A550A441A432A475
:10C8B00023A4848D8983858C768C678C908D9A8354
:10C8C000818D8B83928D9C83838D8D8394899E83B0
:10C8D00085898F83968998878789898790899A87A0
:10C8E00081898B8792899C8783898D8794859E8790
:10C8F00085858F879685988B8785898B90859A8B80
:10C9000081858B8B92859C8B9384D480C580B680E7
:10C91000A78010810181F280E3800FB6F894DEBF1A
:10C920000FBECDBF2BAB3CAB4DAB5EAB0E94CC6F13
:10C930005EA95F934DA94F933CA93F932BA92F93D9
:10C940002F923F924F925F926F927F928F922981A6
:10C950002F932D812F932C812F932B812F932A811D
:10C960002F9329852F9328852F932F812F932E8105
:10C970002F932D852F932C852F932B852F932A85ED
:10C980002F9329892F9328892F932F852F932E85D5
:10C990002F939F922C892F932B892F932A892F9342
:10C9A000AF92BF92CF92DF92EF92FF920F931F93BD
:10C9B0009F938F937F936F93809178351F928F937E
:10C9C000E7E7F5E380811F928F938FE091E19F93DA
:10C9D0008F930E940CA30FB6F894DEBF0FBECDBF9D
:10C9E000E8960FB6F894DEBF0FBECDBFDF91CF91B2
:10C9F0001F910F91FF90EF90DF90CF90BF90AF907D
:10CA00009F908F907F906F905F904F903F902F906E
:10CA1000089580E3809395140895CF93DF936091F8
:10CA2000951470E0C0E3D0E0C61BD70B6D517C4E6F
:10CA3000AE010E943DA2CE01DF91CF910895CF9229
:10CA4000DF92EF92FF920F931F93CF93DF93C090EB
:10CA50009814D09099146091951470E0E601E096D6
:10CA6000C61BD70BC138D105E0F47C0100E310E010
:10CA7000061B170B6D517C4EA8010E943DA26091D0
:10CA8000E1137091E2138091961490919714680FBE
:10CA9000791FA601C701800F911F0E943DA2CE0100
:10CAA00002C080E090E0DF91CF911F910F91FF9045
:10CAB000EF90DF90CF90089590919514890F809317
:10CAC00095140895209198143091991428173907D6
:10CAD00098F04091961450919714480F591F509315
:10CAE000971440939614281B390B30939914209374
:10CAF000981481E090E0089580E090E0089590938C
:10CB00009914809398140895809196149091971495
:10CB10008D5E9B4E08958091951490E08D519C4EB2
:10CB2000089581E090E02091E1133091E2132351C8
:10CB3000344111F480E090E008950E949165892BC2
:10CB400061F06091E1137091E2134091981450915B
:10CB5000991483E194E10C943DA2209196143091B4
:10CB6000971421153105B9F080919814909199147A
:10CB7000C096E3E1F4E1AF01435E53414817590722
:10CB800034F4DF01A20FB31F4C914193F4CF109204
:10CB900097141092961408958091E1139091E213E6
:10CBA00008958091981490919914089590919514F6
:10CBB00080E3891B08958091951490E3981B209140
:10CBC000981430919914A901490F511DCA01089573
:10CBD0000F931F93CF938C01C09195148C2F90E0ED
:10CBE000801791076CF00E94DB65800F911F8138E0
:10CBF000910530F4C01BC093951481E090E002C011
:10CC000080E090E0CF911F910F910895CF93DF9333
:10CC1000E1E8F5E31192119285E3E13BF807D1F7E2
:10CC2000C9E7D5E36CE073E0CE010E94B25C2296C6
:10CC300085E3C138D807B1F7DF91CF9108951092FD
:10CC4000971410929614109299141092981480E3ED
:10CC50008093951483E194E19093E2138093E11320
:10CC60000C940666EF92FF920F931F93CF93DF937E
:10CC700000D0CDB7DEB78C0169837A830E941F662E
:10CC80006981E62E7A81F72E81E8E816F10418F022
:10CC900080E8E82EF12CA701B8018091E113909172
:10CCA000E2130E943DA2F0929914E0929814C701F9
:10CCB0000F900F90DF91CF911F910F91FF90EF9008
:10CCC00008950F931F93CF93DF938C01EB010E9484
:10CCD0001F661093E2130093E113D0939914C0934D
:10CCE0009814DF91CF911F910F910895DC0190E38B
:10CCF000E1E8F5E301900D929A95E1F788E0E9E724
:10CD0000F5E3DB0101900D928A95E1F70895FC01AE
:10CD100090E3A1E8B5E301900D929A95E1F788E0E0
:10CD2000FB01A9E7B5E301900D928A95E1F708951B
:10CD3000E82FF0E0EE0FFF1FEF57FA4C718360838E
:10CD400081E090E00895E82FF0E0EE0FFF1FEF572D
:10CD5000FA4C80819181089590E0880F991F875B3C
:10CD60009A4C0E94B25C81E090E0089590E0880FB8
:10CD7000991F875B9A4C08958115910511F00197D1
:10CD8000F1F70895E091B435F091B5359081809137
:10CD9000B33589230895E091B135F091B235908192
:10CDA0008091B335892B8083E091B635F091B7350A
:10CDB00090818091B335892B80830895E091B135BE
:10CDC000F091B23590818091B3358095892380832D
:10CDD000E091B635F091B73590818091B33580956B
:10CDE0008923808308951F93CF93DF93E091B1351A
:10CDF000F091B23590818091B335809589238083FD
:10CE0000E091B635F091B73590818091B335892B9B
:10CE100080838FEB93E00E94BC661FB7F894E0918B
:10CE2000B635F091B73590818091B33580958923DF
:10CE3000808383E890E00E94BC66E091B435F09175
:10CE4000B535D081C091B3351FBF78948BE393E0A3
:10CE50000E94BC66E091B435F091B5358081909127
:10CE6000B335982319F08D2F8C2301C081E0DF9119
:10CE7000CF911F9108955093B7354093B635709375
:10CE8000B2356093B1359093B5358093B43581E078
:10CE900001C0880F2A95EAF78093B3350C94F366A6
:10CEA000CF93DF93C82FDFB7F894E091B635F091B8
:10CEB000B73590818091B335892B808383E090E0F2
:10CEC0000E94BC66CC2351F0E091B635F091B735A5
:10CED00090818091B33580958923808387E190E0AC
:10CEE0000E94BC66E091B435F091B5359081809197
:10CEF000B335892309F4C0E089E590E00E94BC665F
:10CF0000E091B635F091B73590818091B335809539
:10CF100089238083DFBF8BE390E00E94BC668C2F67
:10CF2000DF91CF910895CF93DF93C82FD8E08C2F56
:10CF300081700E945067C6958111C068D150B9F7C1
:10CF40008C2FDF91CF9108958FEF0C949367DF9230
:10CF5000EF92FF920F931F93CF93DF93E82E8B01F5
:10CF60000E94F366811135C080EF0E949367D0E084
:10CF7000C0E488EFD82EDC0E81E00E945067F82EC6
:10CF800081E00E945067882319F0FF2071F023C0D0
:10CF9000F1100BC0CE1530F0F801808180FF05C084
:10CFA000EC1619F0DC2FFF24F3948F2D0E945067AC
:10CFB000F80190819695FF2011F09068F801908318
:10CFC000C150CD11D9CF0F5F1F4FC111D2CF8D2FBF
:10CFD00003C08FEF01C08EEFDF91CF911F910F91B2
:10CFE000FF90EF90DF900895EF92FF921F93CF9301
:10CFF000DF93182FEB010E94F366209771F085E50F
:10D000000E9493677E0188E0E80EF11C89910E94DE
:10D010009367CE15DF05D1F703C08CEC0E949367B0
:10D02000812FDF91CF911F91FF90EF900C94936728
:10D030000F931F93CF93DF93DB01EC9111969C919B
:10D040001197F0E0F92B803179F4EE7F63E0EE0F79
:10D05000FF1F6A95E1F716969C9116976CE070E0B9
:10D06000691B7109E60FF71FF7FF07C091E0EA019E
:10D070009883F195E195F10902C0EA01188288329E
:10D0800079F414968C91982F9076903649F086FF1B
:10D0900002C0EE7F05C085FF02C0EC7F01C0E87FC3
:10D0A000CF0144E0969587954A95E1F7D9018C9395
:10D0B000EF70E801E88380E0DF91CF911F910F913D
:10D0C00008950F931F93CF93DF93EC018B01B80169
:10D0D00088810E94A76788839FEF980F9D3F30F457
:10D0E000F8019081983211F0903189F7DF91CF915A
:10D0F0001F910F910895CF93DF93EC010E94F36687
:10D10000BE0184EB0E94F46781E00E945067C82F43
:10D110000E94F36681E0C11101C080E0DF91CF91F0
:10D1200008951F93CF93DF9300D0CDB7DEB7182FAC
:10D1300069837A830E94F3660E94C26669817A815C
:10D14000882341F084E40E94F467113029F00E94A2
:10D15000CB6602C082E001C080E00F900F90DF91AB
:10D16000CF911F9108955F926F927F928F929F92BD
:10D17000AF92BF92CF92DF92EF92FF920F931F93E5
:10D18000CF93DF93CDB7DEB729970FB6F894DEBF04
:10D190000FBECDBF5C014B013A0189010E94F366CD
:10D1A000B5018EEB0E94F467CE0101967C016C0103
:10D1B00099E0592E5E0C0E94A467F60181936F01DD
:10D1C0005E12F9CF69E070E0C7010E94B287D82EE5
:10D1D000811108C09301A401B701F50180810E946B
:10D1E000186802C083E0D82E8D2D29960FB6F894CA
:10D1F000DEBF0FBECDBFDF91CF911F910F91FF908A
:10D20000EF90DF90CF90BF90AF909F908F907F90E6
:10D210006F905F9008956F927F928F929F92AF92DE
:10D22000BF92CF92DF92EF92FF920F931F93CF9313
:10D23000DF93CDB7DEB729970FB6F894DEBF0FBEE8
:10D24000CDBF782E5B014A01890160E070E08EEB72
:10D250000E94F467CE0101967C016C0199E0692E71
:10D260006E0C0E94A467F60181936F016E12F9CFD4
:10D2700069E070E0C7010E94B287D82E811107C013
:10D280009401A501B701872D0E94186802C083E0B0
:10D29000D82E8D2D29960FB6F894DEBF0FBECDBFC8
:10D2A000DF91CF911F910F91FF90EF90DF90CF9082
:10D2B000BF90AF909F908F907F906F9008950F9345
:10D2C0001F93CF93DF93CDB7DEB728970FB6F894AF
:10D2D000DEBF0FBECDBF182F062F98E0E8E1F3E0C8
:10D2E000DE01119601900D929A95E1F7242F440FDB
:10D2F000330B41E752E0249FC001259F900D349FDE
:10D30000900D112464E670E00E940A9C84E6089F58
:10D31000600D711D1124FE01319688E08E0F419140
:10D3200050E02417350719F46F5F7F4F02C08E134A
:10D33000F6CF112319F0719561957109CB012896EB
:10D340000FB6F894DEBF0FBECDBFDF91CF911F9116
:10D350000F9108950F931F93CF93DF93CDB7DEB74F
:10D360002B970FB6F894DEBF0FBECDBF182F092F35
:10D37000682F792F88E0810F0E949168882319F027
:10D3800084E391E243C066E471E48FE090E00E94A0
:10D39000116A9E01275F3F4FAE01465F5F4FBE019E
:10D3A000655F7F4F812F902F0E94B3688111E8CF76
:10D3B00088E0E8E1F3E0DE01119601900D928A9594
:10D3C000E1F7298541E752E0249FC001259F900D98
:10D3D000112464E670E00E940A9C8A8594E6899F85
:10D3E000600D711D1124FE01319688E08E0F919120
:10D3F000291303C06F5F7F4F02C08E13F8CF8B8558
:10D40000882319F0719561957109CB012B960FB6A0
:10D41000F894DEBF0FBECDBFDF91CF911F910F916A
:10D420000895DC01CB0181159105A105B10529F015
:10D4300081509040A040B040D9F708959B01AC01C5
:10D440001092B90060E072E18AE790E00E941E9CB1
:10D45000DA01C9014097A109B109B695A795979539
:10D4600087958093B800089594EA9093BC0040EAB1
:10D4700056E861E070E09091BC0097FD07C0415014
:10D48000510961097109B9F781E008959091B900D6
:10D49000987F983011F09031B9F78093BB0084E801
:10D4A0008093BC0080EA96E8A1E0B0E02091BC0047
:10D4B00027FD05C00197A109B109C1F7E5CF80910A
:10D4C000B900887F883111F08034F1F680E008954A
:10D4D00024EA34E844E92093BC009091BC0097FF13
:10D4E000FCCF9091B900987F983011F0903199F766
:10D4F0008093BB003093BC009091BC0097FFFCCFA1
:10D500009091B900987F903211F0983539F440939A
:10D51000BC009091BC0094FDFCCFDDCF08950C942D
:10D52000346A84E98093BC008091BC0084FDFCCF08
:10D5300008958093BB0084E88093BC008091BC0078
:10D5400087FFFCCF9091B900987F81E0983209F471
:10D5500080E0089584EC8093BC008091BC0087FF3C
:10D56000FCCF8091BB00089584E88093BC0080913B
:10D57000BC0087FFFCCF8091BB000895CF93DF9361
:10D58000FC017096EC01A991CE01A0933F01CE174A
:10D59000DF07C1F780913C018F7D80933C01809132
:10D5A0003C01877F80933C01DB015096FB01819118
:10D5B00080933E01EA17FB07D1F780913C01806818
:10D5C00080933C0180913D0180FFFCCF4051510987
:10D5D00080913C01806280933C0180913C01877F77
:10D5E00080933C01141615069CF4FB0181918093F5
:10D5F0003E01EA17FB07D1F780913C0180688093D8
:10D600003C0180913D0180FFFCCF40515109EACFA0
:10D61000F901C901409620913E012193E817F907CD
:10D62000D1F781E090E0DF91CF9108950F931F93A0
:10D63000CF93DF93EC018CE70E94686A8CE70E942D
:10D64000996A8E01005F1F4F89910E94996AC017E5
:10D65000D107D1F7DF91CF911F910F910C94916A6F
:10D66000813019F440E050E002C040EC50E060E04E
:10D6700070E08CE790E00C947412813019F44EE065
:10D6800050E002C048E050E060E070E08CE790E0DD
:10D690000C94741241E050E060E070E08CE790E0A0
:10D6A0000E9474126AE67AE080E090E00C94116ABD
:10D6B00048E350E060E070E08CE790E00E94741274
:10D6C00049E350E060E070E08CE790E00E94741263
:10D6D00044E150E060E070E08CE790E00E9474125A
:10D6E00048E750E060E070E08CE790E00E94741240
:10D6F0004EE550E060E070E08CE790E00E9474122C
:10D700004DE650E060E070E08CE790E00E9474121B
:10D710006CE17AE186E090E00E94116A4CE050E012
:10D7200060E070E08CE790E00E94741241E050E00D
:10D7300060E070E08CE790E00E94741246E050E0F8
:10D7400060E070E08CE790E00E9474126AE67AE094
:10D7500080E090E00C94116ACF93DF93CDB7DEB7F1
:10D76000A2970FB6F894DEBF0FBECDBF81E1EBE507
:10D77000FAE0DE01529601900D928A95E1F781E17F
:10D78000ECE6FAE0DE01119601900D928A95E1F740
:10D790000E94586BCE0142960E94166B82E00E9456
:10D7A000306B6AE67AE080E090E00E94116ACE0178
:10D7B00001960E94166B60E17EEA88E290E00E948A
:10D7C000116A80E00E943D6B60E17EEA88E290E0B1
:10D7D0000E94116A4EE050E060E070E08CE790E05B
:10D7E0000E947412A2960FB6F894DEBF0FBECDBF92
:10D7F000DF91CF910895CF92DF92EF92FF920F9336
:10D800001F93CF93DF9300D01F92CDB7DEB7042FC5
:10D81000122F213061F0223031F0243031F02830E5
:10D8200031F493E005C091E003C092E001C090E0C4
:10D83000E82FF0E08160F82E0C3009F4E0C00E30E3
:10D8400011F49460DCC0003111F49860D8C002314A
:10D8500009F0D5C0613009F4B7C09C60623011F4A2
:10D86000906207C0633011F4906403C0643009F41F
:10D8700090669068692F70E023E030E0AE014F5F62
:10D880005F4FCF010E948B1269E07AE180E090E067
:10D890000E94116A8F2D0E94346A0E94AA6A8983AD
:10D8A0000E94AA6A8A83023119F40E94AA6A8B83B1
:10D8B0000E94AA6A87FDF1CF0E94B46A0E94916A11
:10D8C00069E07AE180E090E00E94116A8F2D0E9469
:10D8D000346A0E94AA6A89830E94AA6A8A830231F2
:10D8E00019F40E94B46A8B830E94B46A0E94916A00
:10D8F00069812A81023139F5862F90E0A0E0B0E0FD
:10D900004B81DC019927882730E0322F2227820FB4
:10D91000931FA11DB11D61FF09C0840F911DA11DA1
:10D92000B11DBC01CD018C6F9F6F06C0BC01CD0144
:10D93000640F711D811D911D0E94139920E83FEF16
:10D940004FEF57E41FC070E0762F6627620F711DFE
:10D95000072E000C880B990B0E9413990C3029F4A8
:10D9600020E030EE4FEF54E40DC00E3029F420E0FB
:10D9700038EF4FEF55E406C0003131F420E03EEFC0
:10D980004FEF56E40E945F982FE632E143E050E407
:10D990000E940B9B6B017C01612F70E080E090E0A6
:10D9A0000E9413999B01AC01C701B6010E945F98C8
:10D9B0000F900F900F90DF91CF911F910F91FF90DB
:10D9C000EF90DF90CF9008959C68692F70E023E07E
:10D9D00030E0AE014F5F5F4FCF010E948B1269E0D4
:10D9E0007AE180E090E00E94116A8F2D0E94346AF3
:10D9F0000E94AA6A89830E94AA6A8A8356CF6130EC
:10DA000009F02CCF9068692F70E023E030E0AE0180
:10DA10004F5F5F4FCF010E948B1269E07AE180E097
:10DA200090E00E94116A8F2D0E94346A0E94AA6AB7
:10DA300089830E94AA6A8A833BCFE6E4F1E0908161
:10DA4000208130818081929596959695937022954C
:10DA50002F70922B892B232F22952F70822B0895C4
:10DA60000F931F93CF93DF9300D0CDB7DEB746E07F
:10DA70006CE080E00E94627089E18093C4001092A3
:10DA8000C50082E08093C00080E00E94F2700E9496
:10DA9000906F84B784B784B784B784B78DE79AE072
:10DAA0009F938F938BEC92E19F938F930E940CA393
:10DAB0000E94EC830E94625E60E070E080E992E088
:10DAC0000E940C5F0E944562E0912003F0912103C7
:10DAD00009950E941D6D90E00E942884CE01019658
:10DAE0000E94BE6E0F900F900F900F90882341F010
:10DAF0008BEA92E19F938F930E940CA30F900F905B
:10DB0000CE0101960E94CD5C0E94CC6E8C010E94D9
:10DB1000C86EAE014F5F5F4FB8010E94C4730E9490
:10DB20002E6E0E94A5730E94D06E0E94FD748EE935
:10DB300092E19F938F930E940CA38A811F928F93EF
:10DB40000AE912E11F930F930E940CA389811F928F
:10DB50008F931F930F930E940CA388E992E19F93E8
:10DB60008F930E940CA30E942C84E0915D03F0919E
:10DB70005E030995E0914F03F09150030995E09100
:10DB80003603F091370309950E940475182F0E94FF
:10DB9000A2731F921F931F928F9380915C038F93A8
:10DBA00080915B038F9380914E038F9380914D03FF
:10DBB0008F938DE792E19F938F930E940CA3E09146
:10DBC0006703F09168030FB6F894DEBF0FBECDBFB8
:10DBD000309791F00995BC0180E890E00E94F69B97
:10DBE0007F936F938AE692E19F938F930E940CA399
:10DBF0000F900F900F900F9088E692E19F938F9374
:10DC00000E940CA360E070E086EE92E00E940C5F40
:10DC10008AEF92E00E94FC8280E692E19F938F93CC
:10DC20000E940CA30F900F900F900F900F900F90E9
:10DC3000DF91CF911F910F9108957F936F939F93E1
:10DC40008F938AE592E19F938F930E940CA30F908C
:10DC50000F900F900F900F900F900895DF92EF921A
:10DC6000FF920F931F93CF93DF93CDB7DEB7A097AB
:10DC70000FB6F894DEBF0FBECDBF83E690E00E94E2
:10DC80000AA6182F282F35EF380F303108F0982FBB
:10DC90009095291709F463C086EE92E19F938F93C4
:10DCA0000E940CA3EBE2F3E18E010F5F1F4F0F9078
:10DCB0000F90D801D02EE12EF02E88E0800F9491A5
:10DCC0009D9331968A13FBCFF89448E050E06FE7BC
:10DCD00070E0C8010E9410A6EDE1F3E1D8018EE0EA
:10DCE0008F0D94919D9331968A13FBCF4EE050E0B7
:10DCF00061E770E0C8010E9410A6E3E1F3E12AE0C9
:10DD00002F0D8491D8018D938D0131962A13F9CF6F
:10DD10004AE050E067E670E08D2D9E2D0E9410A62F
:10DD20006DEC7BEA81E690E00E9428A660E070E05E
:10DD30008FE590E00E9428A660E08EE590E00E94CA
:10DD40001AA660E070E085E690E00E9428A61AE13D
:10DD50006AE175EE83E690E00E9428A67894812F10
:10DD6000A0960FB6F894DEBF0FBECDBFDF91CF9166
:10DD70001F910F91FF90EF90DF900895F89442E08B
:10DD800050E06FE770E00E94F2A5789480E008957B
:10DD900081E690E00C940AA68FE590E00C940AA628
:10DDA0008EE590E00C9402A60F931F930091C2356C
:10DDB0001091C3352091C4353091C535482F50E0BE
:10DDC00060E070E0DB01CA01800F911FA21FB31F4A
:10DDD0008093C2359093C335A093C435B093C535B5
:10DDE0008091BE359091BF35A091C035B091C135BD
:10DDF000840F951FA61FB71F8093BE359093BF3524
:10DE0000A093C035B093C135809162378823A1F0CB
:10DE10008091BA359091BB35A091BC35B091BD359C
:10DE2000480F591F6A1F7B1F4093BA355093BB356B
:10DE30006093BC357093BD351F910F9108951F926B
:10DE40000F920FB60F9211240BB60F922F933F93A0
:10DE50004F935F936F937F938F939F93AF93BF93F2
:10DE6000EF93FF9380919C1490919D140196909351
:10DE70009D1480939C1480919B148F5F80939B14BE
:10DE80008038A9F410929B148091C2359091C335CB
:10DE9000A091C435B091C5350196A11DB11D8093E7
:10DEA000C2359093C335A093C435B093C5358091E6
:10DEB00062378823E1F080919A148F5F80939A14DF
:10DEC0008038A9F410929A148091BA359091BB359C
:10DED000A091BC35B091BD350196A11DB11D8093B7
:10DEE000BA359093BB35A093BC35B093BD350E9435
:10DEF000A161892B11F00E94B460FF91EF91BF9155
:10DF0000AF919F918F917F916F915F914F913F91D1
:10DF10002F910F900BBE0F900FBE0F901F90189572
:10DF2000F8941092B60016BC83EF87BD82E084BDE2
:10DF300094E095BD95B395BB80936E007894089559
:10DF400080919C1490919D1420919C1430919D146B
:10DF500082179307A9F70895009741F022E330E074
:10DF6000000021503109E1F70197F6CF08950F9392
:10DF70001F93CF93DF93EC010E94A06F8C010E944E
:10DF8000A06F801B910B8C179D07C8F3DF91CF9179
:10DF90001F910F91089508950F931F936091C235BB
:10DFA0007091C3358091C4359091C5350091C235CB
:10DFB0001091C3352091C4353091C5356017710774
:10DFC0008207930759F71F910F9108951F920F929F
:10DFD0000FB60F9211241092BC020F900FBE0F903B
:10DFE0001F9018951F920F920FB60F9211240BB627
:10DFF0000F922F933F934F935F936F937F938F93E2
:10E000009F93AF93BF93EF93FF93E091B202F09190
:10E01000B3028081E091BD02F091BE02309709F019
:10E020000995FF91EF91BF91AF919F918F917F9152
:10E030006F915F914F913F912F910F900BBE0F9079
:10E040000FBE0F901F9018951F920F920FB60F9250
:10E0500011241092C9020F900FBE0F901F901895B7
:10E060001F920F920FB60F9211240BB60F922F939F
:10E070003F934F935F936F937F938F939F93AF9350
:10E08000BF93EF93FF93E091BF02F091C0028081B4
:10E09000E091CA02F091CB02309709F00995FF9107
:10E0A000EF91BF91AF919F918F917F916F915F9110
:10E0B0004F913F912F910F900BBE0F900FBE0F907D
:10E0C0001F9018952DE0829FC0011124FC01EE5491
:10E0D000FD4FA281B3811C92A481B5816C93A6816E
:10E0E000B78188ED8C93A085B1854C9312861486F8
:10E0F000138608952DE0829FC0011124FC01EE5487
:10E10000FD4F81E08287A081B1816C933A96808136
:10E110008111FDCF08951F93CF93DF93182FEB014B
:10E12000FE019491992339F0FE016491812F0E94A0
:10E130007A702196F5CFDF91CF911F9108951F93AB
:10E14000CF93DF93182FEB019881992369F09A30D0
:10E1500021F46DE0812F0E947A7069916D30A1F3F6
:10E16000812F0E947A70F0CFDF91CF911F91089597
:10E17000CF93DF93CDB7DEB79E01285F3F4F4E812F
:10E180005F8160E470E08EE994E10E94D1A36EE9C2
:10E1900074E18D810E949F70DF91CF910895CF939C
:10E1A000C82F8A3031F46DE08091DE140E947A70BD
:10E1B00002C08D3029F06C2F8091DE140E947A709D
:10E1C00080E090E0CF9108952DE0829FC00111245E
:10E1D000FC01EE54FD4F748763870895682F80E03B
:10E1E0000C947A708093DE1484EA92E090932F3E30
:10E1F00080932E3E089584B7877F84BF0FB6F8942E
:10E20000A895809160008861809360001092600002
:10E210000FBE08959FE088E10FB6F894A89580930B
:10E2200060000FBE909360000895A89508950FB602
:10E23000F894A895809160008861809360001092A6
:10E2400060000FBE0895F89498E088E10FB6F89446
:10E25000A895809360000FBE90936000FFCF8091DF
:10E26000CD358091CD3590E0089540E06FE181E4B7
:10E2700091E00C949876E9E3F1E0808180818D7FD4
:10E2800080838DE090E00197F1F723E040E06FE1BB
:10E2900082E491E00E94A37683E090E00197F1F799
:10E2A00008959091390191FD0AC0282F803108F01E
:10E2B0002FE040E06FE085E491E00C94A3760895B0
:10E2C0008091390181FD0EC040E06FE181E491E071
:10E2D0000E949876282F2F7E81E090E0213021F057
:10E2E00080E0089580E090E008958091390181FFF9
:10E2F00002C081E0089540E06FE181E491E00E9476
:10E3000098768F3121F08F7E8150823090F780E0B7
:10E3100008950E9475718823E1F30895CF93DF93E8
:10E32000C82F0E9489710E943571D82FC81771F1CA
:10E33000C83019F40E943B7125C0C93121F48631DF
:10E3400089F429E005C0C63169F4893159F426E021
:10E3500040E06FE182E491E00E94A37683E090E0E8
:10E360000197F1F72C2F40E06FE182E491E00E94E9
:10E37000A376D83019F489E691E002C083E090E0FA
:10E380000197F1F70E9435718C1303C080E490E08F
:10E3900002C083E490E0DF91CF9108950E948971DB
:10E3A000109262370E943B718091390182608093A4
:10E3B00039018091E5378823D9F1809194009091BB
:10E3C00095004091F6375091F73784179507A0F4E0
:10E3D0008091C2379091C337A091C437B091C537AF
:10E3E0008C57914EAF4FBF4F8093C2379093C33736
:10E3F000A093C437B093C537209194003091950015
:10E40000241B350B8091C2379091C337A091C4373C
:10E41000B091C537820F931FA11DB11D8093C237E4
:10E420009093C337A093C437B093C5371092E537A4
:10E430008091E7378823D9F18091940090919500DD
:10E440004091FA375091FB3784179507A0F48091DB
:10E45000CA379091CB37A091CC37B091CD378C573C
:10E46000914EAF4FBF4F8093CA379093CB37A09355
:10E47000CC37B093CD372091940030919500241B78
:10E48000350B8091CA379091CB37A091CC37B091A2
:10E49000CD37820F931FA11DB11D8093CA37909372
:10E4A000CB37A093CC37B093CD371092E737089590
:10E4B00080916237882381F080916215882331F042
:10E4C00081E08093601581E090E008950E9475716D
:10E4D0008823B1F30E94CE7180E090E0089580918E
:10E4E0009400909195009093FB378093FA3781E0E8
:10E4F0008093E7379091390191FD08C080913901EF
:10E5000081FD1AC086E10E948E7116C0809361372A
:10E5100020919400309195003093F7372093F6378F
:10E520008093E537809139018D7F80933901809107
:10E5300061378111FCCFE2CF81E08093623708958B
:10E540008091623781110AC080916215882321F081
:10E5500081E08093611502C00E946F7281E090E0BB
:10E5600008951F93CF93DF931F92CDB7DEB78FB778
:10E5700089838091621581111FC0F8948091623760
:10E58000882351F08091390181FD14C00E9475717A
:10E59000882381F080E003C00E94A07281E0909106
:10E5A00047019E3088F4882351F01FEF0E94587273
:10E5B000107429F489818FBF80E090E009C08981BF
:10E5C0008FBF81E090E004C08823A1F310E0EECF7C
:10E5D0000F90DF91CF911F9108958091611588234D
:10E5E00021F00E946F72109261158091601588234E
:10E5F00021F00E94CE71109260151092621508955C
:10E600000F931F93AB0121E0209362150091A63771
:10E610001091A7372091A8373091A9370F5F1F4F6E
:10E620002F4F3F4F0093A6371093A7372093A8375B
:10E630003093A93722E0260F27FF0CC080915F3767
:10E640009091603701969093603780935F370FEF1A
:10E650001FEF07C0BC018FED94E10E943DA200E0D6
:10E6600010E00E94ED72C8011F910F9108958093F0
:10E67000641508950E943571823021F0823111F0C5
:10E6800081E0089580E0089508958FEF80934E0112
:10E6900022E044E060EF8CE691E00E94A37625E062
:10E6A00041E06EE08CE290E00E94A37680E88093E7
:10E6B0006F018091460180936D0121E045E060E2A9
:10E6C00084E491E00C94A376CF93DF93CDEFD3E075
:10E6D000CE010197F1F70E948E761092D6351092F6
:10E6E00058361092DA361092D5351092D435E9E3C7
:10E6F000F1E080818E7F808380818D7F80838DE0BB
:10E7000090E00197F1F780818160808323E040E011
:10E710006FE182E491E00E94A3762197F1F7809166
:10E720005D0180915E010E94457360E070E08CECB9
:10E7300092E00E940C5F0E946F7281E090E0DF9196
:10E74000CF910895809163150895CF93DF931F9221
:10E75000CDB7DEB789830E94897189818093631563
:10E76000282F40E06FE188E491E00F90DF91CF9196
:10E770000C94A3760E94A5738091390181FD03C09A
:10E7800086E00C948E710895FA0180936201909353
:10E79000630160936001709361013097C1F08081E3
:10E7A00080936B01818180936A01828180936901EA
:10E7B0008381809368018481809367018581809340
:10E7C0006601868180936501878180936401089545
:10E7D0008CEC92E00E942D5F81E08093CD3580919A
:10E7E000CE359091CF3501969093CF358093CE352D
:10E7F00081E090E008958091D53592E8899FF001FD
:10E800001124EA52FA4C10828F5F833018F48093FF
:10E81000D53502C01092D535E091D53582E8E89F14
:10E82000F0011124EA52FA4C808181110C94E873B2
:10E830001092CD3508951F93CF93DF932091D53556
:10E8400012E8129F90011124F901EA52FA4C40811A
:10E85000411103C00E94FB7392C05091390151FDD8
:10E860008EC050916237552309F489C047FF16C006
:10E870000E94FB738091963790919737A0919837BB
:10E88000B09199370196A11DB11D80939637909351
:10E890009737A0939837B093993771C04330B0F44D
:10E8A0000E94FB738091923790919337A091943797
:10E8B000B09195370196A11DB11D80939237909329
:10E8C0009337A0939437B093953759C050E0EA013D
:10E8D00022976C177D07B0F40E94FB7380918E37EE
:10E8E00090918F37A0919037B09191370196A11DEB
:10E8F000B11D80938E3790938F37A0939037B0934C
:10E9000091373DC0B90169527A4C0E943DA2E09115
:10E91000D5351E9FF0011124EA5AF94C808180936D
:10E92000C6350E94FB73809147018093C735909153
:10E93000CC35992311F0891710F48093CC35609170
:10E94000C73570E084E00E9498666091C63570E03B
:10E9500083E00E9498668091AA379091AB37A0918E
:10E96000AC37B091AD370196A11DB11D8093AA3788
:10E970009093AB37A093AC37B093AD3702C0C0E0F3
:10E98000D0E0CE01DF91CF911F910895CF93DF9317
:10E99000EC01888199810097E9F08730954021F05A
:10E9A0001982188283E026C06238C1F41092CD35F6
:10E9B0000E941F660E94846560E870E00E941B74DC
:10E9C000181619066CF40E947F65E0916103F091BE
:10E9D0006203099587E095E09983888381E00AC006
:10E9E0008091CA359091CB3501969093CB35809329
:10E9F000CA35F0CFDF91CF91089591E090936215E1
:10EA00000E9451710C94ED728091390181FD06C014
:10EA100040E06FE085E491E00C94987680E1089501
:10EA20000F931F93CF93DF93C82F81E080936215DC
:10EA3000D09162379091390191FF16C020919400D6
:10EA4000309195003093F7372093F6378093E53770
:10EA500080936137809139018D7F80933901809156
:10EA600061378111FCCFD0E00E94897180916237BB
:10EA7000882309F43FC08091E7378823D9F180913A
:10EA80009400909195004091FA375091FB3784178C
:10EA90009507A0F48091CA379091CB37A091CC37DD
:10EAA000B091CD378C57914EAF4FBF4F8093CA373F
:10EAB0009093CB37A093CC37B093CD37209194006F
:10EAC00030919500241B350B8091CA379091CB373C
:10EAD000A091CC37B091CD37820F931FA11DB11DEE
:10EAE0008093CA379093CB37A093CC37B093CD3770
:10EAF0001092E7378091390181FD03C089E10E94BE
:10EB00008E7186E00E94A366892B51F00E940475E5
:10EB1000082F86E00E94A36681500E94517102C0B6
:10EB200000E010E080919400909195009093F93767
:10EB30008093F83781E08093E637F894809139012B
:10EB4000826080933901809139018D7F80933901F2
:10EB500062E06C0F8FED94E10E94D37678948091FF
:10EB60005C3790915D37019690935D3780935C3769
:10EB70000E94897145E060EE82E491E00E949876FF
:10EB8000C82F86E00E94A366892B19F0802F0E946F
:10EB90005171DD2319F00E946F7202C00E94CE7184
:10EBA0008091E6378823D9F1809194009091950067
:10EBB0004091F8375091F93784179507A0F4809168
:10EBC000C6379091C737A091C837B091C9378C57D5
:10EBD000914EAF4FBF4F8093C6379093C737A093E6
:10EBE000C837B093C9372091940030919500241B09
:10EBF000350B8091C6379091C737A091C837B09137
:10EC0000C937820F931FA11DB11D8093C637909302
:10EC1000C737A093C837B093C9371092E6378091B1
:10EC20006237882361F080919400909195009093D1
:10EC3000FB378093FA3781E08093E73707C023E002
:10EC400040E06FE182E491E00E94A3760E94ED72C1
:10EC5000C130E9F0C330A9F480919E3790919F377D
:10EC6000A091A037B091A1370196A11DB11D80934D
:10EC70009E3790939F37A093A037B093A137C2E0FF
:10EC800009C0C53031F0C73029F4C1E003C0C0E08D
:10EC900001C0C3E08C2F90E0DF91CF911F910F91C5
:10ECA0000895CF93DF93EB010E940073009729F43E
:10ECB000CE010E941075009751F020915F3730917E
:10ECC00060372F5F3F4F3093603720935F37DF917E
:10ECD000CF910895CF93DF9380916237811104C063
:10ECE0000E94A072D1E001C0D0E00E94357186314F
:10ECF00011F0813119F4C091470109C040E06FE182
:10ED000086E491E00E949876C82FCC0FC80FD111ED
:10ED10000E9458728C2FDF91CF9108951092661542
:10ED200010926515EFE6F0E080818062808308959F
:10ED3000FC0180816823862F90E002C0959587951D
:10ED40004A95E2F70895FC01922FF8942081362F1E
:10ED50003095522F5323292F01C0220F4A95EAF7ED
:10ED60002623252B208378940895CF93DF93E09179
:10ED70007B01EC01E993A0E8B1E020E82E0F3C9183
:10ED8000399311962A13FBCFE150F0E0E058FE4F83
:10ED90002181FC01E058FF4F2083319681E0808380
:10EDA000DF91CF91089560938001E1E8F1E061582F
:10EDB000DC012D91CD01208331966E13F9CF08959A
:10EDC0001F920F920FB60F9211240BB60F922F9332
:10EDD0003F934F935F936F937F938F939F93AF93E3
:10EDE000BF93EF93FF93809147018093C735809144
:10EDF000D43522E8829FC00111248A529A4C0E9485
:10EE0000B5768091D4358F5F833018F48093D435F4
:10EE100002C01092D4350E94E873FF91EF91BF9128
:10EE2000AF919F918F917F916F915F914F913F91A2
:10EE30002F910F900BBE0F900FBE0F901F90189543
:10EE40001F920F920FB60F9211240F900FBE0F90CA
:10EE50001F9018951F920F920FB60F9211240F90CA
:10EE60000FBE0F901F9018951F920F920FB60F9222
:10EE700011240F900FBE0F901F9018951F920F92A4
:10EE80000FB60F921124109261370F900FBE0F90A2
:10EE90001F9018951F920F920FB60F921124109287
:10EEA00061370F900FBE0F901F9018951F920F9211
:10EEB0000FB60F9211248F9381E08093CD358F91FF
:10EEC0000F900FBE0F901F9018951F920F920FB6C4
:10EED0000F921124109261370F900FBE0F901F9068
:10EEE00018951F920F920FB60F9211248F939F9334
:10EEF00080916515909166150196909366158093A3
:10EF000065159F918F910F900FBE0F901F901895D0
:10EF10008F929F92AF92BF92CF92DF92EF92FF9229
:10EF2000E7E6F5E1408151814A01A12CB12C6B014A
:10EF30007C0124E0F594E794D794C7942A95D1F7FF
:10EF4000C818D908EA08FB08DC01CB0133E0B59505
:10EF5000A795979587953A95D1F7B501A401440FE8
:10EF6000551F661F771F4C015D01841A950AA60A7A
:10EF7000B70AA5019401A281B3810E94989C4B011C
:10EF80005C013BE0B594A794979487943A95D1F7A8
:10EF9000A7019601C701B6010E94DA9B9B01AC0153
:10EFA0006CE055954795379527956A95D1F7A481DB
:10EFB000B5810E94989CDC01CB017EE0B595A795B8
:10EFC000979587957A95D1F7A5019401280F391F58
:10EFD0004A1F5B1F21A332A343A354A3A5E0B0E0C3
:10EFE0000E948D9CDC01CB0180589F4FAF4FBF4FDB
:10EFF000692F7A2F8B2F992787FD9A95FF90EF9095
:10F00000DF90CF90BF90AF909F908F900895EF9238
:10F01000FF921F93CF93DF93CDB7DEB76A970FB6FA
:10F02000F894DEBF0FBECDBF182F21E030E0CE0137
:10F0300001967C01AC0160ED70E08EEE90E00E94E4
:10F040008B128981803609F0CAC046EB50E060EE31
:10F0500070E08EEE90E00E9474126CE17AE186E03E
:10F0600090E00E94116A8AE1F70111928A95E9F70E
:10F070002AE130E0A70168E870E08EEE90E00E949F
:10F080008B128A8190E0982F88272981822B909378
:10F090006815809367158C8190E0982F88272B81C5
:10F0A000822B90936A15809369158E8190E0982F3A
:10F0B00088272D81822B90936C1580936B15888502
:10F0C00090E0982F88272F81822B90936E15809344
:10F0D0006D158A8590E0982F88272985822B90933B
:10F0E000701580936F158C8590E0982F88272B855D
:10F0F000822B90937215809371158E8590E0982FD6
:10F1000088272D85822B9093741580937315888999
:10F1100090E0982F88272F85822B909376158093E7
:10F1200075158A8990E0982F88272989822B9093DA
:10F130007815809377158C8990E0982F88272B89F4
:10F14000822B90937A15809379158E8990E0982F71
:10F1500088272D89822B90937C1580937B15288D91
:10F1600030E0322F22278F89282B30937E15209371
:10F170007D158A8D80937F1528E030E0A70161EE30
:10F1800070E08EEE90E00E948B122A8130E0322FE8
:10F1900022278981282B30938115209380158B811C
:10F1A000809382158C81F0E18F9FC00111242D8105
:10F1B0002F70822B90938415809383158F8120E18B
:10F1C000829FC00111242E812F70822B909386156F
:10F1D0008093851588858093871510938C156A9682
:10F1E0000FB6F894DEBF0FBECDBFDF91CF911F9158
:10F1F000FF90EF9008952F923F924F925F926F92FF
:10F200007F928F929F92AF92BF92CF92DF92EF92B6
:10F21000FF920F931F93CF93DF93CDB7DEB7AD97D8
:10F220000FB6F894DEBF0FBECDBF9E012F5F3F4FDC
:10F23000790198E0F90111929A95E9F7813009F086
:10F2400077C380918C15813009F072C341E050E0A2
:10F2500062EF70E08EEE90E00E94741240E050E0A9
:10F2600065EF70E08EEE90E00E94741246E250E08E
:10F2700064EF70E08EEE90E00E9474120CE211E0F8
:10F2800021E030E0AE01475F5F4F64EF70E08EEE4B
:10F2900090E00E948B12898583708987882351F0C2
:10F2A00065E375E080E090E00E94116A0150110969
:10F2B00039F73EC328E030E0A70167EF70E08EEE3B
:10F2C00090E00E948B12E981E8A7FA81F9A72B81CF
:10F2D0002AA7CF80D12CE12CF12CFE2CED2CDC2C9C
:10F2E000CC248885C82A6D81862F90E0A0E0B0E00C
:10F2F000AC01BD01E4E0440F551F661F771FEA957E
:10F30000D1F78C8190E0A0E0B0E0FCE0880F991F7D
:10F31000AA1FBB1FFA95D1F7842B952BA62BB72BD1
:10F320002E8122952F70BC01CD01622B0E9488771F
:10F33000609366357093673580936835909369352F
:10F340008090881590908915A0908A15B0908B15A3
:10F35000240135013CE2531A31E0630A7108AEE042
:10F36000CC0CDD1CEE1CFF1CAA95D1F780918315F7
:10F3700090918415092E000CAA0BBB0B14E1880F89
:10F38000991FAA1FBB1F1A95D1F7C81AD90AEA0AF2
:10F39000FB0AA0918515B0918615A30192010E94E8
:10F3A000989CC61AD70AE80AF90A40E4D40EE11C70
:10F3B000F11C0FE0F594E794D794C7940A95D1F720
:10F3C000A09187150A2E000CBB0BA30192010E948D
:10F3D000989C9B01AC018AE05595479537952795F8
:10F3E0008A95D1F72A873B874C875D87A091821544
:10F3F000B0E0A30192010E948D9CDC01CB012BE0C7
:10F40000B595A795979587952A95D1F7BC01CD011C
:10F4100070588F4F9F4F2A853B854C855D850E9494
:10F42000DA9BDC01CB013AE0B595A79597958795D6
:10F430003A95D1F79C01AD01405E5F4FA0918015D8
:10F44000B09181150E94989CDC01CB01905EAF4F7A
:10F45000BF4FBC01CD014EE0959587957795679597
:10F460004A95D1F7A70196010E94DA9B6B017C01B6
:10F470005FE095958795779567955A95D1F79B01AC
:10F48000AC010E94DA9B9B01AC0167E05595479562
:10F49000379527956A95D1F7A0917F15B0E00E9426
:10F4A0008D9CDC01CB0174E0B595A7959795879568
:10F4B0007A95D1F7A7019601281B390B4A0B5B0BF4
:10F4C000DA01C90157FF03C080E090E0DC01813020
:10F4D0009105A10539E1B30724F080E090E0A0E0B8
:10F4E000B9E12CE0B595A795979587952A95D1F721
:10F4F00080936A3590936B35A0936C35B0936D35DE
:10F5000075016401FF0CCC08DC2C76019401A50187
:10F510006C2D7C2D8C2D9C2D345F4140510961094F
:10F520007109810991092A873E874F87588B698B1A
:10F530007A8B8B8B9C8B59016A017B018C010E9419
:10F54000A09C28A339A34AA35BA36CA37DA38EA38D
:10F550009FA3409177154BA7509178155D8B8091B3
:10F5600075158CA7E0917615EE8BF0917315FDA7BC
:10F57000209174152F8BB0907015A0906F151B2DD6
:10F58000110F110BC12ED12EE12EF12E012F2A8544
:10F590003E854F85588969897A898B899C890E9423
:10F5A000A09C0CE00E94FB9D19012A013B014C012B
:10F5B000B0907215A09071151B2D110F110BC12E5B
:10F5C000D12EE12EF12E012F28A139A14AA15BA154
:10F5D0006CA17DA18EA19FA10E94A09C08E00E9429
:10F5E000149E51016201730184010E94329E705881
:10F5F0008F4F9F4F20906D1530906E155101C12C8B
:10F60000D12CE12CF12C00E010E00E94A09C01E242
:10F610000E94149E288F398F4A8F5B8F6C8F7D8F4D
:10F620008E8F9F8FA0E00E94599E09F475C1ABA4F4
:10F630001D89110F110BBD88C12ED12EE12EF12E87
:10F64000012F28A139A14AA15BA16CA17DA18EA1A6
:10F650009FA10E94A09C19012A013B014C01ACA46E
:10F660001E89110F110BBE88C12ED12EE12EF12E55
:10F67000012F2A853E854F85588969897A898B892A
:10F680009C890E94A09C01E10E94FB9D59016A0196
:10F690007B018C019101A201B301C4010E94329E41
:10F6A00019012A013B014C01F9A54F2F50E060E000
:10F6B00070E0E4E0440F551F661F771FEA95D1F70D
:10F6C0008AA582958F708A019B01082B88A5482FF7
:10F6D00050E060E070E0DB01CA01FCE0880F991F98
:10F6E000AA1FBB1FFA95D1F7B901A801482B592BC6
:10F6F0006A2B7B2B80E090E0A0E1B0E0841B950BAF
:10F70000A60BB70B6C017D01FF0CCC08DC2C76013D
:10F710009C01AD016C2D7C2D8C2D9C2D0FE10E9448
:10F72000FB9DB22FA32FF42FE52F6A877E878F874B
:10F73000988B2DA59F89990F990B3F89492F592F98
:10F74000692F792F892F03E20E94FB9D59016A01DD
:10F750007B018C019101A201B301C4010E94329E80
:10F7600059016A017B018C012B2F3A2F4F2F5E2FFD
:10F770006A857E858F8598890E94479E39014A0156
:10F78000B62FA72FF82FE92F03E00E94FB9D53010E
:10F790006401EB2EFA2E0F2F1E2F0E94479E590157
:10F7A0006A017B01582E192F03E00E94FB9D052D55
:10F7B0000E94479E03E00E94FB9D53016401EB2ED3
:10F7C000FA2E0F2F1E2F0E94479E02E00E94FB9DE3
:10F7D0000F2F0E94479E01E00E94FB9D0F2F0E9469
:10F7E000479EA88CB98CCA8CDB8CEC8CFD8C0E8D62
:10F7F0001F8D0E94269D2A873E874F87588B698BD5
:10F800007A8B8B8B9C8B0DE00E94149E922E832E04
:10F81000742E652E562E472E382E292E30917E15A9
:10F8200020917D15932F990F990BA92CB82CC72CDB
:10F83000D62CE52CF42C032D122D492F592F692F8E
:10F84000792F892F0E94A09C0E94A09C09E10E9410
:10F85000149E59016A017B018C012A853E854F85E2
:10F86000588969897A898B899C890E94329E1901FD
:10F870002A013B014C0130917C1520917B15932F7F
:10F88000990F990BAA84BE84CF84D888E988FA8816
:10F890000B891C89492F592F692F792F892F0E9495
:10F8A000A09C03E10E94149E59016A017B018C0116
:10F8B0009101A201B301C4010E94329E08E00E949E
:10F8C000149E322E432E542E652E762E872E982E81
:10F8D000B92F30917A1520917915932F990F990BA3
:10F8E000492F592F692F792F892F04E00E94FB9D02
:10F8F00059016A017B018C01232D342D452D562D94
:10F90000672D782D892D9B2F0E94329E722F632F99
:10F91000942F852F9B0104C030E020E090E080E030
:10F9200030936E3520936F35909370358093713599
:10F93000AD960FB6F894DEBF0FBECDBFDF91CF916D
:10F940001F910F91FF90EF90DF90CF90BF90AF90FD
:10F950009F908F907F906F905F904F903F902F90EF
:10F960000895CF92DF92EF92FF920F931F93CF9360
:10F97000DF937C018B016A018DE895E10E94CD5FE8
:10F98000EC01892B51F0EC81FD81309711F0C80119
:10F990000995CE010E947960F3CFA601B801C70195
:10F9A000DF91CF911F910F91FF90EF90DF90CF905B
:10F9B0000C94525D0F931F93CF93DF9300D0CDB77C
:10F9C000DEB780916A3790916B37A0916C37B09118
:10F9D0006D370196A11DB11D80936A3790936B37E7
:10F9E000A0936C37B0936D370E94417F8C018DE8F6
:10F9F00095E10E94CD5F009779F0DC011296ED91C0
:10FA0000FC911397309729F089839A8309959A81FD
:10FA100089810E947960EFCF0115110549F0C80175
:10FA20000F900F90DF91CF911F910F910C94495D32
:10FA30000F900F90DF91CF911F910F9108950E9429
:10FA40002C840E941F660E946B7D8DE493E090934E
:10FA50006537809364370E943F7F2FEF31E040E0AD
:10FA60005EE160E074E082E090E00C940C7FBC0109
:10FA70008DE895E10C943160BC018DE895E10C9422
:10FA80001260CF93DF93EC01409166375091673756
:10FA900060916837709169374F5F5F4F6F4F7F4F4D
:10FAA0004093663750936737609368377093693730
:10FAB0000E94547F009761F00E949D65E091510380
:10FAC000F0915203BE0181EB9CE7099581E090E043
:10FAD000DF91CF91089583E995E10C94C95F0F936D
:10FAE000CF93DF93EC017B836A8318865F834E8319
:10FAF000BC0183E995E10E943160E0918F15F0919E
:10FB00009015309749F04C815D8101E020E030E0B4
:10FB100068858A819B810995DF91CF910F91089526
:10FB2000BC0183E995E10C9412600F93FC011086EF
:10FB3000E0918F15F0919015309761F0DC0100E0B5
:10FB400020E030E040E050E060E012968D919C9122
:10FB5000139709950F9108950F93DC0114962D9139
:10FB60003C91159781E018968C93189715967C9385
:10FB70006E931497E0918F15F0919015309741F0A6
:10FB8000AB0100E061E012968D919C91139709956D
:10FB90000F9108950F93E0918F15F0919015309784
:10FBA00079F0DC0114964D915C91159701E09A0172
:10FBB00018966C91189712968D919C9113970995B0
:10FBC0000F910895E0919115F0919215309709F0F9
:10FBD00009940895909392158093911508959093A8
:10FBE000901580938F15089583E995E10C94CD5F6E
:10FBF000EF92FF920F931F93CF93DF938C01EB0152
:10FC00007A0183E995E10E94CD5F0097D9F0DC018C
:10FC100012962D913C9113972C173D0781F416965F
:10FC2000ED91FC911797309769F09701AE01B801FB
:10FC3000DF91CF911F910F91FF90EF9009940E9457
:10FC40007960E3CFDF91CF911F910F91FF90EF90FB
:10FC500008950895CF93DF93C5E9D5E169A97AA9FD
:10FC600020E030E049E45EE780EB95E10E945162DC
:10FC70000E942A8469A97AA90E94F69B20E030E0BC
:10FC80004DE55EE7BC0180EA95E1DF91CF910C94F0
:10FC900051628091C6159091C7152091C41530917D
:10FCA000C515880F991F2817390708F4C9019093C3
:10FCB000C7158093C6150C942A7ECF93DF930E94BC
:10FCC0001F660E948465EC01198218820E94F47DEF
:10FCD00028813981009719F1FC0140854423F9F00E
:10FCE000FC0142815381F901EE0FFF1FEE0FFF1F50
:10FCF000EC0FFD1F53834283FC01448155812F5F2C
:10FD00003F4FF901EE0FFF1FEE0FFF1FEC0FFD1F1E
:10FD100051834083398328830E947960D9CFC901F8
:10FD2000880F991F880F991F02960E947F6588810E
:10FD30009981892B31F085E995E1DF91CF910C9480
:10FD40001F5DDF91CF910895AF92BF92CF92DF9266
:10FD5000EF92FF920F931F93CF93DF9300D0CDB715
:10FD6000DEB76B010E948465FC01E080F180FA82BD
:10FD7000E982FCE0EF16F10418F400E010E00DC099
:10FD8000FF92EF928BE99AE09F938F930E94F8A2E3
:10FD90000F900F900F900F9022C00E151F05F9F0D5
:10FDA0000E9484659801220F331F220F331F820F98
:10FDB000931FFC01A280B3800E9484650F5F1F4FD8
:10FDC0009801220F331F220F331F820F931FFC0154
:10FDD00040815181B501C6010E94F87DDECF0F90B0
:10FDE0000F90DF91CF911F910F91FF90EF90DF90D7
:10FDF000CF90BF90AF9008950F93013059F4809148
:10FE0000C0159091C1159093C7158093C6150F9199
:10FE10000C942A7E0F910895EF92FF920F931F93F7
:10FE2000CF93DF937B018A01E9014AE353E0BC01F0
:10FE300085E995E10E94025DE5E9F5E1F4A6E3A616
:10FE400016A705A7D0ABC7A78CEF9EE7DF91CF9190
:10FE50001F910F91FF90EF900C94EF7D80EB95E157
:10FE60000E94D56280EA95E10E94D56285E995E11C
:10FE70000C941D5D8091C6159091C71508950C9442
:10FE80005E5DCF93DF93E0913E03F0913F030995D0
:10FE9000EC01892B29F06A817B8181E00E949866C0
:10FEA000CE01DF91CF9108950F931F93CF93DF93EE
:10FEB000EC01E0914003F091410309958C016A81C6
:10FEC0007B8181E00E94986681E090E0012B11F433
:10FED00080E090E0DF91CF911F910F910895E09124
:10FEE0004203F0914303099420E030E00296FC01C4
:10FEF00032974081442331F0FC0131974081240F37
:10FF0000311DF4CFC9010895FC01208130E0322F6A
:10FF100022278181282B02C0220F331F6A95E2F726
:10FF2000232F3327FA01EC5BFC4F808190E0822382
:10FF3000932328E030E0241B350B02C0969587956B
:10FF40002A95E2F708956F927F928F929F92AF92D7
:10FF5000BF92CF92DF92EF92FF920F931F93CF93B6
:10FF6000DF937C018B015A01E9012830310544F40B
:10FF7000A901B501C8010E94847FF701808346C0B2
:10FF8000690183E0D594C7948A95E1F7452B21F068
:10FF90004701612C712C06C0FB01D701CB018C0DF0
:10FFA0009D1D1FC048E050E0B501C801860D971D9A
:10FFB0000E94847FF40181934F01FFEF6F1A7F0A43
:10FFC0006C147D0479F7AE01477055274115510532
:10FFD000E9F0E701C60DD71DB501C801860D971DD3
:10FFE00012C0E817F90719F021912D93FACFAE014D
:10FFF000477055274115510549F0E701CC0DDD1D2E
:020000021000EC
:1000000060E070E0CF010E94847F8883DF91CF9110
:100010001F910F91FF90EF90DF90CF90BF90AF9026
:100020009F908F907F906F9008958F929F92AF9244
:10003000BF92CF92DF92EF92FF920F931F93CF93D5
:10004000DF9300D0CDB7DEB70E9484658C0182E0DB
:1000500090E00E946265892B19F480E090E05FC017
:10006000F801218130E0322F22278081A901480F39
:10007000511DCA010E946F5D7C01892B71F30E94A2
:1000800084654C01F7019681292F269526952695A2
:1000900030E0977041E050E011F440E050E0C901D9
:1000A000840F951F0E946265892BB9F2F7010481C4
:1000B0001581A12CB12CF8018081882379F1F801F8
:1000C000C180D12CA50147705527B50193E07595E6
:1000D00067959A95E1F7680D791D883168F096016A
:1000E000CE0101960E94A37FBE016F5F7F4FF80192
:1000F00080810E94AC660DC01A8219829601CE01E1
:1001000001960E94A37F69817A81F80180810E9413
:100110009866AC0CBD1C0E5F1F4FCDCFC7010F9072
:100120000F90DF91CF911F910F91FF90EF90DF9093
:10013000CF90BF90AF909F908F900895DC0150E0DA
:10014000E0E1F0E0CF01861B970B821B930B02C00E
:10015000440F551F8A95E2F78C91852B8C9311964D
:100160008C911197482B11964C9308956F927F9222
:100170008F929F92AF92BF92CF92DF92EF92FF92B7
:100180000F931F93CF93DF93283031051CF4FA01AE
:1001900040815AC05901E3E0B594A794EA95E1F78C
:1001A0006115710541F03901EA018B017C014A01B9
:1001B000C12CD12C05C0EA01FC014A0D5B1D2AC0EF
:1001C000F40141914F0128E030E0B801C7018C0DE6
:1001D0009D1D0E949E80FFEFCF1ADF0ACA14DB0428
:1001E00079F793012770332721153105E9F1CC0DFB
:1001F000DD1D488150E0021B130B085F1F4F02C03A
:10020000559547950A95E2F760E070E0C7018C0DBF
:100210009D1D1AC0C417D50719F069916193FACFD3
:100220002770332721153105F9F0488150E068E047
:1002300070E0621B730B02C0559547956A95E2F713
:1002400060E070E08A0D9B1DDF91CF911F910F91AF
:10025000FF90EF90DF90CF90BF90AF909F908F90E6
:100260007F906F900C949E80DF91CF911F910F91A2
:10027000FF90EF90DF90CF90BF90AF909F908F90C6
:100280007F906F9008956F927F928F929F92AF921E
:10029000BF92CF92DF92EF92FF920F931F93CF9373
:1002A000DF9300D0CDB7DEB77C01FC018681082F3B
:1002B000069506950695202F30E0877001E010E046
:1002C00011F400E010E0020F131FC80102960E9413
:1002D000E865009709F448C00E948B65F701228108
:1002E000FC012083F7012381FC0121830E948B659F
:1002F00002965C01A80160E070E00E9446A2F7014E
:10030000048115810F5F1F4F812C912CF8013197CB
:100310008081882339F1F801C080D12C3401F7E0C5
:100320006F227724740193E0F594E7949A95E1F7AE
:10033000EA0CFB1C883128F00E94B6669601AC01DD
:1003400008C00E94A3669A8389839601AE014F5F1D
:100350005F4FB301C7010E94B6808C0C9D1C0E5FDD
:100360001F4FD4CF81E090E00F900F90DF91CF919D
:100370001F910F91FF90EF90DF90CF90BF90AF90C3
:100380009F908F907F906F900895E0915F03F09120
:1003900060030994E0913803F09139030994E091E6
:1003A0006303F09164030994E0916503F09166039F
:1003B000099480E090E008950895E0913003F09171
:1003C0003103099480E090E008950F931F93CF9339
:1003D000DF93CDB7DEB7E0970FB6F894DEBF0FBE60
:1003E000CDBF0E94D1658C010E948465AE014F5F34
:1003F0005F4F602F0E94B089882309F442C088A90A
:100400009801281B3109C9010E946265892BC9F135
:100410008E8181110CC0BE016A5E7F4F88E10E940F
:10042000AC66E0915303F091540309952AC02A85E4
:100430003B852D3C9BEA390719F02F3F3F4F09F5CB
:10044000823019F088E090E002C082E090E00197ED
:1004500010F3E1E0F0E0EC0FFD1FE80FF91F23853A
:100460002F3FA9F3BE01645F7F4F89E10E94AC6614
:1004700089E10E94B66667E775E30E94BB5C892B41
:1004800051F6E0960FB6F894DEBF0FBECDBFDF91F8
:10049000CF911F910F910895AF92BF92CF92DF92AB
:1004A000EF92FF920F931F93CF93DF93CDB7DEB7F9
:1004B000E0970FB6F894DEBF0FBECDBF8C016B0185
:1004C000CE0101967C0180E3F70111928A95E9F74C
:1004D00081E089838CE00E94A3668C831D821F8249
:1004E0008091CA1591E0980F9093CA15898783E08F
:1004F000B82EB8868DEC9BEA9B878A8789E10E949B
:10050000B6666CE073E00E94BB5C892B31F082E040
:100510008E838FEF8C878D8709C089E10E94B66634
:10052000BC01CE010C960E94B25CBE828DEC9BEAAF
:100530009D8B8C8B67E775E3CE0146960E94B25C7B
:100540000E9484659FA78EA70E94D16588ABC701D2
:100550000E94B088B82E90E00E94E865892B31F1A6
:100560000E948B654B2DBC01C7010E94CE88E09094
:100570002603F09027030E94DB655C010E948B65D7
:10058000B501F70109950115110581F0009739F0C2
:10059000019761F441E050E064E070E004C041E0A4
:1005A00050E060E070E0C601F8010995E0960FB6F2
:1005B000F894DEBF0FBECDBFDF91CF911F910F9199
:1005C000FF90EF90DF90CF90BF90AF9008950E9482
:1005D0002A848093CA15E0913003F0913103099485
:1005E000892B29F0E0913003F091310304C0E091B0
:1005F0003203F09133030994CF93DF93EC01899197
:100600009991009729F060E070E00E940C5FF7CFAD
:10061000DF91CF910895CF93DF93EC018991999168
:10062000009719F00E945C5EF9CFDF91CF91089599
:10063000CF93DF93EC017B836A830E94A06F998341
:100640008883DF91CF910895FC01208131818281DF
:100650009381820F931F918380830895CF93DF93BB
:10066000EC010E94A06F99838883DF91CF91089558
:10067000CF93DF93EC010E94A06F28813981821B08
:10068000930B9C012F5F3F4F81E090E04A815B819B
:100690004217530710F080E090E0DF91CF9108956A
:1006A000CF93DF93FC01C281D38180819181C80FF8
:1006B000D91F0E94A06F9E01281B390BC901DF9131
:1006C000CF910895CF93DF93ECEEF7E3CEEAD7E333
:1006D000A0EEB7E311921192199219921992199200
:1006E0001D9288E3E430F807A9F7DF91CF910895D0
:1006F000CF93DF93FC01E052F84C40819C01220F24
:10070000331F220F331F4423F9F04091940050917E
:100710009500E901C255D84C880F991FFC01E4519E
:10072000F84C80819181BA01681B790B888199818D
:10073000AA81BB81860F971FA11DB11D8883998354
:10074000AA83BB8351834083F901E255F84C608151
:10075000718182819381DF91CF91089560E070E093
:10076000CB010895880F991F880F991FFC01E2554E
:10077000F84C40835183628373830895CF93DF9352
:10078000C0EED7E3EEEAF7E3ACEEB7E38991882356
:10079000D1F080919400909195002D913C9111970A
:1007A000AC01421B530B9A014081518162817381DC
:1007B000420F531F611D711D4083518362837383F8
:1007C00011969C938E933496129657E3EE3DF5075F
:1007D000E9F6DF91CF9108950C9442880F931F930F
:1007E000FC018091CB159091CC1533832283158326
:1007F000048371836083F093CC15E093CB15892B30
:1008000019F4CB010E945C8880E090E01F910F9169
:1008100008958091CB159091CC150097C1F010925E
:10082000CC151092CB15DC0114966D917C91159727
:100830001296ED91FC9113970995E091CB15F091EB
:10084000CC15309721F0808191810C945C880895BB
:100850000C94B49E0C94B09E8EED92E00E94435F87
:1008600086ED92E00C94435FCF93DF930E949165F5
:10087000892BA9F086ED92E00E94615FEC01892B43
:1008800021F10E94D165998388830E94CC659B8366
:100890008A83CE0104960E940D658CAB14C08EED48
:1008A00092E00E94615FEC01009779F002960E944D
:1008B0001F6599838883BE016E547F4FCE018E578A
:1008C0009F4F0E947666CE0102C080E090E0DF91EB
:1008D000CF910895BC016E547F4F8E579F4F0C945B
:1008E0007666CF93DF93EC01BC018EED92E00E941F
:1008F000AC5FBE01892B19F08EED92E009C086ED48
:1009000092E00E94AC5F892B39F0BE0186ED92E047
:10091000DF91CF910C94865FDF91CF9108950F9373
:100920001F93CF93DF93EC01BC018EED92E00E9408
:10093000AC5F892B91F0FE0161917191CF010E9412
:100940003266BE016E547F4FCE018E579F4FDF91AE
:10095000CF911F910F910C948766BE0186ED92E0B6
:100960000E94AC5F892BD1F00E941F66688179815B
:100970008A819B810E9432668CA990E00E94E86582
:100980000CA910E00E948B65BE016C5F7F4FA8012F
:10099000DF91CF911F910F910C943DA2DF91CF91E8
:1009A0001F910F910895CF93DF93EC01BC018EED61
:1009B00092E00E94AC5F892B19F0CE0102960CC028
:1009C000BE0186ED92E00E94AC5F892B19F08A810E
:1009D0009B8102C080E090E0DF91CF910895FC01FF
:1009E000808191810895860F911D860F911D8E57EC
:1009F0009F4F0895860F911D860F911DFC01EE57A4
:100A0000FF4F80819181089508958AE29CE10E94C0
:100A10008A61892B21F08AE29CE10C947761089528
:100A2000E091161CF091171C309709F0099480E0B2
:100A30000895EF92FF920F931F93CF93DF938C0152
:100A4000EA01FC0180819181009741F08C30934054
:100A500071F1F8011182108283E0F6C080E024E099
:100A6000829FF0011124E85EF34E118210828F5FA5
:100A70008430A9F78093151C80912A1390912B1331
:100A80009093291C8093281C0E94555E8093043803
:100A900060E470E08AE29CE10E9463610E941D8B29
:100AA0008CE093E0F8019183808381E0CDC06230D7
:100AB000D9F48091053890910638892B89F380917B
:100AC0001638863029F480912E3881FD0E940585E4
:100AD00081E00E94728C8091053890910638892BB4
:100AE000F9F20E943287DCCF633060F5611114C0E7
:100AF0002097B1F2D093133DC093123D83E00E9442
:100B0000728C8091053890910638892B11F00E94E3
:100B100010850E940585C4CF613011F6209709F435
:100B2000BFCFD0930F3DC0930E3D85E00E94728CE5
:100B30008091053890910638892B09F4B1CF0E9435
:100B40001085AECF673809F040C01092141C88E1C0
:100B5000E82E8CE1F82E8091141C8430C0F4F7014B
:100B6000828193818C179D0749F4808191810E9435
:100B70003D8CF7011182108213821282F4E0EF0E95
:100B8000F11C8091141C8F5F8093141CE4CFEDE264
:100B9000FDE3838194818C179D0719F414821382DD
:100BA0001082B0962DE3ED3AF20799F7EAEAFDE3F9
:100BB000818592858C179D0711F4158214823D96CC
:100BC0008EE3EC32F807A1F76BCF683809F068CFF5
:100BD000CA52DC4109F064CF8AE29CE10E948A613A
:100BE000892B09F45DCF1092141CE091141CE430A1
:100BF00008F056CF20E2E29FF0011124EC5EF24CA7
:100C0000818D8823D9F08AE29CE10E9477618091EE
:100C1000141CE0E28E9FC00111248C5E924C9093D4
:100C2000133D8093123D82E00E94728C80910538C2
:100C300090910638892B11F00E9410858091141C28
:100C40008F5F8093141CD1CFDF91CF911F910F91B3
:100C5000FF90EF9008959093171C8093161C0895B1
:100C60009C0140912A1350912B1390E0E8E1FCE1A4
:100C70009430A1F0608171816217730761F4628121
:100C800073816417750739F49093131C11821082D5
:100C9000C9010C943D8C34969F5FEACF9093131C4E
:100CA00008959C0190E0E8E1FCE19430B1F081E02E
:100CB000890F40815181452B69F49093121C318337
:100CC000208380912A1390912B1393838283C901EF
:100CD0000C94588C3496982FE8CF9093121C08955A
:100CE00020912A1330912B13FC01358F248F778F9D
:100CF000668F089520912A1330912B13FC013287BF
:100D00002187748763870895CF93DF93EA010E9458
:100D1000CC8B009749F020912A1330912B13FC01C2
:100D200032872187D487C387DF91CF9108950F93AE
:100D30001F93CF93DF9300D000D0CDB7DEB78C01E7
:100D4000AB019FEF99839A839B839C83B801CE016B
:100D500001960E948486009719F0FC011583048394
:100D60000F900F900F900F90DF91CF911F910F91E7
:100D7000089540E050E062E086EE92E00E94FD5E61
:100D800010920638109205380895AC0161E086EEA5
:100D900092E00C94DE5EAC0160E086EE92E00C9492
:100DA000DE5E0F931F93CF93DF938A010E94498BDE
:100DB000EC01892B59F080912A1390912B139D8F70
:100DC0008C8F1F8F0E8FCE010E94CB86CE01DF91BC
:100DD000CF911F910F910895CF93DF93A091123D72
:100DE000B091133D109719F0ED016C9605C0C091BC
:100DF0000E3DD0910F3D299680910D3D86FF23C079
:100E00001092111C80E0E8E1FCE18430C1F04081E7
:100E1000518114962D913C9115974217530761F417
:100E2000228133812115310539F08093111C3983DA
:100E300028831B821A8205C034968F5FE6CF809389
:100E4000111C0E94058588819981009741F04A8193
:100E50005B8160910438DF91CF910C94FD5EDF914E
:100E6000CF9108950F931F93CF93DF9380911638FE
:100E7000863009F071C0809105389091063881154F
:100E8000954009F069C004E912E010930638009318
:100E90000538D2E0D0930F38C4E9C09310381092CF
:100EA0003238109231380E94178B8095909590932C
:100EB00032388093313810921838109217380E94C7
:100EC000068B8095909590931838809317380E94E0
:100ED00010851093063800930538D0930F38C093CF
:100EE0001038A091103DB091113DFD01E459FD4F26
:100EF0008CE692E001900D920197E1F76CE672E0CA
:100F000085E298E30E94C68A80910938809325384B
:100F100080910A388093263880910B388093273847
:100F200080910C38809328381092323810923138E2
:100F30000E94178B8095909590933238809331382A
:100F400010921838109217380E94068B8095909551
:100F50009093183880931738DF91CF911F910F919C
:100F60000C941085FC01680F791F80E048E1E617BA
:100F7000F70781F0219198E0322F3827532F5170D5
:100F800030FD84278695513009F48068269591506C
:100F900099F7EDCF08951F920F920FB60F9211247B
:100FA0000BB60F922F933F934F935F936F937F9363
:100FB0008F939F93AF93BF93EF93FF938091940090
:100FC000909195009093F1378093F03781E0809372
:100FD000E23780917100807D809371000E940984C6
:100FE0008091E2378823D9F1809194009091950007
:100FF0004091F0375091F13784179507A0F4809114
:10100000B6379091B737A091B837B091B9378C57B0
:10101000914EAF4FBF4F8093B6379093B737A093A1
:10102000B837B093B9372091940030919500241BC4
:10103000350B8091B6379091B737A091B837B09102
:10104000B937820F931FA11DB11D8093B6379093BE
:10105000B737A093B837B093B9371092E237FF9102
:10106000EF91BF91AF919F918F917F916F915F9120
:101070004F913F912F910F900BBE0F900FBE0F908D
:101080001F9018959FB7F894E1E7F0E08081807D8C
:10109000808388B38F6288BB10929000E1E9F0E012
:1010A000108210929200109295001092940080810C
:1010B000856080839FBF08959C019FB7F89430930B
:1010C00099002093980088B38F6288BBE1E7F0E035
:1010D0008081826080839FBF0895CF93DF93FC015E
:1010E000DB0185E0EB0119928A95E9F78581837030
:1010F00011F082E08C938781837021F082E0129658
:101100008C9312978581837081F08781837069F059
:1011100023893489818592852817390731F481E044
:10112000848312961C92129701C014828581837069
:10113000823029F0833011F488E001C080E01196FC
:101140008C93119787818370823029F0833011F45A
:1011500088E001C080E013968C93DF91CF910895D1
:10116000CF93DF9300D000D01F92CDB7DEB7BE0182
:101170006F5F7F4F0E946D8899818A81890F8D5F93
:101180009B81890F9C81890F9D81890F0F900F9002
:101190000F900F900F90DF91CF9108954F925F9233
:1011A0006F927F928F929F92AF92BF92CF92DF9277
:1011B000EF92FF920F931F93CF93DF9300D000D055
:1011C00000D0CDB7DEB78C017B01BE016F5F7F4FD2
:1011D0004E830E946D88B9815A80652D70E0AB8185
:1011E0004C80242D30E08B2F90E00396860F971FC4
:1011F0008A0F911D820F931F5D81850F911D4E8176
:1012000050E0481759070CF493C0F801818180FB26
:10121000882480F8912C83E0880C991C8A95E1F74A
:10122000828180FBAA24A0F8B12C94E0AA0CBB1CFC
:101230009A95E1F78A2880818770882A838180FBCC
:10124000CC24C0F8D12C45E0CC0CDD1C4A95E1F74C
:10125000C828848180FB662460F8712C56E0660CF7
:10126000771C5A95E1F76C28F7016082F8018581B7
:101270008370F4E08F9FA0011124F8019681937090
:10128000F0E19F9FC0011124842BF8014781F0E415
:101290004F9FA0011124842BF7018183F8018085E1
:1012A000F7018283B23051F4F8018185F70183831D
:1012B000F8018285F701848385E001C083E0580E40
:1012C000852D952D961B6115710561F06150710991
:1012D000A801460F571FFA014385F701E90FF11DD9
:1012E0004083EECFA23089F4F701E50DF11DD8015E
:1012F00053969C915397908391E0950DF701E90FD8
:10130000F11D8E5F54969C919083B42DB80F8B2F56
:101310009B2F921B2115310561F021503109F801F5
:10132000E20FF31F8589F701E90FF11D8083EFCFED
:1013300080E026960FB6F894DEBF0FBECDBFDF91DA
:10134000CF911F910F91FF90EF90DF90CF90BF90C2
:10135000AF909F908F907F906F905F904F90089587
:10136000BF92CF92DF92EF92FF920F931F93CF9392
:10137000DF93633008F4AEC0EA01D62E7C01FC0195
:10138000908196FBBB24B0F88181282F2695269565
:101390002370C82EC294C694C69453E0C522392F38
:1013A0003770388393FB332730F9398394FB332725
:1013B00030F93A8395FB992790F99B83BC822D8362
:1013C000829583708E83CF8282818887222379F1F0
:1013D0003381848190E0982F8827830F911D9A870D
:1013E000898787010B5F1F4F223071F46CE073E037
:1013F000CE010B960E94B25CF70186818B878581B6
:101400008C870E5F1F4F1EC02330E1F4F7013D961D
:10141000DE011B969E012D5E3F4F9E2F8F2F429126
:101420004D93A217B307D9F7092F182F0BC08701C7
:101430000D5F1F4F6CE073E0CE010B960E94B25C13
:101440001A861986CC20A1F1B1100DC0F8012081B7
:10145000818190E0982F8827820F911D9C8B8B8B28
:101460000E5F1F4F04C089859A859C8B8B8BF2E0A1
:10147000CF120EC06CE073E0CE0145960E94B25CC4
:10148000F80181818D8B80818E8B0E5F1F4F18C07C
:10149000F3E0CF1215C0085F1F4FD801FE0175960B
:1014A000CE014D962E912193E817F907D9F708C080
:1014B0006CE073E0CE0145960E94B25C1C8A1B8AE8
:1014C000C8018E199F092D2D281B2FA71EA70DA718
:1014D000D81608F480E0DF91CF911F910F91FF9013
:1014E000EF90DF90CF90BF900895FB0141505109DC
:1014F000460F571FE417F50778F4208130E0322FAC
:1015000022276181260F311D820F931F82179307B7
:1015100008F401963296EECFE417F50751F42081D6
:1015200030E0322F2227820F931F8217930708F48F
:1015300001960895CF93DF93C0911038D0E064975F
:1015400020910F3830E0322F2227C20FD31F48E0FE
:1015500050E069E178E39E01280F311DC9010E9426
:10156000758AAE0161E278E30E94758A009721F0E6
:1015700098278927982702C08FEF9FEFDF91CF919F
:1015800008959093431C8093421C0895FC0123818D
:10159000260F20930C38A72FBB2792819A0F909388
:1015A0000B38318130930A38408140930938E92F54
:1015B000F0E0EA17FB0748F481E0830F80930A38D4
:1015C000811103C04F5F4093093830E07727261719
:1015D000370788F49F5F90930B3891110CC080916E
:1015E0000A388F5F80930A38811105C080910938CD
:1015F0008F5F809309380895AB01BC0180E090E0D3
:101600000E94758A982789279827089544E150E019
:101610006DE078E380E090E00E94758A009721F009
:1016200098278927982708958FEF9FEF089586E0E0
:101630000C949A8A81E10C949A8A80E0E82FF0E079
:10164000EE0FFF1FEC56F24C118210828F5F843038
:10165000A9F780E090E2899FF0011124EC5EF24C42
:10166000118E8F5F8430B1F780E094E090933D1C41
:1016700080933C1C80E09DE0989FF0011124E6558A
:10168000F24C158214828F5F8A30B1F780933B1C35
:101690000895CF93DF93EC0120913C1C30913D1CC9
:1016A0002F5F3F4F21158DE7380710F020E030E124
:1016B000522F432FE4E1FDE390E0943059F0818D07
:1016C000882329F0A481B581A417B50749F39F5F4A
:1016D000B096F3CF30933D1C20933C1C10923B1CE2
:1016E00090E0E0E0F0E09430E9F080E2989FD001F3
:1016F0001124AC5EB24C59968C915997811104C05B
:1017000090933B1CFD0110C0873041F4309739F0B5
:101710005A962C915A97828D821708F0DF019F5FAD
:10172000FD01E1CF90933B1C309791F182E0818FD6
:1017300080913E1C848780913F1C85878091401C4E
:1017400086878091411C878788ED94E0938B828BFC
:10175000958B848B81E090E0918B808B138E828FB0
:1017600083E0808F168A80E1878B20913C1C30912A
:101770003D1C3227232732273583248377836683D2
:1017800088819981AA81BB8180839183A283B3835D
:10179000CF01DF91CF9108950F931F93CF93DF93E4
:1017A000DC0120913C1C30913D1C2F5F3F4F2115E7
:1017B0008DE7380710F020E030E1522F432FEAEA9E
:1017C000FDE390E09A3041F0C481D5819F5F3D9662
:1017D000C417D507B9F7E9CF30933D1C20933C1CC3
:1017E00090E08DE09A30D1F0492F50E021E0290FB0
:1017F000849FF001859FF00D1124E655F24CEF0116
:10180000249604811581012B39F490933B1C309769
:1018100041F480E090E02CC0922FE4CF90933B1CE9
:10182000F8CF20913C1C30913D1C322723273227D2
:101830003983288377836683109729F41082118275
:101840001282138209C08D919D910D90BC91A02DA3
:1018500080839183A283B3838DE0849FD001859F91
:10186000B00D1124A655B24C80E418968C93CF018C
:10187000DF91CF911F910F9108959C0190E09430DA
:10188000A1F0E92FF0E081E0890FEE0FFF1FEC5689
:10189000F24C408151814217530729F490933B1C2D
:1018A000118210820895982FEACF90933B1C0895DF
:1018B0009C0190E0943099F0E92FF0E081E0890FED
:1018C000EE0FFF1FEC56F24C40815181452B29F45D
:1018D00090933B1C318320830895982FEBCF9093F6
:1018E0003B1C0895AF92BF92CF92DF92EF92FF928E
:1018F0000F931F93CF93DF93C091123DD091133D6F
:10190000843009F4DBC125E338E33093113D2093A3
:10191000103D3093083820930738833059F4898D6F
:101920008F70833009F06AC088899989892B09F002
:10193000D5C67EC0823009F07FC08091411C8F5F88
:101940008093411C811113C08091401C8F5F809354
:10195000401C81110CC080913F1C8F5F80933F1C05
:10196000811105C080913E1C8F5F80933E1C1092B8
:101970000638109205381092A93D1092A83D898D25
:10198000982F9D7F953041F48A8D8F5F8A8F8431A7
:1019900009F0A4C6198EA2C6882309F49FC6288917
:1019A0003989232B09F440C09A8D2FEF290F2A8FF4
:1019B000911194C69B8D983031F02FEF280F223073
:1019C00048F4953039F4198E80E880930D3D0E94DB
:1019D000EC863DC5953038F423E0092E01C0220F76
:1019E0000A94EAF701C020E32A8F9F5F9B8F8F70D4
:1019F0008330A1F048F4813009F445C3823009F006
:101A00006DC610922E3842C3863009F4BCC48830AB
:101A100009F4B9C4843009F061C6B5C484E0809388
:101A20000D3D0E94EC8645C58F70833009F056C687
:101A300088E080930D3D00C5853019F5E0910E3D9D
:101A4000F0910F3D84819581892B09F447C610924E
:101A5000133D1092123D89E298E39093113D8093DB
:101A6000103D90930838809307381092A93D10924A
:101A7000A83D109206381092053888E080930D3DFD
:101A80001BC180910D38853409F028C600910F38AC
:101A900010E0102F002780911038080F111D809141
:101AA0000538909106388017910708F417C61093EF
:101AB000063800930538809113388F7309F00EC6ED
:101AC000F0901438F1100AC68091A43D9091A53D84
:101AD000C0916903D0916A038C179D0759F4409116
:101AE000A63D5091A73D20916B0330916C034217A6
:101AF0005307A1F020911D3830911E38281739075F
:101B000009F0ECC520911F38309120388091A63D16
:101B10009091A73D2817390709F0E0C50E94068B70
:101B2000019609F0DBC580911638863009F429C189
:101B30008131E9F1813009F0D1C5809121388830B7
:101B400009F0CCC510922138809123389091243827
:101B5000873F6FEF960710F0099601C008969093A3
:101B60002438809323388091193890911A38A091A5
:101B70001B38B0911C3880931D3890931E38A09369
:101B80001F38B09320388091A43D9091A53DA0913D
:101B9000A63DB091A73D8093193890931A38A09331
:101BA0001B38B0931C3880E48093153874C50C51F1
:101BB0001109109306380093053889E298E3909351
:101BC000113D8093103D8091273890912838892BC2
:101BD00029F00E941A8B019609F080C520912338C4
:101BE000309124382115310509F478C58AEA9DE33E
:101BF00090930F3D80930E3DA0902138B0902238F5
:101C000040916D0350916E0360916F03709170036A
